:100000000C9456070C9487070C9487070C94870769
:100010000C9487070C9487070C9487070C94870728
:100020000C9487070C9487070C9487070C94870718
:100030000C9487070C94227B0C9487070C948707F9
:100040000C9487070C9487070C9487070C948707F8
:100050000C9487070C9487070C9487070C940179FC
:100060000C9487070C94A2760C9478760C948707EE
:100070000C9487070C9487070C9487070C948707C8
:100080000C9487070C9487070C9487070C948707B8
:100090000C9487070C9487070C9487070C94997D20
:1000A0000C9487070C9487070C9487070C94870798
:1000B0000C9487070C9487070C9487070C94870788
:1000C0000C9487070C9487070C9487070C94870778
:1000D0000C9487070C9487070C9442760C9418763E
:1000E0000C9487070C94066E0C941D6E0C94E76DAF
:1000F0000C94866E0C94F1070C94F9070C94EF6D38
:100100000C94770B0C94500C0C94A06E0C94E36D33
:100110000C94106E0C94F70A0C9482130C94F26DEC
:100120000C94726D0C94B7630C940E130C94DF0B4B
:100130000C941C6F0C940A6E0C941F0A0C94D80A31
:100140000C941F080C941E6E0C945A860C94B507E0
:100150000C94728A0C94846C0C94AC920C94FA07F4
:100160000C94B9070C9451120C9464100C941A0856
:100170000C94776E0C94B1070C94D0070C940C7D02
:100180000C94CD6E0C94FC6E0C94996E0C94509261
:100190000C94856C0C94E5110C94326F0C94836C68
:1001A0000C94B26C0C9489070C94FF0C0C943614CC
:1001B0000C94146E0C9417140C9460750C94E60750
:1001C0000C9450860C94310D0C94710C0C941F5DA2
:1001D0000C94C9070C94826C0C94186E0C94D56C1A
:1001E0000C9484190C94E36C0C94838A0C94FC6D2D
:1001F0000C94766E0C94620A0C94070A0C94100806
:100200000C94256D0C94C90C0C94EB6D0C94226E1F
:100210000C94F86D0C94DD6D0C94026E0C94ED133F
:100220000C941C080C949B070C94A60C0C94F10FD6
:100230000C94D9190C94C16C0C94730B0C943187E9
:100240000C94210B4E414E494E495459494E46CDCE
:10025000CCCC3D0AD7233C17B7D13877CC2B32957D
:1002600095E6241FB14F0A000020410000C842005B
:10027000401C4620BCBE4CCA1B0E5AAEC59D740025
:10028000407A10F35A00A0724E18090010A5D4E865
:100290000000E87648170000E40B54020000CA9AF8
:1002A0003B000000E1F5050000809698000000404A
:1002B000420F000000A0860100000010270000008F
:1002C00000E803000000006400000000000A0000D5
:1002D0000000000100000000002C76D888DC674F89
:1002E0000823DFC1DFAE59E1B1B796E5E3E453C6B9
:1002F0003AE651997696E8E6C28426EB898C9B62B1
:10030000ED407C6FFCEFBC9C9F40F2BAA56FA5F45A
:1003100090055A2AF75C936B6CF9676DC11BFCE082
:10032000E40D47FEF520E6B500D0ED902E030094D5
:100330003577050080841E080000204E0A0000006A
:10034000C80C333333330F986E12831141EF8D2174
:1003500014893BE65516CFFEE6DB18D1844B381BDB
:10036000F77C1D901DA4BBE424203284725E2281A0
:1003700000C9F124ECA1E53D27436F6E74656E74EE
:100380002D547970653A20746578742F68746D6C9B
:100390000D0A0D0A3C68313E45504943204641490B
:1003A0004C3C2F68313E00485454502F312E3020A1
:1003B0003430302042616420526571756573740D6C
:1003C0000A004163636573732D436F6E74726F6CC3
:1003D0002D416C6C6F772D4F726967696E3A202AD8
:1003E0000D0A436F6E74656E742D547970653A20F2
:1003F000005365727665723A205765626475696E5E
:100400006F2F312E370D0A00485454502F312E30A3
:1004100020323030204F4B0D0A00436F6E6E656303
:1004200074696F6E3A20636C6F73650D0A436F6E6B
:1004300074656E742D547970653A206170706C69C2
:10044000636174696F6E2F782D7777772D666F7281
:100450006D2D75726C656E636F64656400506F73AB
:1004600074206661696C65640055706C6F6164200E
:100470004661696C65643A2000234E6F2073656E97
:10048000736F7220666F722074656D70202620680D
:10049000756D696469747921004E6F2053656E73C0
:1004A0006F72210020666F722074656D70202620A7
:1004B00068756D696469747921002353656E736F83
:1004C00072204572726F72200053656E736F7220D6
:1004D0004572726F7221002357726F6E67207365C9
:1004E0006E736F7220666F722074656D70202620A7
:1004F00068756D6964697479210057726F6E672041
:1005000053656E736F7221004320483D00543D00D7
:1005100020202020202020202020202020202020DB
:1005200000202020202020202020202020202020EB
:1005300020002020202020202020202020202020DB
:1005400020200020202020202020202020202020CB
:1005500020200020202020202020202020202020BB
:1005600020200054696D657374616D702075706C26
:100570006F6164206661696C6564005365747469B9
:100580006E6720636C6F636B2074696D6500236513
:1005900072726F72202D2000495020616464726570
:1005A00073733A2000496E76616C696420534D2064
:1005B00073746570732070657220616E676C653D41
:1005C00000534D2073746570732070657220616EE6
:1005D000676C653D003C703E54696D653A20003C97
:1005E0002F68333E0A003C62723E4254206E616DB9
:1005F000653D003C62723E506174683D003C68336A
:100600003E53797374656D3A2056657273696F6EE7
:100610003D00506172616D6574657273207265731F
:10062000657420646F6E6521002F6F652F736D6C8C
:1006300069676874706F2F73332F00616E676C6524
:1006400020646972656374696F6E3A200043757245
:1006500072656E7420534D206973202300534D3A08
:100660005461626C652073746570732070657220CC
:10067000616E676C653D00534D3A506F6C617269F5
:100680007A65722073746570732070657220616E74
:10069000676C653D002344485450494E3D00234457
:1006A00048543D00236E65743D424C4500236E6501
:1006B000743D5769466900236E65743D42540023BA
:1006C00066747020757365726E616D653A003A00EC
:1006D00023486F73742073657276657220495020C9
:1006E000616E6420506F72743A002354696D652006
:1006F0007365727665722049503A002352656C61C9
:100700007920646576696365733A002352656C618C
:100710007920737461747573206C6162656C733ACF
:1007200020002352656C6179207374617465733A9B
:10073000002352656C61792070696E733A00234E14
:100740006F2E206F6620636F6E74726F6C207265FF
:100750006C6179733D00234E6F2E206F66207265A9
:100760006C6179733D0046696E64696E67205769F4
:100770004669204950004E45543D426C7565746F82
:100780006F7468204C45004E45543D426C7565744D
:100790006F6F7468004E45543D5769466900534475
:1007A000206F70656E206661696C004E657720640D
:1007B00061746120636F6C6C656374696F6E207324
:1007C0007461727465640043757272656E7420732F
:1007D000657474696E67733A0053797374656D203C
:1007E000726573657420617420002344532054683B
:1007F00065726D6F6D657465722063616C6962729C
:100800006174656420666F72202300496E76616CA6
:10081000696420616E676C6520666F7220002073CA
:10082000746570732070657220616E676C653D0041
:100830002073746570732070657220616E676C65DB
:100840003D005461626C6520536574203000235470
:1008500075726E7461626C6520536574203000504F
:100860006F6C6172697A6572205365742030002361
:10087000506F6C6172697A65722053657420300024
:100880005461626C65205365742030002354757286
:100890006E7461626C6520536574203000506F6C1B
:1008A0006172697A65722053657420300023506F3D
:1008B0006C6172697A6572205365742030005769E3
:1008C00046692049503A00234C6F67676572204E95
:1008D000616D653A20004C4F4747455200564552DE
:1008E00053494F4E005265626F6F74696E672E2ECA
:1008F0002E005245424F4F54005365727665722068
:10090000506F727420757064617465640053504F49
:1009100052543D0049502075706461746564005301
:1009200049503D002354696D6520536572766572A8
:1009300020495020757064617465640054534950B7
:100940003D004352454C41590044485450494E3DA6
:100950000074696D6520696E74657276616C3D0026
:1009600054494D455354414D503D0054494D455314
:1009700054414D500023776562736572766572202D
:10098000626567696E730053657474696E672049A8
:10099000500053657474696E6720446576696365B9
:1009A000204950202E2E2E00506F6C6172697A659E
:1009B000722053657420300023506F6C6172697A25
:1009C00065722053657474696E6720302E2E2E0078
:1009D00054657374204C616D70732F46616E7300A3
:1009E0006572726F72206F70656E696E67206669DE
:1009F0006C653A20004C616D70204D6F746F720011
:100A00002354696D652020202020204461746520D6
:100A1000202020205365636F6E647320506F6C61DB
:100A200072697A6572205461626C652054286F4344
:100A3000292048282529202000696E69742E206409
:100A40006F6E652E00534420696E69742E206661B6
:100A5000696C65642100696E69742E206661696C39
:100A6000656421002323204F452057656C636F6D1B
:100A70006520232300496E697469616C697A696E27
:100A80006720534420636172642E2E2E0075706CB3
:100A90006F616420627920465450206661696C65FC
:100AA00064210075706C6F61642062792046545037
:100AB000204F4B210053797374656D2073746172FC
:100AC00074696E672E2E2E003C703E4C616D702056
:100AD000616E64204D6F746F722044726976657226
:100AE0007320537461747573EFBC9A3C2F703E0091
:100AF0003C21646F63747970652068746D6C3E3C52
:100B000068746D6C3E3C686561643E3C6D65746103
:100B100020636861727365743D227574662D382296
:100B20003E3C7469746C653E4F6E6C696E65206501
:100B300078706572696D656E74202D20506F6C61E0
:100B400072697A6174696F6E206566666563747335
:100B5000206F66206C696768743C2F7469746C65DB
:100B60003E3C2F686561643E3C626F64793E3C6840
:100B7000313E4F6E6C696E65206578706572696D87
:100B8000656E74202D20506F6C6172697A61746992
:100B90006F6E2065666665637473206F66206C698E
:100BA0006768743C2F68313E003C68343E436F7088
:100BB000797269676874284329323032302D3230B7
:100BC00032322E50726F662E205945554E472059AD
:100BD0006175205975656E3C2F68343E3C2F626FFD
:100BE00064793E3C2F68746D6C3E003C68313E4336
:100BF000616E6E6F74206765742073656E736F72BB
:100C00002072656164696E6773213C2F68313E0014
:100C10007C3C3E5E2B3D3F2F5B5D3B2C2A225C00E3
:100C200000002100240027002A002D00300033009E
:100C300001010000040107010A0100002200250053
:100C400028002B002E0031003400020100000501B5
:100C500008010B01000020002300260029002C00C1
:100C60002F00320000010000030106010901050503
:100C70000505070508080808020202020A0A080812
:100C80000404040401010101010101010303030340
:100C900003030303040707070C0C0C0C0C0C0C0CCF
:100CA0000202020206060606060606060B0B0B0BE0
:100CB0000B0B0B0B01021020200808102040102005
:100CC0004080020102010804020101020408102010
:100CD000408080402010080402018004020180400E
:100CE0002010080402010804020101020408102077
:100CF0004080010204081020408000000A0B020915
:100D00000C0D0E08070304010000000000000000A5
:100D100000000000000000000000000000000000D3
:100D20000000000000001211100000000000000090
:100D300000000000000000000000000000000000B3
:100D400053797374656D2072657374617274656430
:100D500021002053797374656D207265737461721C
:100D600074656421004E6574776F726B206D6169E4
:100D70006E7461696E656420617420002323436F83
:100D80006D6D616E644000417070656E64206D65CC
:100D900061732E200053696E676C65206D65617309
:100DA0002E200053617665206D6561737572652034
:100DB000746F3A0020202020202020202020202096
:100DC000202020200000000100010010100200017E
:100DD000000100B000000016000000280000001014
:100DE00000000020000000010001000000000000E1
:100DF00000000000000000000000000000000000F3
:100E000000000000000000FF000000FFFF0000FFE6
:100E1000FF0000FFFF0000CFBF0000C7BF0000C3FE
:100E2000BF0000C1BF0000C0BF000000000000C044
:100E3000BF0000C1BF0000C3BF0000C7BF0000CF9C
:100E4000BF0000FFFF0000FFFF00000000000000E7
:100E50000000000000000000000000000000000092
:100E60000000000000000000000000000000000082
:100E70000000000000000000000000000000000072
:100E80000000000000000000000000557365722D96
:100E90006167656E743A202A0D0A446973616C6C4F
:100EA0006F773A202F0D0A00AC92509211241FBE8A
:100EB000CFEFD1E2DEBFCDBF00E00CBF1AE0A0E073
:100EC000B2E0E6EEFBE501E00BBF02C007900D9239
:100ED000AA31B107D9F725E1AAE1BAE001C01D9214
:100EE000A935B207E1F717E0C5E5D7E000E006C095
:100EF00021970109802FFE010E94FAAAC435D1076B
:100F000080E00807A9F70E944C950C94E1AD0C9481
:100F10000000CF93DF93EC01898D9A8D892B41F0EE
:100F2000E881F9810284F385E02DCE011995F4CF93
:100F3000DF91CF910895CF93DF931F92CDB7DEB7A6
:100F40006983DC01ED91FC910280F381E02D41E0A9
:100F500050E0BE016F5F7F4F19950F90DF91CF91E9
:100F60000895FC01818D928D0895FC0184899589F5
:100F7000089527E134E0FC0131832083FB0140899F
:100F8000518962897389FC01428353836483758329
:100F90000895DC01ED91FC91048CF58DE02D199400
:100FA000CF93DF931F92CDB7DEB76983DC01ED915C
:100FB000FC910280F381E02D41E050E0BE016F5FC3
:100FC0007F4F19950F90DF91CF910895FC01948583
:100FD000FB018485981303C081E0943009F480E01C
:100FE000089521E0FC018485843009F420E0822FFB
:100FF00008950895CF93DF931F92CDB7DEB769832D
:10100000DC01ED91FC910280F381E02D41E050E0A4
:10101000BE016F5F7F4F19950F90DF91CF910895BB
:10102000DC01ED91FC91068CF78DE02D199591E096
:1010300089270895862F089581E08627089590E0F6
:1010400080E0089590E0982F882744E050E0845F86
:101050009B4F0C94EF8DEF92FF920F931F93CF93C2
:10106000DF93182FC6EFDBE061E08A810E943B77B7
:101070006091B50B8A810E94D87664EF71E080E0C0
:1010800090E00E94917722968BE0CC3FD80761F7E1
:10109000112309F44AC008EF1BE0E8017E016091CA
:1010A000B70B88810E94D87668EE73E080E090E00C
:1010B0000E9491776091B70B8A810E94D87668EE82
:1010C00073E080E090E00E94917722966091B50BEA
:1010D000D7018C910E94D87668EE73E080E090E0B2
:1010E0000E949177BBE0CC3FDB07C1F668EE73E06E
:1010F00080E090E00E949177C1EDD2E0E991F99112
:10110000D8018C910E5F1F4FEE0FFF1FEB54F44F71
:1011100060810E94D87668EC70E080E090E00E94E8
:101120009177B2E0C73DDB0749F7DF91CF911F917F
:101130000F91FF90EF9008959F92AF92BF92CF9240
:10114000DF92EF92FF920F931F93CF93DF935C0197
:101150007B018B01D0E0C0E0F80191908F01650127
:10116000CC0EDD1EC6010E943EA9981621F0692D05
:10117000C6010E9446A92196C233F1E0DF0761F75C
:10118000C701DF91CF911F910F91FF90EF90DF90FA
:10119000CF90BF90AF909F90089581E08093EF0231
:1011A0008091F002882341F088E08093641160E030
:1011B00089E591E10C94DF7C08958091F002882309
:1011C000F9F08091EF028823D9F081E00E94237D1D
:1011D0008BE39FE10197F1F760E080E00E94347DAE
:1011E00063E575E089E591E10E94E87561E080E0E2
:1011F0000E94347D63E475E089E591E10C94E87523
:1012000008950F931F93CF93DF932091F002222331
:1012100009F45CC02091EF02222309F457C0EA01CF
:101220008C016F3F7F4FF1F461E080E00E94347DDC
:10123000B80189E591E10E94C67562E375E089E530
:1012400091E10E94E87561E0F80184810E94347D9B
:10125000BE01DD0F880B990BDF91CF911F910F918C
:101260000C9491770E944F78AB01BC018091E70A02
:101270009091E80AA091E90AB091EA0A8C599F4F2F
:10128000AF4FBF4F84179507A607B707F8F461E083
:1012900080E00E94347DB80189E591E10E94C67525
:1012A00061E275E089E591E10E94E87561E0F8018D
:1012B00084810E94347D0E944F786093E70A709386
:1012C000E80A8093E90A9093EA0AC2CFDF91CF91AE
:1012D0001F910F9108952C9A08952C9808958EBD12
:1012E00000000DB407FEFDCF8EB508959B0190E080
:1012F0000496982F8827642F820F931F0C94998F40
:10130000CF93DF93C82FD62F472F60E170E00E9464
:1013100076094D2F61E170E08C2FDF91CF910C9415
:101320007609CF93DF93C82FD0E02496DC2FCC270B
:10133000C60FD71F0E946D098FE00E946F098D2F85
:101340000E946F098C2F0E946F0980E00E946F0934
:10135000C82F0E946B098C2FDF91CF9108951F93A6
:10136000CF93DF93182F66E270E00E949109C82F97
:1013700067E270E0812F0E9491099C2FDF91CF914D
:101380001F9108951F93CF93DF93182F60E270E0B1
:101390000E949109C82F61E270E0812F0E9491099B
:1013A0009C2FDF91CF911F91089544E050E0BC0144
:1013B0008FE090E00C94EF8D08958CBD9DBD089555
:1013C000EF92FF920F931F93CF93C82F7B0180E57D
:1013D00090E00E94DD0968E270E08C2F0E94910984
:1013E000082F69E270E08C2F0E949109282F302F7E
:1013F000B90121E030E0A7018C2F0E94777181E0D4
:1014000090E0CF911F910F91FF90EF900895CF93AF
:10141000DF931F92CDB7DEB7FC01218D328D8FEFA8
:101420009FEF232B41F0BE016F5F7F4F808D0E94A5
:10143000E009898190E00F90DF91CF9108950F939B
:101440001F93CF93DF931F92CDB7DEB78C01DC01E2
:10145000ED91FC910084F185E02D1995892B79F0AF
:10146000BE016F5F7F4FF80184850E94E00989818A
:1014700090E00F90DF91CF911F910F9108958FEF22
:101480009FEFF7CFFF920F931F93CF93DF93F82E29
:1014900080E590E00E94DD0910E000E08F2D0E94C1
:1014A000AF09EC01892B21F08F2D0E94AF098C012F
:1014B000C017D10799F7CE01DF91CF911F910F91FE
:1014C000FF900895FC018485843011F00C94420A49
:1014D00090E080E00895AF92BF92CF92DF92EF92BA
:1014E000FF921F93CF93DF93182F6B017A0180E552
:1014F00090E00E94DD09B12CA12C812F0E94AF0940
:10150000EC01892B21F0812F0E94AF095C01CA15E3
:10151000DB0599F72097E9F463E070E0812F0E94E2
:101520009109843159F0882349F0C1E0D0E08C3131
:1015300011F4D0E0C0E0D195C195D109CE01DF9181
:10154000CF911F91FF90EF90DF90CF90BF90AF9021
:101550000895EC16FD060CF4E7011C161D0674F741
:1015600068E270E0812F0E949109E82E69E270E044
:10157000812F0E949109282F3E2D79019E01A601FD
:10158000B701812F0E947771EC0EFD1E4F2D68E28E
:1015900070E0812F0E9476094E2D69E270E0812F64
:1015A0000E94760960E470E0812F0E944B71C6CFE3
:1015B000CF93DF93FC01218D328D2115310529F464
:1015C0008FEF9FEFDF91CF910895EC01808D42174F
:1015D000530708F0A9010E946B0A1816190684F730
:1015E000298D3A8D281B390B3A8F298FEBCF0F931A
:1015F0001F93CF93DF931F92CDB7DEB7FC01218DF0
:10160000328D232B41F48FEF9FEF0F90DF91CF911D
:101610001F910F9108958C0141E050E0BE016F5F72
:101620007F4FFC01808D0E946B0A181619065CF72B
:10163000F801818D928D0197928F818F898190E041
:10164000E4CF0F931F93CF93DF9300D000D01F926E
:101650001F92CDB7DEB78C01DC01ED91FC910680C5
:10166000F781E02D1995F801808D0E94420A181625
:101670001906B4F548E050E0BE016F5F7F4FD80116
:1016800058968C910E946B0A18161906F4F4D8012A
:10169000509684E0FE01319601900D928A95E1F713
:1016A0008D8190E0982F88272E81820F911DF8015F
:1016B000958B848B8F81282F30E0322F22278885CD
:1016C000820F932F911D928F818F28960FB6F894D9
:1016D000DEBF0FBECDBFDF91CF911F910F91089557
:1016E00090E080E0F2CFFC0184850C946B0ACF93EC
:1016F000DF931F92CDB7DEB741E050E0BE016F5FD0
:101700007F4FFC0184850E946B0A1816190634F479
:10171000898190E00F90DF91CF9108958FEF9FEF37
:10172000F9CFCF93C82F80E590E00E94DD0960E1FA
:1017300070E08C2F0E944B714FEF62E070E08C2FB5
:10174000CF910C947609FF920F931F93CF93DF9361
:10175000C82FD62F8A01F22E0E94910B80E590E0CF
:101760000E94DD094D2F4F2970E060E08C2F0E9410
:10177000760901151105C1F0412F64E070E08C2F4E
:101780000E947609402F65E070E08C2F0E94760958
:1017900061E070E08C2F0E944B7181E0DF91CF916E
:1017A0001F910F91FF9008950091FF0B1091000C75
:1017B0000F5F1F4F1093000C0093FF0BDDCFBF9204
:1017C000CF92DF92EF92FF920F931F93CF93DF930D
:1017D00000D000D0CDB7DEB7FC01208D243009F059
:1017E0005DC06A017B018C01B12C63E070E08B2D40
:1017F0000E94910981114AC0F801B08EF801808DD4
:10180000843009F44BC096E0EBEFF2E0DE01119674
:1018100001900D929A95E1F7F70193819F779C8350
:1018200094819D8395819E83B7016E5F7F4F0E9457
:101830002208B601F801808D0E948009F801808D90
:1018400090E0982F882746E050E0BE016F5F7F4F01
:101850008A5F9B4F0E94EF8DF801128E118E20E857
:10186000A60162E0808D0E94A30B81E026960FB650
:10187000F894DEBF0FBECDBFDF91CF911F910F91C6
:10188000FF90EF90DF90CF90BF900895883109F4DA
:10189000B3CFB394F4E0BF12A8CFB0CF80E0E6CFCF
:1018A000CF93DF93EC01888D843061F00E94910B1F
:1018B000E88DF0E0EE0FFF1FE65DF34F118210821E
:1018C00084E0888FDF91CF910895CF93C82F80E572
:1018D00090E00E94DD0963E070E08C2FCF910C94C2
:1018E0009109EF92FF921F93CF93DF93FC01208D1C
:1018F000243039F080E0DF91CF911F91FF90EF907D
:1019000008957B01EC0110E0812F0E94650C81118C
:101910000FC0188F888D843069F3FD86EC861A8E8F
:10192000198E20E0A70162E00E94A30B81E0E3CFC3
:10193000883179F31F5F143039F7ECCFFC018485CF
:10194000843011F00C94650C80E00895CF93DF9300
:10195000FC0124852430D9F0EC010E949E0C8431D6
:1019600089F0882379F0883169F021E08C3159F4CD
:10197000E881F9810084F185E02DCE01199521E0FF
:10198000892B09F420E0822FDF91CF91089580E028
:10199000FBCFAF92BF92CF92DF92FF920F931F9334
:1019A000CF93DF938C015B01EA01FC01C688D788E5
:1019B000F08C80E590E00E94DD098F2D0E945B7124
:1019C0008C179D0720F48F2D0E945B71EC019E0106
:1019D000A501B6018F2D0E941E8EF8018689978978
:1019E0008C0F9D1F978B868BCE01DF91CF911F911E
:1019F0000F91FF90DF90CF90BF90AF900895CF935D
:101A0000FC01C08D80E590E00E94DD0960E270E09D
:101A10008C2F0E944B7162E070E08C2F0E94910924
:101A200084FD16C062E070E08C2F0E94910983FF54
:101A30000AC048E162E070E08C2F0E94760990E0D5
:101A400080E0CF91089580E590E00E94DD09E3CF2A
:101A500040E162E070E08C2F0E94760981E090E026
:101A6000F0CFFF920F931F93CF93DF93EB01FC0115
:101A7000178A168A2A81211109C02B81211106C0DB
:101A80002C81211103C02D812223E1F04115510544
:101A9000C9F08A01FC01F08C80E590E00E94DD092C
:101AA000BE016E5F7F4F8F2D0E942208B8018F2DDF
:101AB0000E94800981E090E0DF91CF911F910F910A
:101AC000FF90089590E080E0F7CF4F925F926F9281
:101AD0007F928F929F92AF92BF92CF92DF92EF92BE
:101AE000FF920F931F93CF93DF93CDB7DEB763972A
:101AF0000FB6F894DEBF0FBECDBF7C016B013A017B
:101B0000FB0120E090E080E06AE03191332309F4AA
:101B100061C040ED430F4A3008F04DC0689FA001FE
:101B2000699F500D1124CA01C097830F911D37FD85
:101B30009A958F3F910549F340F3F7014281538114
:101B40006481758180913A0E90913B0EA0913C0E7C
:101B5000B0913D0E481759076A077B0709F439C24F
:101B60008701085F1F4F0E944F786F7077277C5F57
:101B7000C8010E94710C813009F030C287E194E005
:101B80009A838983F70182819381A481B5818B83B4
:101B90009C83AD83BE8345E350E0BE016F5F7F4F02
:101BA000C8010E94310D892BA9F5D12CC12CC80187
:101BB0000E94500C17C03E3209F0BFCF233009F409
:101BC000BCCFD301A20FB11D12968C932F5F90E072
:101BD00080E09BCF233009F0B0CFF3018583CC2484
:101BE000C394D12CC60163960FB6F894DEBF0FBE26
:101BF000CDBFDF91CF911F910F91FF90EF90DF90BC
:101C0000CF90BF90AF909F908F907F906F905F909C
:101C10004F9008950E944F78F70177836683762767
:101C2000672776277A83698342E050E0BE016F5FC1
:101C30007F4FC8010E94C90C81E090E09E878D878C
:101C400042E050E0BE01635F7F4FC8010E94C90CB3
:101C500080E091E09E878D8742E050E0BE01635FA7
:101C60007F4FC8010E94C90C1E861D8642E050E0CD
:101C7000BE01635F7F4FC8010E94C90C42E050E083
:101C8000BE01635F7F4FC8010E94C90C42E050E073
:101C9000BE01635F7F4FC8010E94C90C5601F60167
:101CA0008081882301F16501F60181912F0188234C
:101CB00011F08E32B1F446018A189B0818141904E9
:101CC00074F48F8641E050E0BE01615F7F4FC80130
:101CD0000E94C90CA401B501C8010E94C90C52019F
:101CE000DECF6201E1CF1F8641E050E0BE01615FBF
:101CF0007F4FC8010E94C90CC12CDD24D394DE861D
:101D0000CD8642E050E0BE01635F7F4FC8010E9474
:101D1000C90CDE86CD8642E050E0BE01635F7F4F96
:101D2000C8010E94C90CC8010E94FF0C892B09F44C
:101D30003CCFF3E0AF2EB12C230122E0420E511C28
:101D40005EC0F7014281538164817581808D918DE0
:101D5000A28DB38D481759076A077B0709F02FC179
:101D6000848D958DC59709F02AC181A192A10C9708
:101D70000CF42AC14CE050E0BE016F5F7F4FC801F8
:101D80000E94D80A8B819C819827892798279A8B53
:101D9000898B29813A81322723273227F70146810F
:101DA000578142175307D1F497FF18C08F70927074
:101DB000892B09F042C06F807884762467247624CA
:101DC000D12CC12C6114710409F051C0C8010E94CA
:101DD00089076AEFC62EDD24DA9407C0C8010E9485
:101DE0008907ECEFCE2EDD24DA9481E0A81AB10841
:101DF00009F4DDCEFFEFCF16DF0609F0D8CE0E9442
:101E00004F783B014C01C8010E94210B181619069E
:101E10000CF497CF0E944F786619770988099909C1
:101E2000693873418105910508F0C5C062E370E02F
:101E300080E090E00E949177E6CFC8010E94890778
:101E40007BEFC72EDD24DA94D0CF8D85811117C0AA
:101E5000C8010E94F70AC8010E94F70AC8010E943F
:101E6000F70AC8010E94F70AFFEFCF1ADF0A8D8137
:101E70009E81982789279827C816D906A8F441E09B
:101E800050E0BE01635F7F4FC8010E94D80A8D8574
:101E90008823D9F28D859FEF980F9D878823A9F21B
:101EA000C8010E94F70AF6CF912C812C41E050E046
:101EB000BE016D5E7F4FC8010E94D80A8B89982FA2
:101EC000907C61F4882389F08B899FEF980F9B8B1E
:101ED000882341F0C8010E94F70AF6CFC8010E948A
:101EE000F70A1B8A8B898111E1CF42E050E0BE01E5
:101EF000615F7F4FC8010E94D80A42E050E0BE01F6
:101F0000635F7F4FC8010E94D80AC8010E94F70A88
:101F1000C8010E94F70AC8010E94F70AC8010E947E
:101F2000F70A42E050E0BE016F5E7F4FC8010E9499
:101F3000D80A8F85988981159140E9F4CD84DE8493
:101F4000DC24CD24DC2481E0C816D104A1F48989E5
:101F50009A898115944041F0C8010E94890757EF82
:101F6000C52EDD24DA9441CF44E050E0B201C8012F
:101F70000E94D80A3ACFD12CC12C89899A899827F6
:101F800089279827C816D90638F4C8010E94F70A8D
:101F9000FFEFCF1ADF0AF1CF2FEF821A920A6814EF
:101FA000790409F083CFC8010E94890746EFC42E47
:101FB000DD24DA941ACFCC24CA94DC2C16CF2EEF71
:101FC000C22EDD24DA9411CF9DEFC92EDD24DA94E0
:101FD0000CCF8EEFC82EDD24DA9404CED12CC12C88
:101FE00001CECF92DF92EF92FF920F931F93CF9388
:101FF000DF93CDB7DEB7AF970FB6F894DEBF0FBE55
:10200000CDBF7C016A0107E114E01A8309831C86B5
:102010001B8688EE93E0A0E0B0E08D879E87AF87B7
:10202000B88B8BEA93E09A878987188F0F8B198E6C
:102030001A8E1B8E1C8E84E089A31BA70AA71CA6E0
:102040001DA61EA61FA68091320E9091330EA09160
:10205000340EB091350E8EA39FA3A8A7B9A78B838A
:102060009C83AD83BE8318861F82AE01465D5F4FA1
:10207000CE0101960E94650D81309105B1F4D70122
:10208000ED91FC910488F589E02D1DA30CA38CA58E
:102090009DA5AEA5BFA58EA39FA3A8A7B9A7A6017E
:1020A000BE016C5D7F4FC7011995AF960FB6F894CE
:1020B000DEBF0FBECDBFDF91CF911F910F91FF907B
:1020C000EF90DF90CF900895CF92DF92EF92FF9242
:1020D0000F931F93CF93DF93CDB7DEB7AF970FB6B4
:1020E000F894DEBF0FBECDBF7C016A0107E114E0AA
:1020F0001A8309831C861B8688EE93E0A0E0B0E07B
:102100008D879E87AF87B88B8BEA93E09A87898704
:10211000188F0F8B198E1A8E1B8E1C8E84E089A34C
:102120001BA70AA71CA61DA61EA61FA68091320EDD
:102130009091330EA091340EB091350E8EA39FA3D3
:10214000A8A7B9A78B839C83AD83BE8318861F8203
:10215000AE01465D5F4FCE0101960E94650D813054
:102160009105B1F4D701ED91FC910684F785E02D3E
:102170001DA30CA38CA59DA5AEA5BFA58EA39FA353
:10218000A8A7B9A7A601BE016C5D7F4FC70119952D
:10219000AF960FB6F894DEBF0FBECDBFDF91CF91E3
:1021A0001F910F91FF90EF90DF90CF9008957F9255
:1021B0008F929F92AF92BF92CF92DF92EF92FF9257
:1021C0000F931F93CF93DF93CDB7DEB7A6970FB6CC
:1021D000F894DEBF0FBECDBF8C01762E942E852ED7
:1021E00020E2A22ECE0101967C01DC01EA2D1D9297
:1021F000EA95E9F76801F3E4CF0ED11C87E194E09A
:102200009AA389A38FEF8BA38CA38DA38EA343E402
:1022100050E0BE016F5D7F4FC6010E94310D0196F7
:1022200009F4BFC081E089838A8386E0B82EBB822F
:102230001C82D80114966D917D918D919C91179778
:102240000E9402AB6D837E838F83988789869A86EE
:1022500080E890E09C878B874CE150E0B701C60195
:102260000E94C90CFE0137968AE1DF011D928A9512
:10227000E9F74801B8E08B0E911CF401D7010190F9
:102280000D92BA94E1F740E150E0B701C6010E9417
:10229000C90CF7011192AA94E9F796E0A92EB12C86
:1022A00040E250E0B701C6010E94C90CF1E0AF1A4C
:1022B000B108B1F783E6898392E89A8393E59B831B
:1022C0008C8385E38D8381E08E837F829DE3988775
:1022D00097E099878A8786E0F401DE011B960190DA
:1022E0000D928A95E1F78CE0898B8A8B69E174E025
:1022F000CE0143960E9473ADD8011B966C91CE011E
:1023000049960E94BF71F8016485CE014B960E94E8
:10231000BF71D8011D966C91CE014D960E94BF7180
:102320004EE150E0B701C6010E94C90CB3E07B1238
:102330001EC082E3898384E08A83F80196859B83AB
:1023400097859C8390899D8391899E8396E39F8343
:102350008887828D8987838D8A87848D8B87858DF9
:102360008C874CE050E0B701C6010E94C90C87E39E
:10237000898386E08A8391E09B8393E09C838D83AD
:102380008FE08E838AE38F838BE388878FEF898743
:1023900049E050E0B701C6010E94C90CC6010E9485
:1023A000FF0CA6960FB6F894DEBF0FBECDBFDF912F
:1023B000CF911F910F91FF90EF90DF90CF90BF9042
:1023C000AF909F908F907F9008958F929F92AF9241
:1023D000BF92CF92DF92EF92FF920F931F93CF9312
:1023E000DF93CDB7DEB72D970FB6F894DEBF0FBEE3
:1023F000CDBF7C0110E000E038EE832E33E0932E59
:10240000A12CB12C43EDC42E43E0D42E1C821B82A0
:102410008D829E82AF82B886DA82C9820D87CE0114
:1024200001960E949E0C811135C0F70144815581AF
:1024300020E061E0802F0E94A30B80E590E00E94E5
:10244000DD0963E070E0802F0E949109833129F457
:1024500062E070E0802F0E944B71F70184819581CA
:10246000000F111FF801E65DF34F918380832D96D5
:102470000FB6F894DEBF0FBECDBFDF91CF911F9195
:102480000F91FF90EF90DF90CF90BF90AF909F9013
:102490008F9008950F5F1F4F0430110509F0B6CFDC
:1024A000E6CFCF92DF92EF92FF921F93CF93DF930D
:1024B000FC011485143089F1EC0180E590E00E9464
:1024C000DD0968E070E0812F0E944B710E944F7817
:1024D0006B017C01CE010E949E0C8823A1F061E07B
:1024E00070E080E090E00E9491770E944F786C1934
:1024F0007D098E099F09683E73408105910550F35F
:102500008C850E94910BEC85F0E0EE0FFF1FE65DDD
:10251000F34F1182108284E08C87DF91CF911F915D
:10252000FF90EF90DF90CF9008954F925F926F925F
:102530007F928F929F92AF92BF92CF92DF92EF9253
:10254000FF921F93CF93DF93CDB7DEB72D970FB6D2
:10255000F894DEBF0FBECDBF7C019AE2A92E9CE0AD
:10256000B92E10E0D12CC12C28EE422E23E0522EA1
:10257000612C712C33ED832E33E0932E1C821B8251
:102580004D825E826F8278869A8289821D87D5010C
:102590002D913D915D01F7018481958128173907BF
:1025A000B1F4CE0101960E949E0C843199F1CE01C6
:1025B00001960E949E0C8C3151F4CE0101960E942E
:1025C000620A892B21F4CE0101960E9451121F5FED
:1025D0001430A1F6CD2841F4D701ED91FC9100848F
:1025E000F185E02DC70119952D960FB6F894DEBF41
:1025F0000FBECDBFDF91CF911F91FF90EF90DF9085
:10260000CF90BF90AF909F908F907F906F905F9092
:102610004F900895CC24C394D12CD9CF8F929F9200
:10262000AF92BF92CF92DF92EF92FF920F931F93E0
:10263000CF936C015B017A01FC01C485C430A1F425
:1026400081E090E0F60193838283F12CE12CC701B5
:10265000CF911F910F91FF90EF90DF90CF90BF909F
:10266000AF909F908F9008958A014130584010F0AC
:1026700000E018E080E590E00E94DD098C2F0E94C8
:102680005B714C0163E070E08C2F0E9491098731EF
:1026900011F08C3129F58016910660F380E590E009
:1026A0000E94DD099801A50170E060E08C2F0E9476
:1026B0001E8E60E270E08C2F0E944B7162E070E031
:1026C0008C2F0E94910984FD13C063E070E08C2F71
:1026D0000E949109811107C08C2F0E94910BB0CFED
:1026E00010E000E0DBCF80E590E00E94DD09E6CF5E
:1026F00040E162E070E08C2F0E947609012B09F026
:10270000A6CF9ECF3F924F925F926F927F928F9211
:102710009F92AF92BF92CF92DF92EF92FF920F9370
:102720001F93CF93DF93CDB7DEB72D970FB6F894F5
:10273000DEBF0FBECDBF6C015B014A010E94951246
:102740008AE2E82E8CE0F82E312C10E000E098EEC2
:10275000492E93E0592E612C712C1C821B824D82D4
:102760005E826F82788683ED93E09A8389833D86CB
:10277000F701219131917F01F6018481958128171C
:10278000390771F4CE0101960E949E0C873141F405
:10279000A401B501CE0101960E940E13080F191F66
:1027A0003394F4E03F12D9CFC8012D960FB6F894B8
:1027B000DEBF0FBECDBFDF91CF911F910F91FF9074
:1027C000EF90DF90CF90BF90AF909F908F907F90D1
:1027D0006F905F904F903F900895CF92DF92EF926D
:1027E000FF920F931F93CF93DF938B017A016C01BC
:1027F00027EBC20ED11CF6014081EC012A9644233E
:1028000049F050E0BC0169567F4FCE010E940E1383
:10281000F6011082A701B801CE01DF91CF911F917F
:102820000F91FF90EF90DF90CF900C940E13CF9309
:10283000DF93EC01C954DF4FE88121E02E0F28839C
:10284000E80FF92FF11DE956FF4F6083203249F45C
:10285000BC0169567F4F40E250E00A960E940E1379
:10286000188281E090E0DF91CF910895CF92DF92BE
:10287000FF920F931F93CF93DF93FC0124852430A5
:1028800051F090E080E0DF91CF911F910F91FF9088
:10289000DF90CF9008956A01EB018C01F12C8F2D10
:1028A0000E94650C811129C0F801F486F801848525
:1028B000843039F320916802309169022F5F3F4FD5
:1028C00021F130936902209368024091680250918F
:1028D000690220E061E00E94A30B8A818F3FC1F46E
:1028E0008B818F3F01F58C818F3FE9F48D818F3F84
:1028F000D1F484E0F8018487C4CF8B7F8831A1F2C2
:10290000F394F4E0FF12CBCFD1CF20E030ECD9CF5D
:10291000811109C08B81811106C08C81811103C096
:102920008D81882331F3C114D10419F3F801F484A3
:1029300080E590E00E94DD09BE016E5F7F4F8F2D24
:102940000E942208B6018F2D0E94800964E070E089
:102950008F2D0E944B71C8010E949E0C873161F03F
:1029600061E070E080E090E00E949177C8010E94F1
:102970009E0C8111F0CFBDCF81E090E084CFCF934A
:10298000CFB7F8948091FE0B811127C0E3EAFCE0F9
:102990008491E9EEFCE09491E82FF0E0EE0FFF1F48
:1029A000E05EF34FA591B491EC91E92321F461E04D
:1029B00085E30E94D87661E085E30E943B778CB581
:1029C00080618CBD8CB580648CBD61E084E30E9425
:1029D0003B7761E083E30E943B778091FE0B8F5F42
:1029E0008093FE0BCFBFCF9108954F925F926F926D
:1029F0007F928F929F92AF92BF92CF92DF92EF928F
:102A0000FF920F931F93CF93DF93EC0118161906D3
:102A10001CF44C0104972CF0C1E0D0E063E0862E5A
:102A2000912C8E01000F111F7E01EE0CFF1CEE0C8D
:102A3000FF1C8C169D060CF4B3C097012C5B3D4F18
:102A40005901F90180819181A281B38197012152BD
:102A50003D4F6901181619061A061B063CF50E941F
:102A60007079F60140805180628073806419750925
:102A700086099709F501408051806280738046166F
:102A800057066806790658F4108211821282138262
:102A90000E947079F601608371838283938321960B
:102AA0000E5F1F4FF4E0EF0EF11CC3CF98012952C7
:102AB0003D4F3901F90180819181980121533D4FAA
:102AC0005901F9012081318182179307C1F0880FE4
:102AD000991FFC01EB54F44F6081F801EA50F44F68
:102AE00080810E94D876F30180819181F5019183E4
:102AF00080836CE271E080E090E00E949177F601C3
:102B000080819181A281B381181619061A061B06CD
:102B100034F60E947079F60120813181428153811F
:102B2000621B730B840B950BF701E154FD4F208161
:102B3000318142815381261737074807590708F02A
:102B4000AECFF601108211821282138298012C5AA4
:102B50003D4F6901F90180819181F5012081318129
:102B60008217930709F49BCF880F991FFC01EB5440
:102B7000F44F6081F801EA50F44F80810E94D876CA
:102B8000F60180819181F50191838083F301918326
:102B900080836CE271E080E090E00E9491777FCFCB
:102BA000DF91CF911F910F91FF90EF90DF90CF9029
:102BB000BF90AF909F908F907F906F905F904F905D
:102BC0000895CF93DF93FC0124813581232B69F095
:102BD000EC01BC018CE39DE00E94D475BE018FE93D
:102BE0009CE0DF91CF910C94D475DF91CF91089543
:102BF000CF93DF93FC0124813581232B69F0EC0115
:102C0000BC018CE39DE00E94C675BE018FE99CE08B
:102C1000DF91CF910C94C675DF91CF9108958F927B
:102C20009F92AF92BF92CF92DF92EF92FF920F935B
:102C30001F93CF93DF938C01862F0B30110509F082
:102C40009FC09091E210992309F0F89462E10E94EC
:102C5000C477EC018091E210882309F078942097E2
:102C600001F180E090ECA9E7B4EC8093D51090934B
:102C7000D610A093D710B093D8108093D91090930A
:102C8000DA10A093DB10B093DC10CE3F8FEFD807A3
:102C900009F4A9C0CF3FDC0709F462C0CCEFDFEF35
:102CA00030C1C091DD10E090DE106E2D70E090E03C
:102CB00080E00E9421A82DEC3CEC4CEC5DE30E94EE
:102CC00080A84B015C016C2F70E090E080E00E94D6
:102CD00021A89B01AC01C501B4010E94C8A9609361
:102CE000D5107093D6108093D7109093D810D091B0
:102CF000DF10F090E0106D2F6F7770E090E080E0D3
:102D00000E9421A84B015C016F2D70E090E080E0F3
:102D10000E9421A82DEC3CEC4CEC5DE30E9480A8C5
:102D20009B01AC01C501B4010E94C8A9D7FD26C012
:102D30006093D9107093DA108093DB109093DC10BD
:102D4000CE0DCD0FCF0D81E090E02091E110C213A8
:102D500002C090E080E0892B09F493C0CFEFDFEF51
:102D6000CE01DF91CF911F910F91FF90EF90DF90F7
:102D7000CF90BF90AF909F908F9008959058D8CFEC
:102D8000CFEFDFEF0631110509F0BBC09091E210E3
:102D9000992309F0F89461E00E94C477EC018091D6
:102DA000E210882309F07894209701F180E090ECFC
:102DB000A9E7B4EC8093D5109093D610A093D710C8
:102DC000B093D8108093D9109093DA10A093DB10B1
:102DD000B093DC10CF3FDC0719F2209709F451C003
:102DE000229609F05BCFCEEFDFEF8BC0C091DE10F3
:102DF000D091DD106091DD107091DE10762767278D
:102E0000762790E080E00E941FA82DEC3CEC4CEC73
:102E10005DE30E9480A86093D5107093D6108093D4
:102E2000D7109093D810E090E010F090DF106F2D45
:102E30006F77762F6E2D90E080E00E941FA82DEC1A
:102E40003CEC4CEC5DE30E9480A8F7FC18C060935A
:102E5000D9107093DA108093DB109093DC108C2FD4
:102E60008D0F8E0D8F0DC1E0D0E09091E110891390
:102E700002C0D0E0C0E0D195C195D109ABCF905848
:102E8000E6CFC090D510D090D610E090D710F0903B
:102E9000D81020E030E048EC52E4C701B6010E94AF
:102EA000DCAAD0E0C0E0181614F4CBEFDFEF20E08E
:102EB00030E0A901C701B6010E941AA887FF02C02D
:102EC000CAEFDFEFC090D910D090DA10E090DB109D
:102ED000F090DC1020E030E048EC52ECC701B60185
:102EE0000E941AA887FF02C0C9EFDFEF20E030E0A0
:102EF00040EF52E4C701B6010E94DCAA18160CF498
:102F000083C00C30110509F02BCF81E080939B0C1E
:102F10008CE580939D0C10929C0C10929E0C60E0AE
:102F200089ED9DE00E94CD6E81E00E94EF7B0E94C2
:102F30006C776B017C018091950C811168C081E0F8
:102F40008093950C8093940C9FEF9093930C109228
:102F5000920C94E09093910C8093700C8091700C83
:102F6000886B8093700C80916F0C813009F028C1C0
:102F700010926F0C0E946C776B017C018091700C39
:102F80008093BB008091970C9091980CA091990C24
:102F9000B0919A0C892B8A2B8B2BA1F00E946C7715
:102FA0000091970C1091980C2091990C30919A0CEB
:102FB0006C197D098E099F0906171707280739071D
:102FC00008F446C08091BC0083FDD8CF85EC809387
:102FD000BC000E946C776B017C018091950C813064
:102FE00009F4F0C08091920C853008F00DC18091F9
:102FF000920CA1E7BCE0E1E0FCE090E0981769F1F9
:103000002D9121939F5FFACFC8EFDFEF7ACF8091A8
:10301000970C9091980CA091990CB0919A0C892BD7
:103020008A2B8B2B09F487CF0E946C770091970C29
:103030001091980C2091990C30919A0C6C197D0983
:103040008E099F09061717072807390708F073CF5D
:103050008091960C0E94CE7B80E01092550C80935C
:10306000540C082F10E0CEEFDFEF882309F478CE60
:10307000CDEFDFEF053011050CF472CECAEDDAE0CA
:1030800089ED9DE00E94866E88872196CE018A5D3B
:103090009A4080179107A4F3C091E20A0091E30AD5
:1030A000602F70E090E080E00E9421A82DEC3CECC5
:1030B0004CEC5DE30E9480A86B017C016C2F70E0FA
:1030C00090E080E00E9421A89B01AC01C701B601FD
:1030D0000E94C8A96B017C01C092DA0AD092DB0A77
:1030E000E092DC0AF092DD0AD091E40A1091E50A40
:1030F0006D2F6F7770E090E080E00E9421A84B0177
:103100005C01612F70E090E080E00E9421A82DEC2E
:103110003CEC4CEC5DE30E9480A89B01AC01C50136
:10312000B4010E94C8A9D7FD71C06093DE0A7093F4
:10313000DF0A8093E00A9093E10AC00FCD0FC10F20
:103140008091E60AC8130ACE20E030E048EC52E451
:10315000C701B6010E94DCAAD0E0C0E0181614F442
:10316000CBEFDFEF20E030E040EA50E4C701B601EA
:103170000E941AA887FF02C0CAEFDFEFC090DE0AE4
:10318000D090DF0AE090E00AF090E10A20E030E021
:1031900040EF51ECC701B6010E941AA887FF02C098
:1031A000C9EFDFEF20E030E040EF52E4C701B601A5
:1031B0000E94DCAA18160CF0D3CDC8EFDFEFD0CDFB
:1031C00085EE05CF8091970C9091980CA091990C69
:1031D000B0919A0C892B8A2B8B2B09F4FECE0E947E
:1031E0006C770091970C1091980C2091990C30916C
:1031F0009A0C6C197D098E099F0906171707280775
:10320000390708F0EACE24CF85E0F3CE90588DCF71
:10321000CF93DF93FB0122813381DC0113963C9332
:103220002E931297448155816681778114964D9330
:103230005D936D937C931797408551856285738567
:1032400018964D935D936D937C931B971C96EF019D
:103250002C969C01275E3F4F49914D93A217B307CF
:10326000D9F7218D328DFC01328F218FDF91CF91E3
:1032700008950F931F93CF93DF938C01EB01FE0111
:1032800064912196662349F0D801ED91FC9101905B
:10329000F081E02DC8011995F2CFDF91CF911F91F8
:1032A0000F910895EF92FF920F931F93CF93DF93A7
:1032B000EC017B018A0168E074E00E94391961EF3A
:1032C00073E0CE010E94391962EC73E0CE010E94D6
:1032D0003919B701CE010E94BE7563EC79E0CE01C9
:1032E0000E94BE750115110521F0B801CE010E94A2
:1032F000BE7563EC79E0CE01DF91CF911F910F9104
:10330000FF90EF900C94BE75CF93DF93EC0167EACA
:1033100073E00E94391961EF73E0CE010E94391900
:1033200069E773E0CE01DF91CF910C943919CF9307
:10333000DF93EC01FB01248135810E94A274CE0150
:10334000DF91CF910895EF92FF920F931F93CF9348
:10335000DF9300D000D0CDB7DEB78C017B0163ECEA
:1033600078E00E948D748AE0E816F1042CF461E89C
:1033700076E0C8010E946873B701CE0101960E94F1
:10338000DB71BE016F5F7F4FC8010E947273CE0177
:1033900001960E94EE73C80126960FB6F894DEBF20
:1033A0000FBECDBFDF91CF911F910F91FF90EF9096
:1033B0000895CF92DF92EF92FF920F931F93CF93D6
:1033C000DF93CDB7DEB7C455D1090FB6F894DEBF91
:1033D0000FBECDBF65965FAF4EAF65972091320CA3
:1033E0003091330C2F5F3F4F3093330C2093320CCE
:1033F00020914F0C2111C1C08B016C0181E08093A1
:103400004F0C1092330C1092320C63EC78E0CE012A
:10341000895B9F4F0E948D7463EC78E0CE01835BE3
:103420009F4F0E948D7450E040E060E274E0C6015E
:103430000E9452190130110509F08EC063EC78E04A
:1034400081E79FE00E94D17163EC78E08DE49FE01A
:103450000E94D1716596EEADFFAD6597808188239E
:1034600009F474C000E210E09E012F5F3F4F40E27C
:1034700050E0BE016F5D7F4FCE018D5A9F4F0E947D
:103480002F70049739F3BE016F5D7F4FCE018F5BC4
:103490009F4F0E948D74BE016F5B7F4FCE01895B91
:1034A0009F4F0E94B573CE018F5B9F4F0E94EE73BA
:1034B000BE016F5F7F4FCE018F5B9F4F0E948D7467
:1034C000BE016F5B7F4FCE01835B9F4F0E94B57340
:1034D000CE018F5B9F4F0E94EE732D968EAD9FADF8
:1034E0002D970297029730F469E374E08DE49FE032
:1034F0000E94D171BE01695B7F4F81E79FE00E940E
:10350000727363968EAD9FAD6397892B09F4A2CF3A
:1035100062EF75E0CE018F5B9F4F0E948D74BE01FC
:10352000635B7F4FCE018F5B9F4F0E9409736FEEED
:1035300075E00E94F372BC0181E79FE00E94727304
:10354000CE018F5B9F4F0E94EE7384CF61E77FE0D7
:103550008DE49FE00E94727310924F0CCE01835B4A
:103560009F4F0E94EE73CE01895B9F4F0E94EE73C6
:103570000FB6F894DEBF0FBECDBFCC5ADF4F0FB6EB
:10358000F894DEBF0FBECDBFDF91CF911F910F9199
:10359000FF90EF90DF90CF9008950F931F93CF93FC
:1035A000DF9300D000D0CDB7DEB72091B90B222336
:1035B000A9F08C016BE777E0CE0101960E948D7433
:1035C000B801CE0101960E940973BC018CE39DE015
:1035D0000E94D475CE0101960E94EE7326960FB616
:1035E000F894DEBF0FBECDBFDF91CF911F910F9139
:1035F00008950F931F93CF93DF93CDB7DEB72C972A
:103600000FB6F894DEBF0FBECDBF8C010E941A7BAF
:10361000BC01C8010E94A3190E94127BBC01CE010B
:1036200007960E94A3196FEA76E0CE0101960E94E8
:103630008D74BE01695F7F4FCE0101960E940973B0
:10364000BC01C8010E947273CE0101960E94EE7304
:10365000CE0107960E94EE736FEE75E0C8010E94DE
:1036600068730E940A7BBC01CE0101960E94A319D7
:10367000BE016F5F7F4FC8010E947273CE01019639
:103680000E94EE7360E474E0C8010E9468730E94B7
:10369000027BBC01CE0101960E94A319BE016F5F9F
:1036A0007F4FC8010E947273CE0101960E94EE7393
:1036B00060E474E0C8010E9468730E94F87ABC015B
:1036C000CE0101960E94A319BE016F5F7F4FC80112
:1036D0000E947273CE0101960E94EE73C8012C966F
:1036E0000FB6F894DEBF0FBECDBFDF91CF911F9113
:1036F0000F9108950F931F93CF93DF93CDB7DEB74C
:103700002C970FB6F894DEBF0FBECDBF8C010E9480
:103710001A7BBC01C8010E94A3190E94127BBC0144
:10372000CE0107960E94A3196FEA76E0CE010196BA
:103730000E948D74BE01695F7F4FCE0101960E9489
:103740000973BC01C8010E947273CE0101960E94E8
:10375000EE73CE0107960E94EE730E9470790E946C
:10376000FF796091210C70E0CE0107960E94A319A9
:103770006FEA76E0CE0101960E948D74BE01695F0A
:103780007F4FCE0101960E940973BC01C8010E94BF
:103790007273CE0101960E94EE73CE0107960E94CD
:1037A000EE736FEE75E0C8010E9468730E940A7B99
:1037B000BC01CE0101960E94A319BE016F5F7F4F2D
:1037C000C8010E947273CE0101960E94EE7360E4FC
:1037D00074E0C8010E9468730E94027BBC01CE01A4
:1037E00001960E94A319BE016F5F7F4FC8010E941E
:1037F0007273CE0101960E94EE7360E474E0C8011A
:103800000E9468730E94F87ABC01CE0101960E9462
:10381000A319BE016F5F7F4FC8010E947273CE0172
:1038200001960E94EE73C8012C960FB6F894DEBF85
:103830000FBECDBFDF91CF911F910F910895CF9211
:10384000DF92EF92FF920F931F93CF93DF9300D0FD
:1038500000D0CDB7DEB77C01FB01848195818A0160
:10386000081B190B101611069CF0C7010E947274F8
:10387000C70126960FB6F894DEBF0FBECDBFDF910D
:10388000CF911F910F91FF90EF90DF90CF9008950F
:10389000CE0101960E948474CC24C394D12C6FEE87
:1038A00075E0CE0101960E946873FFEFCF1ADF0A20
:1038B0000C151D05A4F7BE016F5F7F4FC7010E9465
:1038C0007274CE0101960E94EE73D2CFDF92EF9216
:1038D000FF920F931F93CF93DF93CDB7DEB762971D
:1038E0000FB6F894DEBF0FBECDBF8C011092EB0A6D
:1038F00063EC78E0CE010D960E948D74FF24F39462
:103900008CE39DE00E94E36C2091EB0A18161906E7
:103910007CF521112DC08CE39DE00E94C16C8A30A2
:1039200009F07EC089899A89892B09F481C0F092B7
:10393000EB0A62E474E0CE0101960E948D74BE0130
:10394000635F7F4FCE0101960E940973BC01CE01D7
:1039500007960E948474CE0107960E94CD1ACE016C
:1039600007960E94EE73CE0101960E94EE7360C02E
:10397000F12CE12CDD24D394222309F460C0898941
:103980009A89019709F045C061EE74E0CE0107966F
:103990000E948D74BE01695F7F4FCE010D960E941B
:1039A000D872F12C811115C062E574E0CE01019648
:1039B0000E948D74BE016F5F7F4FCE010D960E94F5
:1039C000D872FF24F3948111F12CCE0101960E944C
:1039D000EE73CE0107960E94EE73FF20A1F050E037
:1039E00040E0BE01635F7F4FCE0101960E949719B0
:1039F000BE016F5F7F4F84E19FE00E94B573CE01EF
:103A000001960E94EE7364E170E080E090E00E9415
:103A10009177BE01635F7F4FC8010E9472748EC0B0
:103A20008D3009F47FCF682FCE010D960E9446732A
:103A30006AE070E080E090E00E94917761CF8FE9CA
:103A40009CE00E94E36C1816190614F58FE99CE0BF
:103A50000E94C16C8A30A9F08D3099F09091EB0AE8
:103A600091110FC0682FCE010D960E9446738FEF03
:103A7000E81AF80A65E070E080E090E00E94917733
:103A8000DECF89899A89892BA9F3D092EB0AF2CFEC
:103A900064E170E080E090E00E949177EF2809F403
:103AA0003FC089899A89892BD9F18091B90B8823E4
:103AB00089F16BE777E0CE0101960E948D74BE011B
:103AC0006F5F7F4FCE010D960E94D872F82ECE0107
:103AD00001960E94EE73F1101DC06BE474E0CE01FC
:103AE00001960E948D74CE0101960E94F815CE01B8
:103AF00001960E94EE73BE01635F7F4FCE01019677
:103B00000E948474CE0101960E94E115CE010196B7
:103B10000E94EE7364E170E080E090E00E94917793
:103B200089899A892091EB0A21112BCF009709F0FE
:103B300028CF63EC78E0C8010E948D74CE010D9609
:103B40000E94EE73C80162960FB6F894DEBF0FBEF6
:103B5000CDBFDF91CF911F910F91FF90EF90DF903C
:103B600008950F931F93CF93DF93CDB7DEB72C97B4
:103B70000FB6F894DEBF0FBECDBF2C893D89FE0184
:103B80007496A6EFBBE090E080E0329628173907E4
:103B900034F0408151814D935D930196F6CFCE5B19
:103BA000DE4F88819981C254D140281739070CF023
:103BB0001CC2DC01AA0FBB1FAA50B44F880F991F6B
:103BC000FC01EC50F44F8081918101968D939C9380
:103BD0008C8D9D8D9093B60B8093B50B8E8D9F8DA4
:103BE0009093B80B8093B70BAD968FADAD97BE0198
:103BF00064597F4F8F3209F001C2CE0107960E94AF
:103C00008D7464E574E0CE0101960E948D74BE014E
:103C1000695F7F4FCE0101960E940973BC0181E06C
:103C200091E10E949E73CE0101960E94EE73CE0137
:103C300007960E94EE7361E071E1CE0101960E9449
:103C40008474CE0101960E94E115CE0101960E9476
:103C5000EE736AE674E0CE0101960E948D74BE0197
:103C60006F5F7F4F81E091E10E94B872182FCE0103
:103C700001960E94EE734091051150910611112397
:103C800009F4C3C1BA016250710981E091E10E9457
:103C9000A772682FCE0101960E945974BE016F5F12
:103CA0007F4F83EE90E10E94B573CE0101960E9492
:103CB000EE7363ED7FE0CE0107960E948D746CE693
:103CC00074E0CE0101960E948D74BE01695F7F4F42
:103CD000CE0101960E940973BC018BEF90E10E9416
:103CE0009E73CE0101960E94EE73CE0107960E944C
:103CF000EE7324968FAD24971F928F9323968FADEA
:103D000023971F928F9322968FAD22971F928F93A6
:103D100021968FAD21971F928F9382E794E09F9316
:103D20008F9386EE9BE09F938F930E94B1ADCE520E
:103D3000DF4F88819981C25DD04090938F0280933C
:103D40008E02BE016C527F4FCE0101960E948D748F
:103D5000BE016F5F7F4F85EF90E10E94B573CE018A
:103D600001960E94EE73BE0161527F4FCE01019613
:103D70000E948D74BE016F5F7F4F8FEE90E10E94B5
:103D8000B573CE0101960E94EE734091F3105091ED
:103D9000F410425051096FEE70E1CE0101960E947D
:103DA0009719CE0101960E943F726C596093970259
:103DB000CE0101960E94EE73CC5EDE4F6881798160
:103DC0008A819B81C451D1400E9421A80FB6F894EA
:103DD000DEBF0FBECDBF9B01AC010E94E1AA8823CC
:103DE00089F08CE390E0A0E0B0E0CC5EDE4F888309
:103DF0009983AA83BB83C451D140CD5EDE4F188224
:103E0000C351D140CD5EDE4F8881C351D14088235C
:103E100099F0CC5EDE4F88819981AA81BB81C45123
:103E2000D1408093700290937102A0937202B0937C
:103E3000730281E08093580CC85EDE4F68817981FF
:103E40008A819B81C851D1409B01AC010E94E1AAAB
:103E5000882361F080E090E0A0E7B2E4C85EDE4F26
:103E600088839983AA83BB83C851D140C45EDE4F47
:103E700068817981CC51D140072E000C880B990BB9
:103E80000E9421A89B01AC010E94E1AA882341F075
:103E900082E090E0C45EDE4F99838883CC51D140AC
:103EA000CE5BDE4F68817981C254D140072E000C71
:103EB000880B990B0E9421A89B01AC010E94E1AAEA
:103EC000882341F083E090E0CE5BDE4F99838883C6
:103ED000C254D140C45CDE4F08811981CC53D1401B
:103EE000B801012E000C880B990B0E9421A89B01A0
:103EF000AC010E94E1AA811103C01016110644F022
:103F000080E590E0C45CDE4F99838883CC53D14038
:103F1000C45CDE4F88819981CC53D14090933F029D
:103F200080933E0288E2FE01E551FF4FAAEBBBE021
:103F300001900D928A95E1F7CE5CDE4F88819981E0
:103F4000AA81BB81C253D1408093290290932A0257
:103F5000A0932B02B0932C02CA5CDE4F888199811A
:103F6000AA81BB81C653D14080932502909326023B
:103F7000A0932702B0932802C65CDE4F8881998106
:103F8000CA53D14090935D0280935C02CC5BDE4FBC
:103F900068817981C454D140072E000C880B990B9D
:103FA0000E9421A89B01AC010E94E1AA882341F054
:103FB00088E390E0CC5BDE4F99838883C454D14082
:103FC000CC5BDE4F88819981C454D140909391029B
:103FD000809390022C960FB6F894DEBF0FBECDBF33
:103FE000DF91CF911F910F9108958091FA0B9091DD
:103FF000FB0B9093FD0B8093FC0BEACDCE01079653
:104000000E948D7469E574E0FECD4150510961E074
:1040100071E1CE0101960E949719BE016F5F7F4F3B
:1040200083EE90E10E94B573CE0101960E94EE737B
:1040300061E071E1CE0101960E9484746AE674E049
:10404000CE0101960E94F372BC0181E091E10E94D1
:104050009E732BCEDF92EF92FF920F931F93CF931D
:10406000DF93CDB7DEB762970FB6F894DEBF0FBE11
:10407000CDBF2091F002222379F12091EF0222237B
:1040800059F17A018C016F3F7F4FA1F560E080E02C
:104090000E94347DD12CB80189E591E10E94C6755A
:1040A00060E175E089E591E10E94E875F80184819D
:1040B00060E08D0D0E94347D0E944F7860936B0C00
:1040C00070936C0C80936D0C90936E0CB701FF0C89
:1040D000880B990B0E94917762960FB6F894DEBF19
:1040E0000FBECDBFDF91CF911F910F91FF90EF9049
:1040F000DF90089560E080E00E94347D0E944F7858
:1041000028EE33E040E050E00E9464A9CA01B90102
:1041100020E831E541E050E00E9486A9AB01BC01F6
:1041200020E0CE0101960E942C74BE016F5F7F4F8C
:10413000CE0107960E94847465E678E0CE0107966A
:104140000E94F372BC01CE010D960E948474CE01D0
:1041500007960E94EE73CE0101960E94EE73BE0197
:10416000635F7F4F89E591E10E94C675D98860E061
:104170008D2D0E94347DCE010D960E94EE738BCF63
:10418000CF93DF9300D000D0CDB7DEB70E94DD081B
:10419000CE0101960E94F91A4AE050E06FEF7FEFDE
:1041A000CE0101960E942A20CE0101960E94EE7354
:1041B00061E080E00E94347DCE0101960E9407718B
:1041C00069E571E1CE0101960E9460756EE774E0C9
:1041D00089E591E10E94BE750E944F7860933C0C86
:1041E00070933D0C80933E0C90933F0C26960FB637
:1041F000F894DEBF0FBECDBFDF91CF9108950F932E
:104200001F93CF93DF9300D000D0CDB7DEB78C01E2
:10421000CE0101960E94F91A4AE050E06FEF7FEF5D
:10422000CE0101960E942A20CE0101960E94EE73D3
:10423000B801CE0101960E9484744AE050E06FEF0D
:104240007FEFCE0101960E940109CE0101960E94E6
:10425000EE7326960FB6F894DEBF0FBECDBFDF918A
:10426000CF911F910F9108952F923F924F925F929D
:104270006F927F928F929F92AF92BF92DF92EF9256
:10428000FF920F931F93CF93DF93CDB7DEB7E497E1
:104290000FB6F894DEBF0FBECDBF7C014A015B01B3
:1042A00019010E944F782B013C0187010D5B1F4FC4
:1042B000C8010E94210B181619069CF00E944F7825
:1042C000641975098609970986169706A806B9061E
:1042D00008F490C162E370E080E090E00E94917782
:1042E000E7CF42E250E0BE016F5F7F4FC8010E94FE
:1042F000D80A8981823009F078C1F80184899589CA
:104300008334910509F071C16D817E818F8198851B
:104310000E9402AB2B013C01F1014082518262827A
:10432000738246E050E0B701685F7F4FCE014D9643
:104330000E9430AD892B99F4F70180819181A2818F
:10434000B381481659066A067B0648F08481958138
:10435000A681B78184159505A605B705E8F4C801BF
:104360000E948907D12C8D2DE4960FB6F894DEBFFC
:104370000FBECDBFDF91CF911F910F91FF90EF90B6
:10438000DF90BF90AF909F908F907F906F905F90E5
:104390004F903F902F90089589899A89AB89BC8965
:1043A00086879787A08BB18B8EECA82EB12CC80185
:1043B0000E94F70AF1E0AF1AB108C9F7D12CC70182
:1043C00082969AA789A7F701B696FCA7EBA708964D
:1043D0009EA78DA73C974F01899698AB8FA73897DA
:1043E000FAABE9AB1701F6E12F0E311CC5979CAB78
:1043F0008BABF801818D928D181619060CF0F6C062
:10440000C8010E94F70A8333910509F4D4C0A4F5CA
:104410008130910509F474C074F4892B51F3C801FB
:104420000E94F70AB82EBA94FFEFBF1611F3C80125
:104430000E94F70AF8CF8330910509F46CC0069703
:1044400071F7C8010E94F70AA82E44E050E06BA95A
:104450007CA9C8010E94D80A712C612CEA2DE45075
:10446000FF0B5F016A147B0424F6C8010E94F70A5F
:10447000FFEF6F1A7F0AF6CF8A33910509F46FC0F8
:1044800074F585339105A1F1C69749F6C8010E94DC
:10449000F70AB82EF701828D811109C0838D811131
:1044A00006C0848D811103C0858D8823A1F0EFA5FE
:1044B000F8A94080518062807380B401CE01839658
:1044C0000E940C768DA19EA1AFA1B8A5841595057B
:1044D000A605B705D9F544E050E0B40118C08B3308
:1044E000910509F452C08F3F910509F482CF97CF0F
:1044F000C8010E94F70AC8010E94F70AD82E79CF96
:10450000C8010E94F70A44E050E069A97AA9C801ED
:104510000E94D80A6ECFC8010E94F70AA82E44E074
:1045200050E0B101C8010E94D80A712C612C8A2D7B
:104530008450990B5C016A147B040CF05ACFC801BB
:104540000E94F70A9FEF691A790AF5CFBA94FFEF34
:10455000BF1609F44ECFC8010E94F70AF7CFC80171
:104560000E94F70A44E050E06BA57CA5C8010E94B8
:10457000D80AF70166A177A180A591A50E9402AB98
:1045800066A377A380A791A734CFC8010E94F70A3A
:1045900044E050E06DA57EA5C8010E94D80AF7014D
:1045A00062A573A584A595A50E9402AB62A773A717
:1045B00084A795A71ECFC8010E94F70A44E050E0E7
:1045C00069A57AA5C8010E94D80AF70162A173A162
:1045D00084A195A10E9402AB62A373A384A395A3B7
:1045E00066A777A780AB91AB04CFD12CC8010E94FE
:1045F0008907B9CEDD24DA94B6CE2F923F924F923E
:104600005F926F927F928F929F92AF92BF92CF9262
:10461000DF92EF92FF920F931F93CF93DF9300D01F
:1046200000D0CDB7DEB78C010E94859F2FEC37E01C
:1046300040E050E00E9486A9DC01CB010196A11D5B
:10464000B11DF80184839583A683B783808391830A
:10465000A283B3835801F3E4AF0EB11CC5010E94DD
:10466000500C64E470E0C5010E94710C882309F4C9
:1046700045C10E944F782B013C01480182E4880E1D
:10468000911C48EEC42E43E0D42EE12CF12C52E0D4
:10469000252E1E821D82D4018C918330B1F18111AF
:1046A00066C0F80184819581A681B7810196A11D1C
:1046B000B11D84839583A683B7830E944F786419C4
:1046C000750986099709A70196010E9464A9A901A5
:1046D00061E0C8010E94D71081E0D4018C938D81E4
:1046E0009E810197C1F20E944F786419750986096D
:1046F0009709D801D6962D913D914D915C91D9970E
:10470000261737074807590720F6C5010E94500CA5
:10471000F80184819581A681B7810196A11DB11D03
:1047200084839583A683B7830E944F78F801FE9611
:1047300060837183828393838D819E8126960FB6D9
:10474000F894DEBF0FBECDBFDF91CF911F910F91C7
:10475000FF90EF90DF90CF90BF90AF909F908F90A1
:104760007F906F905F904F903F902F90089584308E
:10477000F1F4F80184819581A681B7810196A11D8C
:10478000B11D84839583A683B7830E944F786419F3
:10479000750986099709A70196010E9464A9A901D4
:1047A00063E0C8010E94D710D4012C9298CF8130C9
:1047B00051F5F80142AD53AD64AD75AD9E012F5F6B
:1047C0003F4FC8010E943421382EF2E08F1390C071
:1047D00089819A81AB81BC81F80184839583A6830A
:1047E000B7830E944F786419750986099709A70154
:1047F00096010E9464A9A90163E0C8010E94D71034
:10480000D4013C926CCF823009F069CFF80142ADFF
:1048100053AD64AD75AD9E012F5F3F4FC8010E943F
:104820003421382EF5E08F135DC0E3E0D401EC9322
:10483000F80182A193A1A4A1B5A1892B8A2B8B2B6E
:1048400041F484E893E0A0E0B0E082A393A3A4A3A2
:10485000B5A3F80186A197A1A0A5B1A5892B8A2BA4
:104860008B2B61F482A193A1A4A1B5A1B695A795C4
:104870009795879586A397A3A0A7B1A7F80182A5CE
:1048800093A5A4A5B5A5892B8A2B8B2BA9F482A16E
:1048900093A1A4A1B5A1AC01BD0123E076956795D4
:1048A000579547952A95D1F7841B950BA60BB70B07
:1048B00082A793A7A4A7B5A7F80186A197A1A0A551
:1048C000B1A586A797A7A0ABB1AB82A593A5A4A5D8
:1048D000B5A582AB93ABA4ABB5AB81E090E09E8372
:1048E0008D83FDCE96E0891303C0D4011C92F7CED0
:1048F000BFEF3B12F4CEF4011082F1CE1E821D8276
:104900001BCFEF92FF920F931F93CF93DF93CDB7FF
:10491000DEB7E8970FB6F894DEBF0FBECDBF63ECED
:1049200078E0CE0187960E948D7463EC78E0CE012A
:104930008D960E948D7482E0E82EF12C2496FFAEB5
:10494000EEAE249786E0E1E0F3E0DE01D39601903D
:104950000D928A95E1F786E0FE01F396DE01AC5BED
:10496000BF4F01900D928A95E1F72C961FAE1EAEB7
:104970002C9701E010E02E961FAF0EAF2E9788E027
:10498000E7E0F3E0DE01599601900D928A95E1F798
:1049900088E0FE017996DE01A25BBF4F01900D9287
:1049A0008A95E1F788E1EFE0F3E0DE0111960190EE
:1049B0000D928A95E1F788E1FE013196DE01AA5A4F
:1049C000BF4F01900D928A95E1F780912703909156
:1049D0002803A0912903B0912A03E2968CAF9DAFE2
:1049E000AEAFBFAFE29762E874E0CE0187960E9457
:1049F000D17160E0CE0187960E9446734BA55CA5FD
:104A0000BE016E587F4FCE0187960E94257169E2E4
:104A100076E0CE018D960E94797368ED74E083EEA6
:104A200090E10E94D17160E0CE018D960E944673A4
:104A300049A95AA9BE0166567F4FCE018D960E94A4
:104A4000257163EC78E0CE0187960E94D17163EC0A
:104A500078E0CE018D960E94D171C250DF4F19824D
:104A60001882CE5FD04080918E0290918F02C0500C
:104A7000DF4F99838883C050D14080E090E0A0E769
:104A8000B2E4CA5BDE4F88839983AA83BB83C65492
:104A9000D140C65BDE4FF982E882CA54D14080E043
:104AA00090E0A0E2B2E4C45BDE4F88839983AA83DE
:104AB000BB83CC54D14080E090E0A4E3B2E4C05B7F
:104AC000DE4F88839983AA83BB83C055D14084EB92
:104AD00090E0CC5ADE4F99838883C455D14088E753
:104AE00090E0CA5ADE4F99838883C655D1408CE244
:104AF00091E0A0E0B0E0C85ADE4F88839983AA8392
:104B0000BB83C855D140C45ADE4F19830883CC55A6
:104B1000D140C25ADE4FF982E882CE55D14060E0E2
:104B200085EF90E10E94467360E08FEE90E10E9475
:104B300046734091F9105091FA10BE016E5F7E4F9E
:104B400085EF90E10E9425714091F3105091F4108F
:104B5000BE01635F7E4F8FEE90E10E94257188E277
:104B6000EAEBFBE0DE01A75EBE4F01900D928A9555
:104B7000E1F78CE390E0A0E0B0E0CE5BDE4F88830D
:104B80009983AA83BB83C254D140CF5BDE4F188286
:104B9000C154D14084EE98E3AEE8B2E4C05ADE4F8F
:104BA00088839983AA83BB83C056D14084EE98E35F
:104BB000AEE8B1E4CC59DE4F88839983AA83BB83E6
:104BC000C456D140C859DE4F19830883C856D14016
:104BD00080E590E0C659DE4F99838883CA56D1405C
:104BE00083E090E0C059DE4F99838883C057D1405D
:104BF00088E390E0CE58DE4F99838883C257D14036
:104C000084EF91E09093670280936602BE016E5B31
:104C10007F4F0E949C0864EF71E080E090E00E946A
:104C2000917762E176E0CE0181960E947B74CE019D
:104C300081960E94E115CE0181960E94EE73CE010D
:104C40008D960E94EE73CE0187960E94EE73E896D1
:104C50000FB6F894DEBF0FBECDBFDF91CF911F918D
:104C60000F91FF90EF9008959F92AF92BF92CF92D5
:104C7000DF92EF92FF920F931F93CF93DF93CDB705
:104C8000DEB7C859D1090FB6F894DEBF0FBECDBF4D
:104C90005C017B016A016BEF7FE0CE0189579F4F7A
:104CA0000E948D746AE674E08E010F5F1F4FC80189
:104CB0000E948D74B801CE0189579F4F0E94D8720F
:104CC000982EC8010E94EE73911014C06AE674E039
:104CD000C8010E948D74BE0169577F4FC8010E94B0
:104CE0000973BC01CE0189579F4F0E949E73C80172
:104CF0000E94EE73B501CE0183579F4F0E948D74C1
:104D00006AE874E0E114F10471F068E974E021E00C
:104D1000E216F10441F063EA74E032E0E316F104D4
:104D200011F06BEA74E0CE0189579F4F0E946873BF
:104D300060E0CE0189579F4F0E944673B601C801BB
:104D40000E9484746AE0C8010E945A73BC01CE01BB
:104D50008D569F4F0E948474C8010E94EE73C55700
:104D6000DF4F48815981CB58D040B801CE018957D7
:104D70009F4F0E9425718091590C882399F163EB14
:104D800074E0CE018F579F4F0E948D74CE018F57D4
:104D90009F4F0E94F815CE018F579F4F0E94EE73D0
:104DA000BE0169577F4FCE018F579F4F0E94847479
:104DB000CE018F579F4F0E94F815CE018F579F4FFE
:104DC0000E94EE73B801CE018F579F4F0E948D74E1
:104DD000CE018F579F4F0E94F815CE018F579F4FDE
:104DE0000E94EE73CC56DF4F8881C459D0408F9318
:104DF000CD56DF4F8881C359D0408F93C257DF4FC4
:104E00008881CE58D0408F93C357DF4F8881CD58CB
:104E1000D0408F9383EC94E09F938F938AE1E82EA8
:104E20008AE0F82EFF92EF920E94B1AD40913E02CF
:104E300050913F0266EE7BE084E89FE00E946410A0
:104E40000FB6F894DEBF0FBECDBF019709F07CC04E
:104E50001F930F9389EC94E09F938F9300E21BE0E4
:104E60001F930F930E94B1ADB80184E89FE00E94A8
:104E7000AA7586EE9BE09F938F938AED94E09F93B3
:104E80008F931F930F930E94B1ADB80184E89FE008
:104E90000E94AA756AE174E084E89FE00E94E875C8
:104EA00063EC79E084E89FE00E94EE74F7010190E2
:104EB0000020E9F7CF018B519A409F938F9383EEA7
:104EC00094E09F938F931F930F930E94B1ADB8010D
:104ED00084E89FE00E94AA75B70184E89FE00E94E1
:104EE000BE7562E370E080E090E00E94917784E814
:104EF0009FE00E9451120FB6F894DEBF0FBECDBFE7
:104F000011E0CE018D569F4F0E94EE73CE01835764
:104F10009F4F0E94EE73CE0189579F4F0E94EE7300
:104F2000812FC856DF4F0FB6F894DEBF0FBECDBF3E
:104F3000DF91CF911F910F91FF90EF90DF90CF9075
:104F4000BF90AF909F9008956DE574E0CE018F57AC
:104F50009F4F0E947B74CE018F579F4F0E94E11597
:104F6000CE018F579F4F0E94EE7369E674E0CE0129
:104F70008F579F4F0E947B74CE018F579F4F0E9487
:104F8000F815CE018F579F4F0E94EE736AE17AE0C9
:104F9000CE018F579F4F0E948D74CE018F579F4F28
:104FA0000E94E115CE018F579F4F0E94EE7310E0D3
:104FB000A8CFEF92FF920F931F93CF93DF93CDB7BC
:104FC000DEB768970FB6F894DEBF0FBECDBF81E0A5
:104FD00080934F0C0E947E8E8C0160ED77E080E024
:104FE00090E00E9491778BE0E82EF12C0D7F01304C
:104FF000110571F481E0E81AF10851F00E947E8EEB
:105000008C0160ED77E080E090E00E949177EECF38
:105010000E94B48F7C0168EE73E080E090E00E9413
:1050200091770BE010E0EF2899F40150110981F01D
:1050300060ED77E080E090E00E9491770E94B48F6D
:105040007C0168EE73E080E090E00E949177EBCF06
:1050500082E49EE00E94E51110924F0C0E94C02055
:1050600063EC78E0CE0107960E948D7468E975E0E4
:10507000CE010D960E947B74CE0143960E9407716B
:10508000888D1F928F938F891F928F938E891F9285
:105090008F938D891F928F9382E794E09F938F93D4
:1050A00080E29BE09F938F930E94B1AD60E27BE032
:1050B000CE0101960E948D74BE016F5F7F4FCE01BD
:1050C00007960E94B573CE0101960E94EE73BE0151
:1050D000635F7F4FCE0101960E948474CE010196DA
:1050E0000E94F815CE0101960E94EE73BE01695F21
:1050F0007F4FCE0101960E948474CE0101960E94DA
:10510000E115CE0101960E94EE73BE01695F7F4FEB
:10511000CE0101960E948474AE014F5F5F4F63E041
:1051200070E080E092E00E943426182FCE010196B4
:105130000E94EE730FB6F894DEBF0FBECDBF111103
:105140002BC06EE875E0CE0101960E947B74CE0103
:1051500001960E94F815CE0101960E94EE73BE01E1
:10516000635F7F4FCE0101960E948474CE01019649
:105170000E94F815CE0101960E94EE7363E57FE070
:10518000CE0101960E948474CE0101960E94E11521
:10519000CE0101960E94EE73CE010D960E94EE7331
:1051A000CE0107960E94EE7368960FB6F894DEBFA4
:1051B0000FBECDBFDF91CF911F910F91FF90EF9068
:1051C00008957F928F929F92AF92BF92CF92DF927B
:1051D000EF92FF920F931F93CF93DF93CDB7DEB77C
:1051E00062970FB6F894DEBF0FBECDBF6BE775E0D8
:1051F000CE0101960E947B74CE0101960E94E115BA
:10520000CE0101960E94EE7304E010E03CEEC32E46
:105210003AE0D32E40E3E42E53EEB52E66E0A62E00
:105220007CEE972EE1E3FE2EFEE48F2EA4E37A2E91
:1052300068EB72E286E29FE00E94710CF6018E2D0F
:1052400011928A95E9F7B092EC0AA092EE0A909238
:10525000EF0AF092F80A8092F90AF092FA0A709234
:10526000FB0A60E472E0CE0101960E940C764BE7E7
:1052700050E0BE016F5F7F4F86E29FE00E94310DDC
:1052800040E350E06CEE7AE086E29FE00E94C90CB9
:1052900086E29FE00E94FF0C68EE73E080E090E001
:1052A0000E94917786E29FE00E94210B892B09F0F2
:1052B0004FC00150110909F07CC080911C0B9091E6
:1052C0001D0BA0911E0BB0911F0B892B8A2B8B2BD2
:1052D00009F089C063EC78E081E79FE00E94D1711A
:1052E00061E77FE0CE0101960E948474AE014F5FBA
:1052F0005F4F70E060E084E792E00E943426182F50
:10530000CE0101960E94EE7311110EC063E675E0A6
:10531000CE0101960E947B74CE0101960E94E11598
:10532000CE0101960E94EE7362960FB6F894DEBF2E
:105330000FBECDBFDF91CF911F910F91FF90EF90E6
:10534000DF90CF90BF90AF909F908F907F90089507
:1053500040E350E06CEE7AE086E29FE00E94D80ADB
:105360006091140B7091150B76276727762790E0D4
:1053700080E0CB01772766270091160B1091170B61
:1053800010270127102730E020E0602B712B822BA3
:10539000932B7E508A4A93480E944B790E947079E1
:1053A00060931C0B70931D0B80931E0B90931F0B2F
:1053B00084CF68EE73E080E090E00E9491774091A6
:1053C0001C0B50911D0B60911E0B70911F0B2AE05E
:1053D0008CE39DE00E94FD7463EC79E08CE39DE03A
:1053E0000E94EE7425CF68EE73E080E090E00E94AA
:1053F00091770E9470796093460C7093470C80936C
:10540000480C9093490C0E9470796093400C709303
:10541000410C8093420C9093430CCE0101960E9464
:105420007A1BCE0101960E94E115CE0101960E94E1
:10543000EE730E940A7BBC01CE0107960E94A3195D
:1054400060E474E0CE0107960E9468730E94027BBC
:10545000BC01CE0101960E94A319BE016F5F7F4F70
:10546000CE0107960E947273CE0101960E94EE73E0
:1054700060E474E0CE0107960E9468730E94F87A97
:10548000BC01CE0101960E94A319BE016F5F7F4F40
:10549000CE0107960E947273CE0101960E94EE73B0
:1054A00068EF74E0CE0101960E948D74BE01695FC1
:1054B0007F4FCE0101960E940973BC01CE010D966B
:1054C0000E9484744AE050E06FEF7FEFCE010D96AA
:1054D0000E942A20CE010D960E94EE73CE01019605
:1054E0000E94EE73CE0107960E94EE7368EE73E0A1
:1054F00080E090E00E9491770E941A7BBC01CE016F
:105500000D960E94A3190E94127BBC01CE01019648
:105510000E94A3196FEA76E0CE0107960E948D746F
:10552000BE016F5F7F4FCE0107960E940973BC01D9
:10553000CE010D960E947273CE0107960E94EE7303
:10554000CE0101960E94EE730E9470790E94FF794D
:105550006091210C70E0CE0101960E94A3196FEAC0
:1055600076E0CE0107960E948D74BE016F5F7F4F7B
:10557000CE0107960E940973BC01CE010D960E94D0
:105580007273CE0107960E94EE73CE0101960E94BF
:10559000EE736EEF74E0CE0101960E948D74BE0131
:1055A000635F7F4FCE0101960E940973BC01CE015B
:1055B00007960E9484744AE050E06FEF7FEFCE01BF
:1055C00007960E942A20CE0107960E94EE73CE0114
:1055D00001960E94EE73CE010D960E94EE7368EE66
:1055E00073E080E090E00E949177CE0101960E94E6
:1055F000F91A4AE050E06FEF7FEFCE0101960E946A
:105600002A208ECECF92DF92EF92FF920F931F93BC
:10561000CF93DF93CDB7DEB768970FB6F894DEBFB0
:105620000FBECDBF63EC78E0CE0143960E948D742F
:1056300066E577E0CE0101960E947B74CE0101966B
:105640000E94F815CE0101960E94EE736CA17DA117
:10565000CE0101960E94DB71CE0101960E94E115F8
:10566000CE0101960E94EE736EE377E0CE010196C3
:105670000E947B74CE0101960E94F815CE0101961E
:105680000E94EE73CE5ADE4F68817981C255D140B7
:10569000CE0101960E94DB71CE0101960E94E115B8
:1056A000CE0101960E94EE7361E377E0CE01019690
:1056B0000E947B74CE0101960E94F815CE010196DE
:1056C0000E94EE7306EF1BE0EE24E394F12CCE5A19
:1056D000DE4F88819981C255D1408E159F050CF40B
:1056E0004AC0F80182819381C6979CF164E075E01D
:1056F000CE0101960E948D74CE0101960E94F8158C
:10570000CE0101960E94EE73F801628173816653A7
:105710007109CE0101960E94DB71CE0101960E94B3
:10572000F815CE0101960E94EE736FEE75E0CE0182
:1057300001960E948D74CE0101960E94F815CE014B
:1057400001960E94EE73FFEFEF1AFF0A0E5F1F4FE4
:10575000BECF6CE676E0CE0101960E948D74CE013C
:1057600001960E94F815CE0101960E94EE73F80191
:1057700062817381CECF6FEE75E0CE0101960E94FB
:105780008D74CE0101960E94E115CE0101960E9412
:10579000EE7362E277E0CE0101960E947B74CE0147
:1057A00001960E94F815CE0101960E94EE73609159
:1057B000B50B7091B60BCE0101960E94DB71CE0144
:1057C00001960E94F815CE0101960E94EE736FEECD
:1057D00075E0CE0101960E948D74CE0101960E9463
:1057E000F815CE0101960E94EE736091B70B70918F
:1057F000B80BCE0101960E94DB71CE0101960E948A
:10580000E115CE0101960E94EE736BE077E0CE01C8
:1058100001960E947B74CE0101960E94F815CE017C
:1058200001960E94EE73BE01605D7F4FCE0101962E
:105830000E948D74CE0101960E94F815CE0101964A
:105840000E94EE736FEE75E0CE0101960E948D749A
:10585000CE0101960E94F815CE0101960E94EE73CA
:10586000BE016C5C7F4FCE0101960E948D74CE010B
:1058700001960E94E115CE0101960E94EE736BEF36
:1058800076E0CE0101960E947B74CE0101960E94C3
:10589000E115CE0101960E94EE738E010C5D1F4F43
:1058A000EE24E394F12C680188E0C80ED11C8CA191
:1058B0009DA18E159F050CF449C0B701CE01079636
:1058C0000E94DB716BE777E0CE0101960E948D7438
:1058D000BE01695F7F4FCE0101960E940973BC0132
:1058E000CE010D960E948474CE010D960E94F8158B
:1058F000CE010D960E94EE73CE0101960E94EE73CA
:10590000CE0107960E94EE736FEA76E0CE01019613
:105910000E948D74CE0101960E94F815CE01019669
:105920000E94EE73B801645E7F4FCE0101960E9423
:105930008D74CE0101960E94E115CE0101960E9460
:10594000EE73EFEFEE1AFE0A8601ADCF6AEE76E057
:10595000CE0101960E947B74CE0101960E94F8153B
:10596000CE0101960E94EE737E01F2EBEF1AFEEF7C
:10597000FF0A10E000E0F70161917F0170E0CE01C5
:1059800001960E94DB71CE0101960E94F815CE01AE
:1059900001960E94EE730330110571F06EEC78E011
:1059A000CE0101960E948D74CE0101960E94F815D9
:1059B000CE0101960E94EE730F5F1F4F0430110558
:1059C000D1F66FEE75E0CE0101960E948D74CE0186
:1059D00001960E94E115CE0101960E94EE73C45B10
:1059E000DE4F68817981CC54D140072E000C880BA2
:1059F000990B0E9421A89B01AC010E94E1AA882377
:105A000041F080E590E0C45BDE4F99838883CC54FD
:105A1000D140C45BDE4F88819981CC54D1409093B2
:105A20003F0280933E0260ED76E0CE0101960E9437
:105A30007B74CE0101960E94F815CE0101960E945A
:105A4000EE7366EE7BE0CE0101960E948D74CE016E
:105A500001960E94F815CE0101960E94EE736EEC3D
:105A600076E0CE0101960E947B74CE0101960E94E1
:105A7000F815CE0101960E94EE7360913E0270917E
:105A80003F02CE0101960E94DB71CE0101960E9479
:105A9000E115CE0101960E94EE736FEB76E0CE0128
:105AA00001960E947B74CE0101960E94F815CE01EA
:105AB00001960E94EE73BE016C5A7F4FCE01019693
:105AC0000E948D74CE0101960E94E115CE010196CF
:105AD0000E94EE7366E075E0CE0101960E948D741F
:105AE000CE0101960E94F815CE0101960E94EE7338
:105AF000BE0164587F4FCE0101960E948D74CE0185
:105B000001960E94E115CE0101960E94EE73C052EB
:105B1000DF4F88819981C05ED040892B71F467EB9B
:105B200076E0CE0101960E947B74CE0101960E9420
:105B3000E115CE0101960E94EE73C052DF4F8881BD
:105B40009981C05ED040019771F46DEA76E0CE0194
:105B500001960E947B74CE0101960E94E115CE0150
:105B600001960E94EE73C052DF4F88819981C05E1A
:105B7000D040029771F464EA76E0CE0101960E946B
:105B80007B74CE0101960E94E115CE0101960E9420
:105B9000EE736EE976E0CE0101960E947B74CE0131
:105BA00001960E94F815CE0101960E94EE73CE5127
:105BB000DF4F68817981C25ED040CE0101960E949C
:105BC000DB71CE0101960E94E115CE0101960E9483
:105BD000EE7365E976E0CE0101960E947B74CE01FA
:105BE00001960E94F815CE0101960E94EE73CC5AE0
:105BF000DE4F88819981C455D140C6970CF41FC1EE
:105C000064E075E0CE0101960E948D74CE0101968C
:105C10000E94F815CE0101960E94EE73CC5ADE4F19
:105C200068817981C455D14066537109CE010196CE
:105C30000E94DB71CE0101960E94E115CE01019612
:105C40000E94EE734091380C5091390C60913A0CDF
:105C500070913B0C21E0CE0107960E94F67361E142
:105C600075E0CE0101960E948D74BE01695F7F4F81
:105C7000CE0101960E9409736CE175E00E94F372F7
:105C8000BC01CE010D960E948474CE010D960E9437
:105C9000E115CE010D960E94EE73CE0101960E9491
:105CA000EE73CE0107960E94EE734091340C509132
:105CB000350C6091360C7091370C21E0CE010796BF
:105CC0000E94F67361E275E0CE0101960E948D7428
:105CD000BE01695F7F4FCE0101960E9409736CE19E
:105CE00075E00E94F372BC01CE010D960E9484748F
:105CF000CE010D960E94E115CE010D960E94EE7325
:105D0000CE0101960E94EE73CE0107960E94EE73BB
:105D100067E776E0CE0101960E947B74CE01019682
:105D20000E94F815CE0101960E94EE73409129025F
:105D300050912A0260912B0270912C0225E0CE0135
:105D400001960E94F673CE0101960E94E115CE01E4
:105D500001960E94EE736DE576E0CE0101960E94F9
:105D60007B74CE0101960E94F815CE0101960E9427
:105D7000EE734091250250912602609127027091A6
:105D8000280225E0CE0101960E94F673CE0101960D
:105D90000E94E115CE0101960E94EE736DE476E05B
:105DA000CE0101960E947B74CE0101960E94F815E7
:105DB000CE0101960E94EE7360916E0270916F02A7
:105DC000CE0101960E94DB71CE0101960E94E11581
:105DD000CE0101960E94EE736BE376E0CE01019650
:105DE0000E947B74CE0101960E94F815CE010196A7
:105DF0000E94EE73C65BDE4F68817981CA54D14040
:105E0000CE0101960E94DB71CE0101960E94E11540
:105E1000CE0101960E94EE73CE0143960E94EE736E
:105E200068960FB6F894DEBF0FBECDBFDF91CF915D
:105E30001F910F91FF90EF90DF90CF9008956CE647
:105E400076E0CE0101960E948D74CE0101960E94EB
:105E5000F815CE0101960E94EE73CC5ADE4F688190
:105E60007981C455D140E2CE2F923F924F925F92FA
:105E70006F927F928F929F92AF92BF92CF92DF925A
:105E8000EF92FF920F931F93CF93DF93CDB7DEB7BF
:105E9000EC970FB6F894DEBF0FBECDBF9CA78BA7C3
:105EA0001B0170E060E00E94A772182F63EC78E09D
:105EB000CE0149960E948D7480916E0290916F027E
:105EC000019709F07AC082E090E00E94B67988E0FC
:105ED00090E0909324028093230289E090E09093D5
:105EE0002202809321028091B30B9091B40B909386
:105EF000B20B8093B10B80911D0290911E02A09174
:105F00001F02B09120028093190290931A02A0936D
:105F10001B02B0931C028091350290913602A09131
:105F20003702B09138028093390290933A02A093DD
:105F30003B02B0933C028091B00B8093AF0B8091F9
:105F4000AB0B9091AC0BA091AD0BB091AE0B8093CD
:105F5000A70B9093A80BA093A90BB093AA0B8AE36D
:105F600090E090931802809317028091380C9091E2
:105F7000390CA0913A0CB0913B0C8093E20B9093BA
:105F8000E30BA093E40BB093E50B80911502909185
:105F9000160290931402809313028091290290912B
:105FA0002A02A0912B02B0912C0280932D02909393
:105FB0002E02A0932F02B093300280916E02909136
:105FC0006F02029709F07AC083E090E00E94B679F0
:105FD0008AE090E090932402809323028BE090E08B
:105FE00090932202809321028091A50B9091A60BA1
:105FF0009093B20B8093B10B80910F02909110029D
:10600000A0911102B09112028093190290931A028A
:10601000A0931B02B0931C02809131029091320236
:10602000A0913302B09134028093390290933A02E6
:10603000A0933B02B0933C028091A40B8093AF0BE2
:106040008091A00B9091A10BA091A20BB091A30BFA
:106050008093A70B9093A80BA093A90BB093AA0BC6
:106060008BE390E090931802809317028091340C98
:106070009091350CA091360CB091370C8093E20BC7
:106080009093E30BA093E40BB093E50B80910D028A
:1060900090910E0290931402809313028091250236
:1060A00090912602A0912702B091280280932D02A0
:1060B00090932E02A0932F02B09330021335C1F4B7
:1060C0001092B20B1092B10B8091B90B882371F032
:1060D00068E275E0CE0101960E948D74CE010196B2
:1060E0000E94E115CE0101960E94EE73E12CE1C001
:1060F000C1010197029708F07AC181E090E0A0E029
:10610000B0E08093190290931A02A0931B02B093FF
:106110001C02ABA5BCA514968D919C911597029776
:1061200050F141E050E0BD01CE0101960E94971967
:10613000BE016F5F7F4FCE0149960E94B573CE01BD
:1061400001960E94EE73CE014996B1E02B16310400
:1061500071F50E94347220E030E040E251E40E9488
:1061600080A80E94A6AA6093190270931A028093D5
:106170001B0290931C0281E090E09093B20B8093FD
:10618000B10B1134F9F48091B90B882371F06DE2F1
:1061900075E0CE0101960E948D74CE0101960E9499
:1061A000E115CE0101960E94EE73E12C4FC00E94D2
:1061B000347220912D0230912E0240912F02509185
:1061C0003002CDCF163409F0FCC08091B90B882382
:1061D00071F066E375E0CE0101960E948D74CE01E8
:1061E00001960E94F815CE0101960E94EE73EE24EE
:1061F000E394F12C60E0809121020E94D87664E65D
:1062000070E080E090E00E9491776E2D80912302F3
:106210000E94D87664EF71E080E090E00E94917770
:1062200060E0809121020E94D87664E670E080E010
:1062300090E00E9491776E2D809123020E94D87683
:1062400064EF71E080E090E00E9491778091B90B5B
:10625000882379F14091190250911A0260911B0232
:1062600070911C022AE0CE0101960E942C74BE019E
:106270006F5F7F4FCE0107960E9484746AE475E0D9
:10628000CE0107960E94F372BC01CE010D960E94CA
:106290008474CE010D960E94E115CE010D960E94E8
:1062A000EE73CE0107960E94EE73CE0101960E9416
:1062B000EE738091190290911A02A0911B02B09185
:1062C0001C02181619061A061B060CF053C51634C4
:1062D00009F459C4123509F45AC46E2D8091230271
:1062E0000E94D87664EF71E080E090E00E949177A0
:1062F0006E2D809123020E94D87660ED77E080E0D9
:1063000090E00E9491776E2D809123020E94D876B2
:106310006CED75E080E090E00E94917781E090E084
:106320009093B20B8093B10B61E0809121020E94A7
:10633000D87661E070E080E090E00E94917760E0C4
:10634000809121020E94D8766AE070E080E090E0BF
:106350000E949177C12CD12C7601C39480911902AF
:1063600090911A02A0911B02B0911C02C816D90686
:10637000EA06FB060CF00DC46091B10B809121027E
:106380000E94D87661E070E080E090E00E94917712
:1063900060E0809121020E94D8766091390270916C
:1063A0003A0280913B0290913C026F5F7F4F8F4F8A
:1063B0009F4F0E949177FFEFCF1ADF0AEF0AFF0A83
:1063C000CDCF123591F48091B90B882371F060E440
:1063D00075E0CE0101960E948D74CE0101960E9457
:1063E000F815CE0101960E94EE73E12C03CF211423
:1063F000310429F0E3E02E16310409F077CE8091C4
:106400006E0290916F0220E137E240E050E081306F
:10641000910521F420E43CE940E050E02FA738AB9F
:1064200049AB5AAB21E030E03093B20B2093B10B73
:1064300030935D0220935C02029761F433E02316EF
:10644000310441F48091C9109091CA1090935D027B
:1064500080935C0240915C0250915D025EA74DA763
:10646000052F001F0027001F81E090E090935D0240
:1064700080935C0260E0809121020E94D87664E6FD
:1064800070E080E090E00E949177602F809123027D
:106490000E94D87664EF71E080E090E00E949177EE
:1064A000602F809123020E94D87668EE73E080E02E
:1064B00090E00E94917760E0809121020E94D8765E
:1064C00064E670E080E090E00E949177602F809118
:1064D00023020E94D87664EF71E080E090E00E9491
:1064E00091778FEF9FEF9093140280931302812C8A
:1064F000912C54011FA218A619A61AA61BA21CA211
:106500001DA21EA21F8E18A219A21AA2412C512C44
:1065100032011FAA18AE19AE1AAE1BAA1CAA1DAAD8
:106520001EAA61E0809121020E94D87661E070E0AD
:1065300080E090E00E94917760E0809121020E94CB
:10654000D87661E070E080E090E00E949177C5012C
:10655000B40126E030E040E050E00E9486A9672BBD
:10656000682B692B09F0F8C0A2E0B0E0BCAFABAF7C
:10657000C12CD12C760180911702863308F0865306
:1065800020917B00982F9870277F922B90937B000F
:106590008770806480937C0080917A00806480930F
:1065A0007A0080917A0086FDFCCF8091780060911E
:1065B0007900762F682F072E000C880B990B0E940C
:1065C00021A89B01AC01C701B6010E94C8A96B01BB
:1065D0007C0162E070E080E090E00E9491772BAD5A
:1065E0003CAD2130310509F0ADC020E030EC4FEF7B
:1065F00054E4C701B6010E9434AA6B017C0180916A
:10660000B90B882399F12DEC3CEC4CE45EE3C70117
:10661000B6010E94DCAA87FD29C022E0B701A601CD
:10662000CE0107960E94F67361E575E0CE010196F2
:106630000E948D74BE01695F7F4FCE0101960E945A
:106640000973BC01CE010D960E948474CE010D9693
:106650000E94E115CE010D960E94EE73CE010196C7
:106660000E94EE73CE0107960E94EE732AE939E983
:1066700049E95EE3C701B6010E94DCAA87FD13C0A9
:10668000411451046104710411F4240135018BA1FA
:106690009CA1ADA1BEA1892B8A2B8B2B21F48BA2AF
:1066A0009CA2ADA2BEA22DEC3CEC4CE45EE3C70183
:1066B000B6010E941AA818160CF449C041145104DE
:1066C0006104710409F448C02F8D38A149A15AA171
:1066D000232B242B252B69F48FA198A5A9A5BAA556
:1066E000892B8A2B8B2B09F403C18F8E98A2A9A228
:1066F000BAA22F8D38A149A15AA1421653066406A9
:10670000750654F5809113029091140297FFF5C01D
:106710001092140210921302420E531E641E751E34
:10672000D301C201B595A795979587958FAB98AF83
:10673000A9AFBAAF1F8E18A219A21AA2412C512CD0
:1067400032010AC0E1E0F0E0FCAFEBAF14CF41143E
:1067500051046104710469F6E0901302F090140290
:1067600092E0E916F1043CF4F7FCE3C0A3E02A163A
:10677000310409F0DEC08FA498A8A9A8BAA8BAE08D
:106780008B0E911CA11CB11C8FA598A9A9A9BAA90F
:1067900088169906AA06BB060CF4C3CEF2E0EF16E3
:1067A000F1040CF479C06BA97CA98DA99EA92FA92D
:1067B00038AD49AD5AAD621B730B840B950B0E942B
:1067C00021A84B015C01B701FF0C880B990B0E94BB
:1067D00021A89B01AC01C501B4010E9434AA20E0AC
:1067E00030E044EB53E40E9434AA6B017C01C09278
:1067F0002D02D0922E02E0922F02F092300220E081
:1068000030E040E85FE30E94DCAA87FDACC08091E5
:106810006E0290916F028130910509F090C0C09294
:10682000C110D092C210E092C310F092C410C09276
:106830002902D0922A02E0922B02F0922C0261EC03
:1068400075E0CE0101960E947B74CE0101960E94F4
:10685000F815CE0101960E94EE7340912D025091E1
:106860002E0260912F027091300225E0CE01019638
:106870000E94F673CE0101960E94E115CE010196A9
:106880000E94EE7384EF91E090936702809366021A
:1068900063EA7FE00E949C0833E02316310429F06C
:1068A000E02E2114310409F004CD8BA59CA50E9493
:1068B00034726B017C01C092E20BD092E30BE09248
:1068C000E40BF092E50B20E030E044EB53E4C70129
:1068D000B6010E94DCAA87FD6AC020E030E044EBEC
:1068E00053E4C701B6010E94C7A96B017C01EBCF3D
:1068F0008FA298A6A9A6BAA6F8CE2114310409F051
:106900002BCF019690931402809313022F8D38A100
:1069100049A15AA1420E531E641E751ED301C20125
:10692000B595A795979587958BAB9CABADABBEAB5B
:1069300001CFEFEF8E1A9E0AAE0ABE0A25CF02974C
:1069400009F07DCFC092C510D092C610E092C7105A
:10695000F092C810C0922502D0922602E09227023F
:10696000F09228026CCF65EA75E0CE0101960E9494
:106970007B74CE0101960E94F815CE0101960E940B
:10698000EE7340912D0250912E0260912F02709172
:10699000300225E0CE0101960E94F673CE010196E9
:1069A0000E94E115CE0101960E94EE7375CF20E0A2
:1069B00030E0A901C701B6010E941AA887FF0BC0E9
:1069C00020E030E044EB53E4C701B6010E94C8A9BF
:1069D0006B017C01ECCFC092A70BD092A80BE09288
:1069E000A90BF092AA0B4FA058A469A47AA48BA17A
:1069F0009CA1ADA1BEA1481A590A6A0A7B0A2114BA
:106A00003104D9F41092A70B1092A80B1092A90B85
:106A10001092AA0BADA5BEA5C12CD12C7601C394B2
:106A2000812C912C5401B7FF1CC0812C912C540156
:106A3000CC24CA94DC2C760114C0EDA5FEA5C12C93
:106A4000D12C7601C394F7FF04C0CC24CA94DC2C6B
:106A500076018090A70B9090A80BA090A90BB09006
:106A6000AA0B20912D0230912E0240912F025091BD
:106A70003002C501B4010E9480A84B015C01A30152
:106A80009201C701B6010E9454A90E9421A820E0EA
:106A900030E040E05FE30E9480A89B01AC01C501AB
:106AA000B4010E94C7A90E94A6AA6093190270931C
:106AB0001A0280931B0290931C028091B90B8823C9
:106AC00009F441C02AE04FA158A569A57AA5CE01D5
:106AD0000D960E942C742AE04BA15CA16DA17EA1B1
:106AE000CE0107960E942C7468E575E0CE010196F0
:106AF0000E948D74BE01695F7F4FCE0101960E9496
:106B000009736FEE75E00E94F372BE01635F7F4F01
:106B10000E940973BC01CE0143960E948474CE0189
:106B200043960E94E115CE0143960E94EE73CE017A
:106B300001960E94EE73CE0107960E94EE73CE017D
:106B40000D960E94EE738091190290911A02A09105
:106B50001B02B0911C02E12C12E5B7FFAACBB09545
:106B6000A095909581959F4FAF4FBF4F809319028D
:106B700090931A02A0931B02B0931C02EE24E3949C
:106B8000F12C16E496CBEE24E394F12CA6CBE12C69
:106B9000A4CB22E02216310424F42114310409F09C
:106BA000E1C061E080E00E94347D32E023163104D0
:106BB00024F42114310409F09CC0C090E20BD09061
:106BC000E30BE090E40BF090E50B20E030E044EBC9
:106BD00053E4C701B6010E94DCAA87FD0BC020E088
:106BE00030E044EB53E4C701B6010E94C7A96B0132
:106BF0007C01EBCF20E030E0A901C701B6010E9483
:106C00001AA887FF0BC020E030E044EB53E4C70133
:106C1000B6010E94C8A96B017C01ECCFC092E20BC7
:106C2000D092E30BE092E40BF092E50B80916E02C0
:106C300090916F020197B1F461E175E082E09FE00D
:106C40000E94D1718091E20B9091E30BA091E40B33
:106C5000B091E50B8093380C9093390CA0933A0CCB
:106C6000B0933B0C80916E0290916F020297B1F449
:106C700061E275E082E09FE00E94D1718091E20BB9
:106C80009091E30BA091E40BB091E50B8093340C51
:106C90009093350CA093360CB093370C4091E20BD7
:106CA0005091E30B6091E40B7091E50B20E0CE0175
:106CB00007960E94F67362E07FE0CE0101960E9483
:106CC0008474BE01695F7F4FCE0101960E940973F3
:106CD0006DE175E00E94F372BC0182E09FE00E94CA
:106CE0009E73CE0101960E94EE73CE0107960E941C
:106CF000EE7341E02416310439F5409119025091A8
:106D00001A0260911B0270911C0221E0CE010796CD
:106D10000E942C7460E675E0CE0101960E948D748D
:106D2000BE01695F7F4FCE0101960E940973BC01CD
:106D300082E09FE00E949E73CE0101960E94EE7356
:106D4000CE0107960E94EE7362E07FE0CE010196CD
:106D50000E948474CE0101960E94FF20CE0101960C
:106D60000E94EE731092190210921A0210921B02E6
:106D700010921C0280916E0290916F0281309105F9
:106D800009F083C08091B10B9091B20B9093B40B3A
:106D90008093B30B8091190290911A02A0911B026B
:106DA000B0911C0280931D0290931E02A0931F02BB
:106DB000B09320028091390290913A02A0913B0257
:106DC000B0913C028093350290933602A093370233
:106DD000B09338028091AF0B8093B00B8091A70BDA
:106DE0009091A80BA091A90BB091AA0B8093AB0B2B
:106DF0009093AC0BA093AD0BB093AE0B8091E20BD4
:106E00009091E30BA091E40BB091E50B8093380CCB
:106E10009093390CA0933A0CB0933B0C80911302E1
:106E2000909114029093160280931502232881F406
:106E300080912D0290912E02A0912F02B0913002EC
:106E40008093290290932A02A0932B02B0932C02E4
:106E5000CE0149960E94EE73EC960FB6F894DEBF11
:106E60000FBECDBFDF91CF911F910F91FF90EF909B
:106E7000DF90CF90BF90AF909F908F907F906F905A
:106E80005F904F903F902F900895029709F780915F
:106E9000B10B9091B20B9093A60B8093A50B8091B0
:106EA000190290911A02A0911B02B0911C028093CA
:106EB0000F0290931002A0931102B09312028091DE
:106EC000390290913A02A0913B02B0913C0280932A
:106ED000310290933202A0933302B0933402809136
:106EE000AF0B8093A40B8091A70B9091A80BA0915E
:106EF000A90BB091AA0B8093A00B9093A10BA09328
:106F0000A20BB093A30B8091E20B9091E30BA091A5
:106F1000E40BB091E50B8093340C9093350CA09367
:106F2000360CB093370C8091130290911402909319
:106F30000E0280930D02232809F08ACF80912D0242
:106F400090912E02A0912F02B091300280932502E1
:106F500090932602A0932702B093280279CF2F9214
:106F60003F924F925F926F927F928F929F92AF92D9
:106F7000BF92CF92DF92EF92FF920F931F93CF9326
:106F8000DF93CDB7DEB7E3970FB6F894DEBF0FBE41
:106F9000CDBF60E27FE0CE018E960E9484740EA584
:106FA0001FA50115110571F0D8018D918D01882360
:106FB00049F0082E000C990B0E9428ADF80131977A
:106FC0008083F2CF67E675E0CE0101960E948D7452
:106FD000BE016F5F7F4FCE018E960E94D872182F30
:106FE000CE0101960E94EE73112309F401C145E020
:106FF00050E060E27FE0CE0101960E949719BE0149
:107000006F5F7F4F8CEF9EE00E94B573CE010196BB
:107010000E94EE738CEF9EE00E944A7260E08CEF5B
:107020009EE00E9446734091000F5091010F6BEF5C
:107030007FE08CEF9EE00E9425716AE674E0CE014D
:1070400001960E948D74BE016F5F7F4F8CEF9EE0B2
:107050000E94D872182FCE0101960E94EE7364E54B
:1070600074E0111102C069E574E0CE0101960E943E
:107070008D746CEF7EE0CE0101960E940973BC0115
:1070800081E091E10E949E73CE0101960E94EE7311
:1070900081E091E10E944A724091051150910611E0
:1070A0004150510961E071E1CE0101960E949719AA
:1070B000BE016F5F7F4F83EE90E10E94B573CE01FA
:1070C00001960E94EE7383EE90E10E943F720E944F
:1070D00021A89B01AC010E94E1AA882309F448C0C1
:1070E00060910511709106116250710981E091E182
:1070F0000E94A772682FCE0101960E945974BE01AA
:107100006F5F7F4F83EE90E10E94B573CE010196D1
:107110000E94EE736AE674E0CE0101960E948D74BF
:10712000BE016F5F7F4F83EE90E10E94D872182FEF
:10713000CE0101960E94EE731123D1F060910511EA
:10714000709106116350710981E091E10E94A7726C
:10715000682FCE0101960E945974BE016F5F7F4F68
:1071600083EE90E10E94B573CE0101960E94EE730A
:1071700084EF91E0909367028093660263EA7FE078
:107180000E949C0864E670E080E090E00E949177A5
:1071900080913D02882371F060E27FE0CE0101968C
:1071A0000E948474CE0101960E94CD1ACE010196F0
:1071B0000E94EE73CE018E960E94EE7381E0E396FC
:1071C0000FB6F894DEBF0FBECDBFDF91CF911F91F8
:1071D0000F91FF90EF90DF90CF90BF90AF909F9076
:1071E0008F907F906F905F904F903F902F90089579
:1071F0006DE675E0CE0101960E948D74BE016F5F51
:107200007F4FCE018E960E94D872182FCE01019624
:107210000E94EE73112309F447C045E050E060E29C
:107220007FE0CE0101960E949719BE016F5F7F4FEC
:107230008CEF9EE00E94B573CE0101960E94EE7322
:107240008CEF9EE00E944A7260E08CEF9EE00E940C
:1072500046734091000F5091010F63ED7FE08CEF7A
:107260009EE00E94257163ED7FE0CE014C960E9466
:107270008D746CE674E0CE0101960E948D74BE019F
:10728000645E7F4FCE0101960E940973BC018BEFB3
:1072900090E10E949E73CE0101960E94EE73CE0192
:1072A0004C960E94EE7364CF63E775E0CE010196C1
:1072B0000E948D74BE016F5F7F4FCE018E960E943B
:1072C000D872182FCE0101960E94EE731123E1F0BF
:1072D00043E050E060E27FE0CE0101960E94971902
:1072E000BE016F5F7F4F8CEF9EE00E94B573CE01B1
:1072F00001960E94EE736CEF7EE0CE0101960E9433
:107300008474CE010196CDCF67E775E0CE0101967A
:107310000E948D74BE016F5F7F4FCE018E960E94DA
:10732000D872182FCE0101960E94EE73112301F13D
:1073300044E050E060E27FE0CE0101960E949719A0
:10734000BE016F5F7F4F8CEF9EE00E94B573CE0150
:1073500001960E94EE738CEF9EE00E943F72709344
:1073600062106093611070938F0260938E0200CF61
:107370006CE775E0CE0101960E948D74BE016F5FCF
:107380007F4FCE018E960E94D872182FCE010196A3
:107390000E94EE73112309F449C045E050E060E219
:1073A0007FE0CE0101960E949719BE016F5F7F4F6B
:1073B0008CEF9EE00E94B573CE0101960E94EE73A1
:1073C0008CEF9EE00E943F727093BE106093BD10E0
:1073D00084EF91E0909367028093660263EA7FE016
:1073E0000E949C0864E670E080E090E00E94917743
:1073F0006BE777E0CE0101960E948D7460E27FE03A
:10740000CE0101960E940973BC01CE014C960E94E8
:107410008474CE014C960E94E115CE014C960E94D8
:10742000EE73CE0101960E94EE73B2CE62E875E073
:10743000CE0101960E948D74BE016F5F7F4FCE0119
:107440008E960E94D872182FCE0101960E94EE737C
:107450001123E1F044E050E060E27FE0CE010196CC
:107460000E949719BE016F5F7F4F8CEF9EE00E94D4
:10747000B573CE0101960E94EE738CEF9EE00E94E0
:107480003F727093C0106093BF10A2CF67E875E0A1
:10749000CE0101960E948D74BE016F5F7F4FCE01B9
:1074A0008E960E94D872182FCE0101960E94EE731C
:1074B0001123A1F044E050E060E27FE0CE010196AC
:1074C0000E949719BE016F5F7F4F8CEF9EE00E9474
:1074D000B573CE0101960E94EE7384CF6CE875E01F
:1074E000CE0101960E948D74BE016F5F7F4FCE0169
:1074F0008E960E94D872182FCE0101960E94EE73CC
:107500001123A1F047E050E060E27FE0CE01019658
:107510000E949719BE016F5F7F4F8CEF9EE00E9423
:10752000B573CE0101960E94EE732CCE64E975E02E
:10753000CE0101960E948D74BE016F5F7F4FCE0118
:107540008E960E94D872182FCE0101960E94EE737B
:107550001111D8CF6CE975E0CE0101960E948D74AF
:10756000BE016F5F7F4FCE018E960E94D872182F9A
:10757000CE0101960E94EE73112321F081E00E945A
:107580002B0800CE66EA75E0CE0101960E948D744C
:10759000BE016F5F7F4FCE018E960E94D872182F6A
:1075A000CE0101960E94EE73112319F00E94D92793
:1075B000E9CD6BE679E0CE0101960E947B74BE01B5
:1075C0006F5F7F4FCE018E960E94D872182FCE012A
:1075D00001960E94EE73112309F485C060E679E0FC
:1075E000CE0101960E947B74BE016F5F7F4FCE017A
:1075F0008E960E94D872182FCE0101960E94EE73CB
:10760000112309F454C04AE050E060E27FE0CE016B
:1076100001960E949719BE016F5F7F4F8CEF9EE02D
:107620000E94B573CE0101960E94EE738CEF9EE02E
:107630000E943F720E944B790E9470796093460CC1
:107640007093470C8093480C9093490C0E9470797A
:107650006093400C7093410C8093420C9093430CC8
:10766000CE014C960E947A1B6DEA75E0CE01019620
:107670000E948D74BE01645E7F4FCE0101960E9410
:107680000973BC01CE0182960E948474CE01829659
:107690000E94E115CE0182960E94EE73CE01019602
:1076A0000E94EE73CE014C960E94EE7371CD4BE0BA
:1076B00050E060E27FE0CE0101960E949719BE0182
:1076C0006F5F7F4F8CEF9EE00E94B573CE010196F5
:1076D0000E94EE738CEF9EE00E943F7260587F48DC
:1076E0008F4F9F4FA7CF63EF76E0CE0101960E94A8
:1076F0008D74BE016F5F7F4FCE018E960E94D8724F
:10770000182FCE0101960E94EE73112309F46AC06E
:1077100045E050E060E27FE0CE0101960E949719BB
:10772000BE016F5F7F4F8CEF9EE00E94B573CE016C
:1077300001960E94EE730E9470796093460C7093DC
:10774000470C8093480C9093490C8CEF9EE00E946C
:107750003F726093700270937102809372029093F3
:1077600073026093A3107093A4108093A51090935C
:10777000A6102091A2102093580C672B682B692B20
:1077800011F41092580C84EF91E09093670280936B
:10779000660263EA7FE00E949C0864E670E080E095
:1077A00090E00E94917761E579E0CE0101960E9418
:1077B0007B74CE0101960E94F815CE0101960E94BD
:1077C000EE7340917002509171026091720270915B
:1077D0007302CE0101960E940772CE0101960E94AB
:1077E000E115DBC16EEB75E0CE0101960E948D7450
:1077F000BE016F5F7F4FCE018E960E94D872182F08
:10780000CE0101960E94EE731123D9F14AE050E0B7
:1078100060E27FE0CE0101960E949719BE016F5F82
:107820007F4F8CEF9EE00E94B573CE0101960E94BF
:10783000EE738CEF9EE00E943F726130710581050E
:10784000910519F481E08093A2108CEF9EE00E94D4
:107850003F72672B682B692B11F41092A210809154
:10786000A2108093580C882309F4B2CD0E9470793D
:107870006093460C7093470C8093480C9093490C8E
:10788000A7CD69EC75E0CE0101960E948D74BE0112
:107890006F5F7F4FCE018E960E94D872182FCE0157
:1078A00001960E94EE731123A1F048E050E060E2DF
:1078B0007FE0CE0101960E949719BE016F5F7F4F56
:1078C0008CEF9EE00E94B573CE0101960E94EE738C
:1078D0008FCD62ED75E0CE0101960E948D74BE01E0
:1078E0006F5F7F4FCE018E960E94D872182FCE0107
:1078F00001960E94EE73112321F145E050E060E211
:107900007FE0CE0101960E949719BE016F5F7F4F05
:107910008CEF9EE00E94B573CE0101960E94EE733B
:107920008CEF9EE00E943F726130710521F481E08E
:107930008093590C2DCC672B09F02ACC1092590C4E
:1079400027CC68ED75E0CE0101960E948D74BE01D2
:107950006F5F7F4FCE018E960E94D872182FCE0196
:1079600001960E94EE73112351F163E070E080E212
:107970009FE00E94A772682FCE0101960E94597461
:10798000BE016F5F7F4F8CEF9EE00E94B573CE010A
:1079900001960E94EE738CEF9EE00E944A728CEF7B
:1079A0009EE00E943F729B01215031092330310536
:1079B00008F0EECB7093D2106093D110D9CB6CED60
:1079C00075E0CE0101960E948D74BE016F5F7F4FFE
:1079D000CE018E960E94D872182FCE0101960E9479
:1079E000EE73112309F46AC066E070E080E29FE064
:1079F0000E94A772682FCE0101960E945974BE01A1
:107A00006F5F7F4F8CEF9EE00E94B573CE010196B1
:107A10000E94EE738CEF9EE00E944A7260E08CEF51
:107A20009EE00E9446738CEF9EE00E943F726B01C5
:107A3000CB010197039708F0ABCB48E050E060E240
:107A40007FE0CE0101960E949719BE016F5F7F4FC4
:107A50008CEF9EE00E94B573CE0101960E94EE73FA
:107A60008CEF9EE00E944A728091000F9091010F6E
:107A70000997A8F028E030E050E040E06CEF7EE0AD
:107A8000CE0101960E94A274BE016F5F7F4F8CEF02
:107A90009EE00E94B573CE0101960E94EE73B6017E
:107AA00013E0660F771F1A95E1F76954704F48E0AD
:107AB00050E08CEF9EE00E9425715ACB69E479E09A
:107AC000CE0101960E947B74BE016F5F7F4FCE0195
:107AD0008E960E94D872182FCE0101960E94EE73E6
:107AE000112309F486C063EC78E0CE0101960E9470
:107AF0008D7447E050E0BE01625D7F4FCE014C9631
:107B00000E949719BE01645E7F4FCE0101960E94CC
:107B1000B573CE014C960E94EE7364E075E0CE0121
:107B20004C960E948D74BE01645E7F4FCE0101961B
:107B30000E94D872182FCE014C960E94EE7311232A
:107B400079F141E050E0BE016F5F7F4FCE014C966E
:107B50000E949719CE014C960E943F728B010A5CDD
:107B60001F4FCE014C960E94EE731093D4100093D9
:107B7000D310109391020093900284EF91E09093C0
:107B800067028093660263EA7FE00E949C0864E6D5
:107B900070E080E090E00E949177CE01019684CD64
:107BA0006CE676E0CE014C960E948D74BE01645E58
:107BB0007F4FCE0101960E94D872182FCE014C96AD
:107BC0000E94EE73112379F041E050E0BE016F5F37
:107BD0007F4FCE014C960E949719CE014C960E9481
:107BE0003F728B01BECFCE0101960E943F728B0186
:107BF000BCCF62E479E0CE0101960E947B74BE01A5
:107C00006F5F7F4FCE018E960E94D872182FCE01E3
:107C100001960E94EE73112309F4AAC062EF75E089
:107C2000CE0101960E948D7446E050E0BE016F5F68
:107C30007F4FCE018E960E94F39D8C01CE0101965E
:107C40000E94EE73980146E050E0BE01625D7F4FF6
:107C5000CE0101960E94A274CE0101960E943F724D
:107C60006B01CE0101960E94EE7363EC78E0CE01C9
:107C700001960E948D74A8014F5F5F4FBE01625D47
:107C80007F4FCE014C960E949719BE01645E7F4FD4
:107C9000CE0101960E94B573CE014C960E94EE7300
:107CA00064E075E0CE014C960E948D74BE01645E66
:107CB0007F4FCE0101960E94D872182FCE014C96AC
:107CC0000E94EE73112321F141E050E0BE016F5F8D
:107CD0007F4FCE014C960E949719CE014C960E9480
:107CE0003F728B010A5C1F4FCE014C960E94EE73CF
:107CF000F6013196EE0FFF1FED55F04F1183008313
:107D0000F601EE0FFF1FEA50F44F1183008335CFC9
:107D10006CE676E0CE014C960E948D74BE01645EE6
:107D20007F4FCE0101960E94D872182FCE014C963B
:107D30000E94EE73112379F041E050E0BE016F5FC5
:107D40007F4FCE014C960E949719CE014C960E940F
:107D50003F728B01C9CFCE0101960E943F72009104
:107D6000F80B1091F90B01501109060F171FC0CF26
:107D700069E374E0CE014C960E948D74BE01645E8E
:107D80007F4FCE018E960E94D87211E0811115C0EE
:107D900063EE75E0CE0101960E948D74BE016F5FA7
:107DA0007F4FCE018E960E94D87211E0811101C0E2
:107DB00010E0CE0101960E94EE73CE014C960E9417
:107DC000EE73112309F411C26FEE75E0CE014C96EB
:107DD0000E948D746AEE75E0CE0101960E948D744A
:107DE000AE01445E5F4FBE016F5F7F4FCE018E9646
:107DF0000E94FA9CCE0101960E94EE73CE014C9631
:107E00000E94EE736FEE75E0CE014C960E948D7469
:107E10006CEE75E0CE0101960E948D74AE01445E59
:107E20005F4FBE016F5F7F4FCE018E960E94FA9C1E
:107E3000CE0101960E94EE73CE014C960E94EE7325
:107E40006FEE75E0CE014C960E948D746EEE75E07B
:107E5000CE0101960E948D74AE01445E5F4FBE015B
:107E60006F5F7F4FCE018E960E94FA9CCE010196E5
:107E70000E94EE73CE014C960E94EE7362EF75E0A5
:107E8000CE014C960E948D7461EF75E0CE01019693
:107E90000E948D74AE01445E5F4FBE016F5F7F4FE5
:107EA000CE018E960E94FA9CCE0101960E94EE733E
:107EB000CE014C960E94EE7362EF75E0CE014C96B7
:107EC0000E948D746FE178E0CE0101960E948D745E
:107ED000AE01445E5F4FBE016F5F7F4FCE018E9655
:107EE0000E94FA9CCE0101960E94EE73CE014C9640
:107EF0000E94EE73CE018E960E944A720E947079A3
:107F000060934A0C70934B0C80934C0C90934D0CE7
:107F100056E0E52EF12C64E6462E512C612C712C96
:107F200022242394312C5701B3E0AB0EB11C8AA953
:107F30009BA90197A816B90608F02AC9B701CE0176
:107F40008E960E94A772682FCE014C960E9459749B
:107F50006701E2E0CE0ED11CFFEFEF1AFF0A960197
:107F6000A701BE01625D7F4FCE0101960E94A274FF
:107F7000CE0101960E943F728B01CE0101960E94B4
:107F8000EE730130110521F40091BD101091BE1067
:107F90000330110521F40091BF101091C0106FEE55
:107FA00075E0CE0101960E948D74A601BE016F5F3F
:107FB0007F4FCE018E960E94F39D6C01CE010196FB
:107FC0000E94EE7363EC78E0CE0101960E948D74FE
:107FD000480181E0881A91081C141D042CF59601B3
:107FE000A501BE01625D7F4FCE0182960E94A27400
:107FF000BE016E5D7F4FCE0101960E94B573CE012A
:1080000082960E94EE7393E08916910420F1760126
:10801000AFEFEA1AFA0ACE0101960E94EE73CE0182
:108020004C960E94EE737FCFA501BE01625D7F4F2B
:10803000CE0182960E949719BE016E5D7F4FCE01E0
:1080400001960E94B573CE0182960E94EE73B3E052
:108050008B16910400F770E060E0CE014C960E9410
:10806000A772823509F061C0CE0101960E943F726D
:10807000672B682B692BB1F4F801EE0FFF1FE95253
:10808000FD4F11821082F801EE0FFF1FEE0FFF1F50
:10809000E154FD4F82E090E0A0E0B0E08083918366
:1080A000A283B383CE0101960E943F7261307105B5
:1080B00081059105A9F5F801EE0FFF1FE952FD4F6B
:1080C00031822082000F111F000F111FF801E154AF
:1080D000FD4F80819181A281B381181619061A067D
:1080E0001B0624F04082518262827382CE01019687
:1080F0000E943F7262307105810591053CF0F801E4
:10810000E154FD4F60837183828393830E94707971
:1081100001521D4FD8016D937D938D939C931397BE
:108120001C141D040CF473CF76CF8634E9F5CE0110
:1081300001960E943F72672B682B692B39F4F80176
:10814000EE0FFF1FEC5AFD4F11821082CE010196F7
:108150000E943F72613071058105910539F4F80183
:10816000EE0FFF1FEC5AFD4F31822082000F111FCE
:10817000000F111FF801E154FD4F80819181A28110
:10818000B381181619061A061B0624F04082518284
:10819000628273820E94707901521D4FF8016083E0
:1081A000718382839383BCCF843461F4CE010196C2
:1081B0000E943F72000F111F000F111FF801EC5BAE
:1081C000FD4FA0CF843509F0ABCFCE0101960E94C0
:1081D0003F72000F111F000F111FF801E154FD4FF6
:1081E0006083718382839383D5CF6CE379E0CE0182
:1081F00001960E947B74BE016F5F7F4FCE018E9609
:108200000E94D872182FCE0101960E94EE7311239E
:1082100009F49DC045E050E060E27FE0CE010196A8
:108220000E949719BE016F5F7F4F8CEF9EE00E9406
:10823000B573CE0101960E94EE738CEF9EE00E9412
:108240004A7260E08CEF9EE00E9446736EEC78E02C
:10825000CE014C960E948D746CEF7EE0CE010196AB
:108260000E948474AE014E5D5F4FBE01645E7F4F1D
:10827000CE0101960E940F9E182FCE0101960E94FA
:10828000EE73CE014C960E94EE73112311F40C9400
:10829000C8388E010E5D1F4F5DECA52E50E1B52E46
:1082A00060E4C62E62E0D62EF12CE12CD8016D914F
:1082B0008D01F50161935F01D6016D936D01CE01D2
:1082C00001960E94829CCE0101960E94F815CE0173
:1082D00001960E94EE73B3E0EB16F10471F06EECC0
:1082E00078E0CE0101960E948D74CE0101960E9425
:1082F000F815CE0101960E94EE73EFEFEE1AFE0A1A
:10830000F4E0EF16F10491F663EC78E0CE0101960B
:108310000E948D74CE0101960E94E115CE01019656
:108320000E94EE7363EA7FE080916602909167029B
:108330000E949C0864E670E080E090E00E949177E3
:1083400064E279E0CE0101960E947B7446CA6FE137
:1083500079E0CE0101960E947B74BE016F5F7F4F72
:10836000CE018E960E94D872182FCE0101960E94DF
:10837000EE73112309F47CC044E050E060E27FE03A
:10838000CE0101960E949719BE016F5F7F4F8CEF5F
:108390009EE00E94B573CE0101960E94EE738CEFB1
:1083A0009EE00E944A7260E08CEF9EE00E9446735D
:1083B0004091000F5091010F66EE7BE08CEF9EE044
:1083C0000E9425716EEC78E0CE014C960E948D746F
:1083D0006CEF7EE0CE0101960E948474AE014E5D8A
:1083E0005F4FBE01645E7F4FCE0101960E940F9EDB
:1083F000182FCE0101960E94EE73CE014C960E947A
:10840000EE73112311F40C94C8388E010E5D1F4FCA
:108410004FECE42E4FE0F42E6E0186E2C80ED11C24
:10842000D8016D918D01F70161937F01CE01019615
:108430000E94829CCE0101960E94E115CE01019618
:108440000E94EE730C151D0559F784EF91E090938F
:1084500067028093660263EA7FE00E949C0864E6FC
:1084600070E080E090E00E94917764E179E06ACF6B
:108470006DE079E0CE0101960E947B74BE016F5FD2
:108480007F4FCE018E960E94D872182FCE01019692
:108490000E94EE731123F1F146E050E060E27FE0CC
:1084A000CE0101960E949719BE016F5F7F4F8CEF3E
:1084B0009EE00E94B573CE0101960E94EE738CEF90
:1084C0009EE00E944A728091000F9091010F892BCB
:1084D00011F40C94C8388CEF9EE00E943F727093A8
:1084E000CC106093CB1070933F0260933E0284EFF8
:1084F00091E0909367028093660263EA7FE00E94B6
:108500009C0864E670E080E090E00E94917769EF5B
:1085100078E018CF62EF78E0CE0101960E947B747C
:10852000BE016F5F7F4FCE018E960E94D872182FCA
:10853000CE0101960E94EE731123B9F065EE78E04A
:10854000CE0101960E947B7444E650E06FEF7FEF0E
:10855000CE0101960E940109CE0101960E94EE73A0
:10856000F0E0E0E019950C94C8386DED78E0CE01AC
:1085700001960E947B74BE016F5F7F4FCE018E9685
:108580000E94D872182FCE0101960E94EE7311231B
:1085900001F164EF75E0CE0101960E948D7469EEE1
:1085A00070E1CE0101960E940973BC0182E09FE058
:1085B0000E949E73CE0101960E94EE7362E07FE0FE
:1085C000CE0101960E948474CE0101960E94E115AD
:1085D000ACC466ED78E0CE0101960E947B74BE01CA
:1085E0006F5F7F4FCE018E960E94D872182FCE01FA
:1085F00001960E94EE73112361F167EC78E082E04E
:108600009FE00E94797365EF70E18FEE90E10E9428
:108610009E736FEE70E1CE0101960E948474BE01DC
:108620006F5F7F4FCE014C960E94847460E0CE0154
:108630004C960E945A73BC0182E09FE00E947273C4
:10864000CE014C960E94EE73CE0101960E94EE730D
:10865000B5CF6FEF75E0CE0101960E948D74BE011B
:108660006F5F7F4FCE018E960E94D872182FCE0179
:1086700001960E94EE73112331F00E94E1281092BE
:108680003D020C94C83868E076E0CE014C960E941A
:108690008D74BE01645E7F4F80E29FE00E94D872BD
:1086A00011E0811115C06DE076E0CE0101960E94C7
:1086B0008D74BE016F5F7F4F80E29FE00E94D87291
:1086C00011E0811101C010E0CE0101960E94EE730D
:1086D000CE014C960E94EE73112309F441C062EF63
:1086E00075E0CE0101960E948D744091240F509147
:1086F000250F8D819E81481B590BBE016F5F7F4FF7
:1087000080E29FE00E94AC9CAC014F5F5F4F60E253
:108710007FE0CE014C960E949719BE01645E7F4FA8
:108720008CEF9EE00E94B573CE014C960E94EE73D2
:10873000CE0101960E94EE738CEF9EE00E943F7284
:108740006115710531F481E08093F0020E94F5908B
:1087500096CF6130710509F092CF1092F002F6CFFA
:1087600062E176E0CE0101960E948D74BE016F5FDA
:108770007F4FCE018E960E94D872182FCE0101969F
:108780000E94EE73112309F43BC143E050E060E224
:108790007FE0CE0101960E949719BE016F5F7F4F67
:1087A0008CEF9EE00E94B573CE0101960E94EE739D
:1087B0006CEF7EE0CE0101960E948474CE0101969A
:1087C0000E94CD1ACE0101960E94EE7384EF91E0D3
:1087D00090936702809366026CEF7EE0CE01019673
:1087E0000E94847460E0CE0101960E945A73BC011D
:1087F00085EF90E10E949E73CE0101960E94EE7378
:108800006CEF7EE0CE0101960E94847460E0CE01A0
:1088100001960E945A73BC018FEE90E10E949E73F4
:10882000CE0101960E94EE734091F9105091FA101A
:1088300063E670E185EF90E10E9425714091F310AD
:108840005091F4106EE670E18FEE90E10E94257178
:1088500063EA7FE080916602909167020E949C0823
:1088600066E176E0CE0101960E948D746CEF7EE0A9
:10887000CE0101960E940973BC01CE0182960E942E
:108880008474CE0101960E94EE7380915F109091E6
:108890006010892B39F4BE016E5D7F4F8FE99CE03B
:1088A0000E94C67568EB7BE080E090E00E949177C3
:1088B00080915F1090916010029709F087C06CEF73
:1088C0007EE0CE0188960E9484746EE176E0CE014F
:1088D00001960E948D74CE0101960E942191CE01D5
:1088E00001960E94EE7364EF71E080E090E00E94D8
:1088F000917761E276E0CE0101960E948D74CE01FF
:1089000001960E942191CE0101960E94EE736CEDBA
:1089100075E080E090E00E9491776AE276E0CE0117
:1089200001960E948D74CE0101960E942191CE0184
:1089300001960E94EE7364EF71E080E090E00E9487
:10894000917768E376E0CE0101960E948D74CE01A6
:1089500001960E942191CE0101960E94EE7364EF70
:1089600071E080E090E00E94917766E176E0CE01D0
:1089700001960E948D74BE01685D7F4FCE01019605
:108980000E940973BC01CE014C960E948474CE01F2
:1089900001960E94EE73CE014C960E944A72BE016F
:1089A000645E7F4FCE0101960E948474CE010196D1
:1089B0000E942191CE0101960E94EE73CE014C9649
:1089C0000E94EE73CE0188960E94EE7368EB7BE006
:1089D00080E090E00E94917763E670E1CE0101961D
:1089E0000E948D74CE0101960E94CD1ACE0101968F
:1089F0000E94EE7310923D02CE0182960C94543B7D
:108A000066E476E0CE0101960E948D74BE016F5F30
:108A10007F4FCE018E960E94D872182FCE010196FC
:108A20000E94EE73112309F486C044E050E060E236
:108A30007FE0CE0101960E949719BE016F5F7F4FC4
:108A40008CEF9EE00E94B573CE0101960E94EE73FA
:108A50006BE476E0CE0101960E948D746CEF7EE0AF
:108A6000CE0101960E940973BC01CE014C960E9472
:108A70008474CE0101960E94EE7380915F109091F4
:108A80006010892B39F4BE01645E7F4F8FE99CE052
:108A90000E94C67568E873E180E090E00E949177DB
:108AA00080915F1090916010029759F562E576E031
:108AB000CE0101960E948D748091000F9091010F5C
:108AC000892B19F56BE576E0CE0101960E94D171F4
:108AD000BE01645E7F4FCE0182960E948474CE01F7
:108AE00082960E942191CE0182960E94EE7368E8E0
:108AF00073E180E090E00E949177CE0101960E94A0
:108B0000EE7310923D020C94523BBE016F5F7F4F9B
:108B1000CE0182960E948474CE0182960E94219199
:108B2000CE0182960E94EE7360E777E180E090E0EC
:108B30000E949177CDCF64E676E0CE0101960E9447
:108B40008D74BE016F5F7F4FCE018E960E94D872EA
:108B5000182FCE0101960E94EE73112309F475C0FF
:108B600060E27FE08CEF9EE00E949E7381E0809344
:108B70003D0260E27FE0CE0101960E948474CE0146
:108B800001960E94CD1ACE0101960E94EE7380914B
:108B90005F1090916010029709F16CEF7EE08FE911
:108BA0009CE00E94C67568EB7BE080E090E00E944C
:108BB0009177CE0101960E94BA91BE016F5F7F4FFF
:108BC00080E29FE00E94B573CE0101960E94EE7391
:108BD00060ED77E080E090E00E94917780915F10F7
:108BE00090916010029771F46CEF7EE0CE010196D7
:108BF0000E948474CE0101960E942191CE010196BB
:108C00000E94EE738091240F9091250F892B09F417
:108C100036CD6BE777E0CE0101960E948D7460E25D
:108C20007FE0CE0101960E940973BC01CE014C96F3
:108C30000E948474CE014C960E94E115CE014C96A0
:108C40000E94EE73CE01019650C268E676E0CE0136
:108C500001960E948D74BE016F5F7F4FCE018E968C
:108C60000E94D872182FCE0101960E94EE73112334
:108C700009F495C180915F1090916010019709F0FF
:108C8000FECC6EE676E0CE0188960E948D74BE0121
:108C9000685D7F4F8FE99CE00E94C6756CE271E0D1
:108CA00080E090E00E949177CE0182960E94BA9176
:108CB00064E670E080E090E00E94917710E000E0D0
:108CC00025E0C22ED12C3AE0A32EB12C69E776E044
:108CD000CE0101960E948D7450E040E0BE016F5FAE
:108CE0007F4FCE0182960E94F39D7C01CE010196BA
:108CF0000E94EE73A7014F5F5F4FBE016E5D7F4F15
:108D0000CE0101960E949719BE016F5F7F4FCE0181
:108D100088960E94B573CE0101960E94EE738CA5D1
:108D20009DA5892B09F170E060E0CE0188960E9434
:108D3000A772082E000C990BC0970A97A8F46BE74E
:108D400076E0CE0101960E948D74BE016F5F7F4F69
:108D5000CE0188960E94D872E82ECE0101960E941C
:108D6000EE73FF24F394E110F12C66E677E0CE0178
:108D700001960E947B7464E170E0CE0101960E942E
:108D8000C99ECE0101960E94EE730F5F1F4F62E3F2
:108D900070E080E090E00E949177C801B6010E94E7
:108DA000E6AA0197C1F4CE0101960E94661C8D814E
:108DB0009E81892B09F4BEC0BE016F5F7F4F80E2A8
:108DC0009FE00E949E730E94AF37FF24F394CE0170
:108DD00001960E94EE73CE0101960E94BA91BE01E7
:108DE0006F5F7F4FCE0182960E94B573CE010196D0
:108DF0000E94EE7362E370E080E090E00E94917761
:108E00000436110519F0FF2009F460CF8091B90BE9
:108E10008823F1F06BE777E0CE014C960E948D74C9
:108E2000BE01685D7F4FCE014C960E940973BC0164
:108E3000CE0101960E948474CE0101960E94E11534
:108E4000CE0101960E94EE73CE014C960E94EE7305
:108E50008CA59DA5892B69F070E060E0CE01889615
:108E60000E94A772082E000C990BC0970A9708F46D
:108E70007AC063E876E0CE0101960E948D74CE013F
:108E800082960E94EE73CE0188960E94EE738D81C9
:108E90009E81009709F449C0E981FA81208122234B
:108EA00009F443C0079708F440C06EEB78E0CE01A8
:108EB0004C960E947B7468EC70E0CE014C960E9448
:108EC000C99ECE014C960E94EE73BE016F5F7F4F2C
:108ED000CE014C960E94847440ED57E06FEF7FEF17
:108EE000CE014C960E940109CE014C960E94EE7371
:108EF0006FE876E0CE014C960E948D7460E27FE0D0
:108F0000CE014C960E940973BC01CE0182960E944C
:108F10008474CE0182960E94E115CE0182960E9451
:108F2000EE73CE014C960E94EE73CE0101960E9424
:108F3000EE73A5CB043111050CF449CFC801B5017E
:108F40000E94E6AA892B09F042CFBE01685D7F4FDF
:108F50008FE99CE00E94C67568EC70E080E090E0CC
:108F60000E94917734CF6BE776E0CE0101960E94A4
:108F70008D74BE016F5F7F4FCE0188960E94D872BC
:108F8000182FCE0101960E94EE73111172CFBE010F
:108F9000685D7F4FCE0101960E94727470CF6DE9BB
:108FA00076E0CE0101960E948D74BE016F5F7F4F07
:108FB000CE018E960E94D872182FCE0101960E9483
:108FC000EE73112309F4EAC025E030E044E050E0FC
:108FD00060E27FE0CE0101960E94A274BE016F5F45
:108FE0007F4F8CEF9EE00E94B573CE0101960E94E8
:108FF000EE7360E27FE0CE0101960E948474CE01A0
:1090000001960E94CD1ACE0101960E94EE738CEF5C
:109010009EE00E943F726130710509F069C0709353
:10902000601060935F1065E977E0CE0101960E94C1
:109030007B74CE0101960E94CD1ACE0101960E944A
:10904000EE7362EA76E0CE014C960E948D746FEE6C
:1090500070E1CE014C960E940973BC01CE010196CD
:109060000E94847448EC50E06FEF7FEFCE010196D0
:109070000E942A20CE0101960E94EE73CE014C96EA
:109080000E94EE730E94659C40E052EC61E070E04B
:109090008FE99CE00E94EB6F84EF91E09093670270
:1090A0008093660263EA7FE00E949C0861EB76E0B1
:1090B000CE014C960E948D7469EE70E1CE014C9603
:1090C0000E940973BC01CE0101960E94847440ED98
:1090D00057E06FEF7FEFCE0101960E940109CE01AC
:1090E00001960E94EE73CE014C960E94EE73C7CAA1
:1090F00061157105D1F51092601010925F1067E84C
:1091000077E0CE0101960E947B74CE0101960E9409
:10911000CD1ACE0101960E94EE7368EA76E0CE0188
:109120004C960E948D746FEE70E1CE014C960E94B9
:109130000973BC01CE0101960E94847448EC50E092
:109140006FEF7FEFCE0101960E942A20CE0101969B
:109150000E94EE73CE014C960E94EE730E94659CB5
:1091600040E855E260E070E093CF6230710509F0AD
:1091700086CA7093601060935F1066E777E0CE0157
:1091800001960E947B74CE0101960E94CD1ACE01F9
:1091900001960E94EE736CEA76E0C1CF66EB76E052
:1091A000CE0101960E948D74BE016F5F7F4FCE018C
:1091B0008E960E94D872182FCE0101960E94EE73EF
:1091C000112309F441C047E050E060E27FE0CE01A6
:1091D00001960E949719BE016F5F7F4F8CEF9EE052
:1091E0000E94B573CE0101960E94EE7361E876E0AD
:1091F000CE0101960E948D74BE016F5F7F4F8CEF90
:109200009EE00E94D872182FCE0101960E94EE7344
:1092100011111092570C68ED74E0CE0101960E9476
:109220008D74BE016F5F7F4F8CEF9EE00E94D872FD
:10923000182FCE0101960E94EE73112309F4E9CC98
:1092400081E08093570CE5CC6EEB76E0CE01019681
:109250000E948D74BE016F5F7F4FCE018E960E947B
:10926000D872182FCE0101960E94EE73112381F15E
:1092700046E050E060E27FE0CE0101960E9497193F
:10928000BE016F5F7F4F8CEF9EE00E94B573CE01F1
:1092900001960E94EE738CEF9EE00E943472609300
:1092A000A7107093A8108093A9109093AA1084EF30
:1092B00091E0909367028093660263EA7FE00E94E8
:1092C0009C0864E670E080E090E00E949177A1CC79
:1092D00065EC76E0CE0101960E948D74BE016F5F51
:1092E0007F4FCE018E960E94D872182FCE01019624
:1092F0000E94EE73112301F148E050E060E27FE04C
:10930000CE0101960E949719BE016F5F7F4F8CEFCF
:109310009EE00E94B573CE0101960E94EE738CEF21
:109320009EE00E9434726093AD107093AE108093F3
:10933000AF109093B010BBCF6EEC76E0CE010196EB
:109340000E948D74BE016F5F7F4FCE018E960E948A
:10935000D872182FCE0101960E94EE73112301F1ED
:1093600049E050E060E27FE0CE0101960E9497194B
:10937000BE016F5F7F4F8CEF9EE00E94B573CE0100
:1093800001960E94EE738CEF9EE00E94347260930F
:10939000B1107093B2108093B3109093B41087CF34
:1093A00068ED76E0CE0101960E948D74BE016F5F7C
:1093B0007F4FCE018E960E94D872182FCE01019653
:1093C0000E94EE731123F1F049E050E060E27FE08B
:1093D000CE0101960E949719BE016F5F7F4F8CEFFF
:1093E0009EE00E94B573CE0101960E94EE738CEF51
:1093F0009EE00E9434720E94A6AA7093B8106093F7
:10940000B71055CF62EE76E0CE0101960E948D74C2
:10941000BE016F5F7F4FCE018E960E94D872182FCB
:10942000CE0101960E94EE731123F1F04AE050E064
:1094300060E27FE0CE0101960E949719BE016F5F46
:109440007F4F8CEF9EE00E94B573CE0101960E9483
:10945000EE738CEF9EE00E9434720E94A6AA709375
:10946000B6106093B51023CF6DEE76E0CE01019675
:109470000E948D74BE016F5F7F4FCE018E960E9459
:10948000D872182FCE0101960E94EE73112311F1AC
:109490004BE050E060E27FE0CE0101960E94971918
:1094A000BE016F5F7F4F8CEF9EE00E94B573CE01CF
:1094B00001960E94EE738CEF9EE00E9434720E942F
:1094C000A6AA6093B9107093BA108093BB109093C2
:1094D000BC10EDCE69EF76E0CE0101960E948D744E
:1094E000BE016F5F7F4FCE018E960E94D872182FFB
:1094F000CE0101960E94EE731123E1F045E050E0A9
:1095000060E27FE0CE0101960E949719BE016F5F75
:109510007F4F8CEF9EE00E94B573CE0101960E94B2
:10952000EE738CEF9EE00E943F727093AC106093DC
:10953000AB10BDCE6FEF76E0CE0101960E948D7428
:10954000BE016F5F7F4FCE018E960E94D872182F9A
:10955000CE0101960E94EE73112359F00E9470799A
:1095600060934A0C70934B0C80934C0C90934D0C71
:1095700086C865E077E0CE0101960E948D74BE0139
:109580006F5F7F4FCE018E960E94D872182FCE014A
:1095900001960E94EE73112389F143E050E0BE0171
:1095A000625D7F4FCE0101960E949719BE016F5FE9
:1095B0007F4F8CEF9EE00E94B573CE0101960E9412
:1095C000EE738091000F9091010F892B41F08CEF89
:1095D0009EE00E943F7270936F0260936E028091D2
:1095E0006E0290916F020197029708F412CB81E00E
:1095F00090E090936F0280936E020BCB66EE76E064
:10960000CE014C960E948D74BE01645E7F4FCE01E8
:109610008E960E94D87211E0811115C060E577E046
:10962000CE0101960E948D74BE016F5F7F4FCE0107
:109630008E960E94D87211E0811101C010E0CE0117
:1096400001960E94EE73CE014C960E94EE73112398
:1096500009F468C066EE76E0CE0101960E948D7432
:10966000BE016F5F7F4FCE018E960E94D872182F79
:10967000CE0101960E94EE731123A1F046E050E066
:10968000BE01625D7F4FCE0101960E949719BE0117
:109690006F5F7F4F8CEF9EE00E94B573CE01019605
:1096A0000E94EE7360E577E0CE0101960E948D7412
:1096B000BE016F5F7F4FCE018E960E94D872182F29
:1096C000CE0101960E94EE731123A1F042E050E01A
:1096D000BE01625D7F4FCE0101960E949719BE01C7
:1096E0006F5F7F4F8CEF9EE00E94B573CE010196B5
:1096F0000E94EE738091000F9091010F892B09F465
:1097000088CA6CEF7EE0CE0101960E94847461E00D
:1097100070E0CE0101960E94342FCE0101960E9486
:10972000EE7377CA62E177E0CE0182960E948D7473
:10973000BE016E5D7F4FCE018E960E94D87211E001
:10974000811129C069E077E0CE014C960E948D74AA
:10975000BE01645E7F4FCE018E960E94D87211E0EA
:10976000811115C061E177E0CE0101960E948D74F0
:10977000BE016F5F7F4FCE018E960E94D87211E0BE
:10978000811101C010E0CE0101960E94EE73CE015E
:109790004C960E94EE73CE0182960E94EE731123C6
:1097A00009F4E6C062E177E0CE0101960E948D7473
:1097B000BE016F5F7F4FCE018E960E94D872182F28
:1097C000CE0101960E94EE73112309F466C046E0B3
:1097D00050E0BE01625D7F4FCE0101960E94971955
:1097E000BE016F5F7F4F8CEF9EE00E94B573CE018C
:1097F00001960E94EE738CEF9EE00E9434726B0122
:109800007C0120E030E0A9010E94DCAA18160CF0CF
:109810008EC0A701960160E070E08AE794E40E94A0
:1098200034AA0E94A6AA6093390270933A028093E8
:109830003B0290933C028091390290913A02A091B0
:109840003B02B0913C02181619061A061B0664F07A
:1098500081E090E0A0E0B0E08093390290933A027A
:10986000A0933B02B0933C0280916E0290916F02F4
:109870008130910509F068C08091390290913A02D7
:10988000A0913B02B0913C02809335029093360246
:10989000A0933702B0933802BCC947E050E0BE0144
:1098A000625D7F4FCE0101960E949719BE016F5FE6
:1098B0007F4F8CEF9EE00E94B573CE0101960E940F
:1098C000EE7360E874E0CE0101960E948D74BE01D3
:1098D0006F5F7F4FCE018E960E94D872182FCE01F7
:1098E00001960E94EE73112331F081E090E0909395
:1098F0006F0280936E026FE176E0CE0101960E94C6
:109900008D74BE016F5F7F4FCE018E960E94D8721C
:10991000182FCE0101960E94EE73112309F46BCF2C
:1099200082E090E090936F0280936E0264CF81E0BA
:1099300090E0A0E0B0E08093390290933A02A093C7
:109940003B02B0933C0277CF029709F062C9809145
:10995000390290913A02A0913B02B0913C0280936F
:10996000310290933202A0933302B093340251C972
:1099700069E177E0CE014C960E948D74BE01645E71
:109980007F4FCE018E960E94B87211E0811115C0F2
:109990006EE177E0CE0101960E948D74BE016F5F8B
:1099A0007F4FCE018E960E94D87211E0811101C0C6
:1099B00010E0CE0101960E94EE73CE014C960E94FB
:1099C000EE73112309F48DC26BEA77E0CE010196A4
:1099D0000E948D74BE016F5F7F4FCE018E960E94F4
:1099E000D872182FCE0101960E94EE73112309F44C
:1099F000FBC001E010E010936F0200936E02109321
:109A00005D0200935C0265E277E08CEF9EE00E94CD
:109A1000D17110935D0200935C0281E090E0A0E0C0
:109A2000B0E08093390290933A02A0933B02B09346
:109A30003C028093350290933602A0933702B09394
:109A400038026CEF7EE0CE0101960E94847462E0E1
:109A500070E0CE0101960E94342FCE0101960E9443
:109A6000EE736DEA78E0CE0101960E947B74CE0120
:109A700001960E94E115CE0101960E94EE736DE9F8
:109A800078E0CE0101960E947B74CE0101960E947F
:109A9000FF20CE0101960E94EE7361E876E08CEF24
:109AA0009EE00E94D1716CEF7EE0CE0101960E9493
:109AB000847463E070E0CE0101960E94342FCE01E1
:109AC00001960E94EE7382E090E090936F02809383
:109AD0006E026CE878E0CE0101960E947B74CE01A4
:109AE00001960E94E115CE0101960E94EE7360E896
:109AF00078E0CE0101960E947B74CE0101960E940F
:109B0000FF20CE0101960E94EE7365E277E08CEFB4
:109B10009EE00E94D1718091C9109091CA1097FF68
:109B200006C069E277E08CEF9EE00E94D1716CEF95
:109B30007EE0CE0101960E94847462E070E0CE0166
:109B400001960E94342FCE0101960E94EE7361E8C7
:109B500076E08CEF9EE00E94D17182E090E09093DD
:109B60006F0280936E026CEF7EE0CE0101960E9440
:109B7000847463E070E0CE0101960E94342FCE0120
:109B800001960E94EE7384EF91E0909367028093B8
:109B9000660263EA7FE00E949C0864E670E080E071
:109BA00090E00E94917781E090E090936F02809323
:109BB0006E021092DA021092D90282E090E0A0E0E8
:109BC000B0E08093C3029093C402A093C502B09307
:109BD000C6020E9470796093E3027093E40280935E
:109BE000E5029093E60215C869E177E0CE0101969F
:109BF0000E948D74BE016F5F7F4FCE018E960E94D2
:109C0000D872182FCE0101960E94EE7311110C9498
:109C1000094660E874E0CE0101960E948D74BE0191
:109C20006F5F7F4FCE018E960E94D872182FCE01A3
:109C300001960E94EE73112331F081E090E0909341
:109C40006F0280936E026FE176E0CE0101960E9472
:109C50008D74BE016F5F7F4FCE018E960E94D872C9
:109C6000182FCE0101960E94EE73112331F082E08D
:109C700090E090936F0280936E0281E090E0A0E00C
:109C8000B0E08093390290933A02A0933B02B093E4
:109C90003C0280916E0290916F028130910509F033
:109CA00099C090935D0280935C026EE177E0CE01F3
:109CB00001960E948D74BE016F5F7F4FCE018E961C
:109CC0000E94D872182FCE0101960E94EE731123C4
:109CD00019F146E050E0BE01625D7F4FCE014C9627
:109CE0000E9497196DE277E0CE0101960E948D7473
:109CF000BE01645E7F4FCE0101960E940973BC01D4
:109D00008CEF9EE00E949E73CE0101960E94EE733E
:109D1000CE014C960E94EE738091390290913A02E6
:109D2000A0913B02B0913C028093350290933602A1
:109D3000A0933702B093380265E277E08CEF9EE0A3
:109D40000E94D1716CEF7EE0CE0101960E94847476
:109D500062E070E0CE0101960E94342FCE010196A0
:109D60000E94EE736FE678E0CE0101960E947B744C
:109D7000CE0101960E94E115CE0101960E94EE737C
:109D800081E090E090935D0280935C0261E876E070
:109D90008CEF9EE00E94D1716CEF7EE0CE010196C7
:109DA0000E94847463E070E0CE0101960E94342F1B
:109DB000CE0101960E94EE736FE578E0CE01019628
:109DC0000E947B74CE0101960E94FF20CE01019675
:109DD0000E94EE7380916E0290916F02029711F0D3
:109DE0000C94094665E277E08CEF9EE00E94D17109
:109DF0008091C9109091CA1097FF06C069E277E080
:109E00008CEF9EE00E94D17101E010E010935D02A2
:109E100000935C026CEF7EE0CE0101960E94847498
:109E200062E070E0CE0101960E94342FCE010196CF
:109E30000E94EE7361E876E08CEF9EE00E94D171A3
:109E40006EE478E0CE0101960E947B74CE0101960B
:109E50000E94E115CE0101960E94EE736CEF7EE048
:109E6000CE0101960E94847463E070E0CE010196F9
:109E70000E94342FCE0101960E94EE7362E478E0D6
:109E8000CE0101960E947B74CE0101960E94FF20B4
:109E9000CE0101960E94EE738091C9109091CA1074
:109EA0009195819591099093CA108093C910109350
:109EB0005D0200935C0284EF91E0909367028093CF
:109EC000660263EA7FE00E949C0864E670E080E03E
:109ED00090E00E94917710936F0200936E020C94B1
:109EE00009466FE277E0CE0188960E948D74BE012C
:109EF000685D7F4FCE018E960E94D87201E081117D
:109F00003DC060E877E0CE0182960E948D74BE016C
:109F10006E5D7F4FCE018E960E94D87201E0811156
:109F200029C06FE777E0CE014C960E948D74BE0188
:109F3000645E7F4FCE018E960E94D87201E081113F
:109F400015C066E377E0CE0101960E948D74BE01D4
:109F50006F5F7F4FCE018E960E94D87201E0811113
:109F600001C000E0CE0101960E94EE73CE014C9636
:109F70000E94EE73CE0182960E94EE73CE01889607
:109F80000E94EE73002309F41FC26FE277E0CE0156
:109F900001960E948D74BE016F5F7F4FCE018E9639
:109FA0000E94D872082FCE0101960E94EE7346E0FF
:109FB00050E0011117C060E877E0CE0101960E94E1
:109FC0008D74BE016F5F7F4FCE018E960E94D87256
:109FD000082FCE0101960E94EE73002309F48BC076
:109FE00042E050E0BE01625D7F4FCE0101960E94CB
:109FF0009719BE016F5F7F4F8CEF9EE00E94B57393
:10A00000CE0101960E94EE738091000F9091010F96
:10A01000892B11F40C9409466DE277E0CE014C9641
:10A020000E948D74BE01645E7F4F8CEF9EE00E94A3
:10A03000D872811114C06FE678E0CE0101960E94BB
:10A040008D74BE016F5F7F4F8CEF9EE00E94D872CF
:10A0500011E0811110E0CE0101960E94EE73CE0155
:10A060004C960E94EE73C12CD12C7601112309F479
:10A070006AC18CEF9EE00E9434726B017C0180917A
:10A080006E0290916F02019709F09FC08CEF9EE0E5
:10A090000E9434729B01AC016091E20B7091E30B62
:10A0A0008091E40B9091E50B0E94C8A96093E20BAC
:10A0B0007093E30B8093E40B9093E50B8090E20B9D
:10A0C0009090E30BA090E40BB090E50B20E030E023
:10A0D00044EB53E4C501B4010E94DCAA87FD86C0AD
:10A0E00020E030E044EB53E4C501B4010E94C7A96D
:10A0F0004B015C01EBCF43E050E0BE01625D7F4F5E
:10A10000CE0101960E949719BE016F5F7F4F8CEFC1
:10A110009EE00E94B573CE0101960E94EE7360E846
:10A1200074E0CE0101960E948D74BE016F5F7F4F77
:10A13000CE018E960E94D872082FCE0101960E9401
:10A14000EE730023B1F081E090E090936F02809372
:10A150006E028091380C9091390CA0913A0CB0911C
:10A160003B0C8093E20B9093E30BA093E40BB09332
:10A17000E50B6FE176E0CE0101960E948D74BE0181
:10A180006F5F7F4FCE018E960E94D872082FCE014E
:10A1900001960E94EE73002309F436CF82E090E02E
:10A1A00090936F0280936E028091340C9091350CE5
:10A1B000A091360CB091370C8093E20B9093E30B97
:10A1C000A093E40BB093E50B1FCF8CEF9EE00E94B1
:10A1D00034729B01AC016091E20B7091E30B8091B2
:10A1E000E40B9091E50B0E94C7A960CF20E030E01E
:10A1F000A901C501B4010E941AA887FF0BC020E085
:10A2000030E044EB53E4C501B4010E94C8A94B01FE
:10A210005C01ECCF8092E20B9092E30BA092E40BF6
:10A22000B092E50B20E030E0A901C701B6010E9421
:10A23000DCAA87FD15C06FE678E0CE0101960E948A
:10A240008D746CEF7EE0CE0101960E940973BC0113
:10A250008CEF9EE00E949E73CE0101960E94EE73E9
:10A2600020E030E0A901C701B6010E941AA887FFCB
:10A270006AC080916E0290916F02019799F520E07B
:10A2800030E0A901C701B6010E94DCAA18160CF043
:10A2900092C020E030E040E251E4C701B6010E94E4
:10A2A000C8A922E0AB01BC01CE014C960E94F67316
:10A2B0006DE277E0CE0101960E948D74BE01645E6E
:10A2C0007F4FCE0101960E940973BC018CEF9EE086
:10A2D0000E949E73CE0101960E94EE73CE014C96B1
:10A2E0000E94EE7380916E0290916F02019759F176
:10A2F00020E030E0A901C701B6010E94DCAAB70145
:10A30000A60118160CF0705822E0CE014C960E945F
:10A31000F6736DE277E0CE0101960E948D74BE0166
:10A32000645E7F4FCE0101960E940973BC018CEFE1
:10A330009EE00E949E73CE0101960E94EE73CE01B4
:10A340004C960E94EE7381E090E090935D028093C2
:10A350005C026CEF7EE0CE0101960E94847462E0A4
:10A3600070E0CE0101960E94342FCE0101960E942A
:10A37000EE7320E030E0A901C701B6010E941AA8DF
:10A3800087FD02C00C94094680916E0290916F0285
:10A39000019711F00C9409466AE377E08CEF9EE098
:10A3A0000E94D1716CEF7EE0CE0101960E94847410
:10A3B00062E070E0AEC9A701960160E070E080E263
:10A3C00091E40E94C7A96DCF6FE377E0CE0182963A
:10A3D0000E948D74BE016E5D7F4FCE018E960E94ED
:10A3E000D87211E0811129C06EE377E0CE014C965E
:10A3F0000E948D74BE01645E7F4FCE018E960E94D6
:10A40000D87211E0811115C065E477E0CE010196A4
:10A410000E948D74BE016F5F7F4FCE018E960E94A9
:10A42000D87211E0811101C010E0CE0101960E94A6
:10A43000EE73CE014C960E94EE73CE0182960E947E
:10A44000EE73112309F49BC0CE018E960E944A72CE
:10A4500065E277E08CEF9EE00E94D17160E874E0E5
:10A46000CE0101960E948D74BE016F5F7F4FCE01B9
:10A470008E960E94D872182FCE0101960E94EE731C
:10A48000112331F081E090E090936F0280936E028F
:10A490006FE176E0CE0101960E948D74BE016F5F80
:10A4A0007F4FCE018E960E94D872182FCE01019652
:10A4B0000E94EE73112391F082E090E090936F027E
:10A4C00080936E028091C9109091CA1097FF06C0C8
:10A4D00069E277E08CEF9EE00E94D17181E090E02C
:10A4E00090935D0280935C026CEF7EE0CE0101965A
:10A4F0000E94847462E070E0CE0101960E94342FC5
:10A50000CE0101960E94EE736FE377E0CE010196D3
:10A510000E948D74BE016F5F7F4FCE018E960E94A8
:10A52000D872182FCE0101960E94EE7345E050E0DC
:10A53000111102C046E050E0BE01625D7F4FCE01C6
:10A5400001960E949719BE016F5F7F4F8CEF9EE0CE
:10A550000E94B573CE0101960E94EE738091000FA8
:10A560009091010F892B11F40C9409466CEF7EE059
:10A57000CE0101960E94847463E070E0CAC86DE465
:10A5800077E0CE0182960E948D74BE016E5D7F4F92
:10A59000CE018E960E94D87211E0811129C06CE420
:10A5A00077E0CE014C960E948D74BE01645E7F4FB1
:10A5B000CE018E960E94D87211E0811115C063E51C
:10A5C00077E0CE0101960E948D74BE016F5F7F4FD0
:10A5D000CE018E960E94D87211E0811101C010E068
:10A5E000CE0101960E94EE73CE014C960E94EE734E
:10A5F000CE0182960E94EE73112309F426C16DE408
:10A6000077E0CE0101960E948D74BE016F5F7F4F8F
:10A61000CE018E960E94D872182FCE0101960E940C
:10A62000EE73112309F443C045E050E0BE01625DC2
:10A630007F4FCE0101960E949719BE016F5F7F4F39
:10A640008CEF9EE00E94B573CE0101960E94EE73DE
:10A650008091000F9091010F892B61F08CEF9EE0AB
:10A660000E9434726093E20B7093E30B8093E40BCF
:10A670009093E50BC090E20BD090E30BE090E40BDD
:10A68000F090E50B20E030E044EB53E4C701B60165
:10A690000E94DCAA87FD55C020E030E044EB53E483
:10A6A000C701B6010E94C7A96B017C01EBCF46E050
:10A6B00050E0BE01625D7F4FCE0101960E94971966
:10A6C000BE016F5F7F4F8CEF9EE00E94B573CE019D
:10A6D00001960E94EE7360E874E0CE0101960E943C
:10A6E0008D74BE016F5F7F4FCE018E960E94D8722F
:10A6F000182FCE0101960E94EE73112331F081E0F4
:10A7000090E090936F0280936E026FE176E0CE014D
:10A7100001960E948D74BE016F5F7F4FCE018E96B1
:10A720000E94D872182FCE0101960E94EE73112359
:10A7300009F48ECF82E090E090936F0280936E02D6
:10A7400087CF20E030E0A901C701B6010E941AA816
:10A7500087FF0BC020E030E044EB53E4C701B601B3
:10A760000E94C8A96B017C01ECCFC092E20BD09291
:10A77000E30BE092E40BF092E50B80916E02909176
:10A780006F02019771F4C092380CD092390CE092AC
:10A790003A0CF0923B0C61E175E082E09FE00E9490
:10A7A000D1718091E20B9091E30BA091E40BB091F9
:10A7B000E50B20916E0230916F022230310571F469
:10A7C0008093340C9093350CA093360CB093370CD7
:10A7D00061E275E082E09FE00E94D1714091E20B5E
:10A7E0005091E30B6091E40B7091E50B21E0CE01F9
:10A7F0004C960E94F67362E07FE0CE0101960E94C3
:10A800008474BE01645E7F4FCE0101960E9409737D
:10A810006CE175E00E94F372BC0182E09FE00E944F
:10A820009E73CE0101960E94EE73CE014C960E945B
:10A83000EE7362E07FE0CE0101960E948474CE0147
:10A8400001960E94FF200C948D4B6BE577E0CE01C2
:10A8500082960E948D74BE016E5D7F4FCE018E96F2
:10A860000E94D87211E0811129C06AE577E0CE011B
:10A870004C960E948D74BE01645E7F4FCE018E9611
:10A880000E94D87211E0811115C060E677E0CE0118
:10A8900001960E948D74BE016F5F7F4FCE018E9630
:10A8A0000E94D87211E0811101C010E0CE01019622
:10A8B0000E94EE73CE014C960E94EE73CE018296FA
:10A8C0000E94EE73112309F412C2C0903902D09095
:10A8D0003A02E0903B02F0903C0266E677E0CE015F
:10A8E00001960E948D74BE016F5F7F4FCE018E96E0
:10A8F0000E94D872182FCE0101960E94EE73112388
:10A9000009F465C044E050E0BE01625D7F4FCE01B6
:10A9100001960E949719BE016F5F7F4F8CEF9EE0FA
:10A920000E94B573CE0101960E94EE7380916E0273
:10A9300090916F028130910509F093C0C09035026B
:10A94000D0903602E0903702F090380281E090E03B
:10A95000A0E0B0E08093350290933602A0933702D6
:10A96000B09338028091000F9091010F892B09F06C
:10A9700090C06BE677E08CEF9EE00E94D1718091F1
:10A98000000F9091010F892B81F06CEF7EE0CE01DA
:10A9900001960E94847470E060E0CE0101960E94EE
:10A9A000342FCE0101960E94EE7380916E02909139
:10A9B0006F028130910509F08CC1C0923502D092AE
:10A9C0003602E0923702F09238020C94094645E0D4
:10A9D00050E0BE01625D7F4FCE0101960E94971943
:10A9E000BE016F5F7F4F8CEF9EE00E94B573CE017A
:10A9F00001960E94EE7360E874E0CE0101960E9419
:10AA00008D74BE016F5F7F4FCE018E960E94D8720B
:10AA1000182FCE0101960E94EE73112331F081E0D0
:10AA200090E090936F0280936E026FE176E0CE012A
:10AA300001960E948D74BE016F5F7F4FCE018E968E
:10AA40000E94D872182FCE0101960E94EE73112336
:10AA500009F46CCF82E090E090936F0280936E02D5
:10AA600065CF029709F07ECFC0903102D0903202BC
:10AA7000E0903302F090340281E090E0A0E0B0E09A
:10AA80008093310290933202A0933302B093340248
:10AA900069CF61E777E0CE0101960E948D74BE0117
:10AAA0006F5F7F4F8CEF9EE00E94B872182FCE012F
:10AAB00001960E94EE73112309F477CF8CEF9EE08C
:10AAC0000E94347220E030E0A9010E941AA881118E
:10AAD00028C080916E0290916F02019731F464E773
:10AAE00077E08CEF9EE00E94D17180916E02909190
:10AAF0006F02029731F46BE677E08CEF9EE00E94E4
:10AB0000D1718091000F9091010F892B09F44DCFE5
:10AB10006CEF7EE0CE0101960E94847461E070E0EB
:10AB20003CCF62EF75E0CE0101960E948D74BE01AC
:10AB30006F5F7F4F8CEF9EE00E94B872182FCE019E
:10AB400001960E94EE73112309F42FCF41E050E0EB
:10AB50006CEF7EE0CE0101960E949719CE0101961E
:10AB60000E9434724B015C01CE0101960E94EE738B
:10AB700020E030E0A901C501B4010E941AA818160E
:10AB800034F0812C912C90E8A92E9FE3B92E0091EE
:10AB90006E0210916F020130110509F075C0A50118
:10ABA000940160E070E48CE995E40E9434AA60931B
:10ABB0002D0270932E0280932F02909330026093A7
:10ABC000C1107093C2108093C3109093C41060930F
:10ABD000290270932A0280932B0290932C02B801D1
:10ABE000CE014C960E94DB7169E777E0CE010196B9
:10ABF0000E948D74BE01645E7F4FCE0101960E945B
:10AC00000973BC01CE0182960E948474CE018296A3
:10AC10000E94F815CE0182960E94EE73CE01019635
:10AC20000E94EE73CE014C960E94EE7360E378E0D2
:10AC3000CE0101960E947B74CE0101960E94F81508
:10AC4000CE0101960E94EE7340912D0250912E028A
:10AC500060912F027091300225E0CE0101960E9492
:10AC6000F673CE0101960E94E115CE0101960E9475
:10AC7000EE7384EF91E0909367028093660263EA3B
:10AC80007FE00E949C0891CE0230110509F0A7CF09
:10AC9000A501940160E070E48CE196E40E9434AA7E
:10ACA00060932D0270932E0280932F0290933002B6
:10ACB0006093C5107093C6108093C7109093C8100E
:10ACC00060932502709326028093270290932802B6
:10ACD00086CF029711F00C940946C0923102D092AF
:10ACE0003202E0923302F09234020C9409466EE78D
:10ACF00077E0CE0182960E948D74BE016E5D7F4F1B
:10AD0000CE018E960E94D87211E0811129C06DE7A4
:10AD100077E0CE014C960E948D74BE01645E7F4F39
:10AD2000CE018E960E94D87211E0811115C063E8A1
:10AD300077E0CE0101960E948D74BE016F5F7F4F58
:10AD4000CE018E960E94D87211E0811101C010E0F0
:10AD5000CE0101960E94EE73CE014C960E94EE73D6
:10AD6000CE0182960E94EE73112309F429C18AA9AB
:10AD70009BA9059710F40C94094644E050E0BE01ED
:10AD8000625D7F4FCE0101960E949719BE016F5FF1
:10AD90007F4F8CEF9EE00E94B573CE0101960E941A
:10ADA000EE736EE777E0CE0101960E948D74BE01CE
:10ADB0006F5F7F4FCE018E960E94D872182FCE0102
:10ADC00001960E94EE73112309F49BC044E050E009
:10ADD000BE01625D7F4FCE0101960E949719BE01B0
:10ADE0006F5F7F4F8CEF9EE00E94B573CE0101969E
:10ADF0000E94EE738CEF9EE00E94347220E030E0FF
:10AE0000A9010E94DCAA181614F00C9409468CEFD4
:10AE10009EE00E94347260932D0270932E02809304
:10AE20002F029093300220916E0230916F022130F8
:10AE3000310509F0B0C06093C1107093C2108093C7
:10AE4000C3109093C4106093290270932A028093D8
:10AE50002B0290932C02B901CE014C960E94DB711B
:10AE600069E777E0CE0101960E948D74BE01645EB1
:10AE70007F4FCE0101960E940973BC01CE018296DC
:10AE80000E948474CE0182960E94F815CE018296AB
:10AE90000E94EE73CE0101960E94EE73CE014C9695
:10AEA0000E94EE736EE178E0CE0101960E947B7401
:10AEB000CE0101960E94F815CE0101960E94EE7314
:10AEC00040912D0250912E0260912F02709130021C
:10AED00025E0CE0101960E94F673CE0101960E94F4
:10AEE000E115CE0101960E94EE7384EF91E09093FC
:10AEF00067028093660263EA7FE00E949C080C94DC
:10AF0000094645E050E0BE01625D7F4FCE010196EB
:10AF10000E949719BE016F5F7F4F8CEF9EE00E94E9
:10AF2000B573CE0101960E94EE7360E874E0CE0125
:10AF300001960E948D74BE016F5F7F4FCE018E9689
:10AF40000E94D872182FCE0101960E94EE73112331
:10AF500031F081E090E090936F0280936E026FE198
:10AF600076E0CE0101960E948D74BE016F5F7F4F27
:10AF7000CE018E960E94D872182FCE0101960E94A3
:10AF8000EE73112309F436CF82E090E090936F02C4
:10AF900080936E022FCF2230310509F05CCF609391
:10AFA000C5107093C6108093C7109093C81060931B
:10AFB00025027093260280932702909328024BCF9C
:10AFC00064E875E0CE014C960E948D74BE01645E0B
:10AFD0007F4FCE018E960E94D87211E0811115C06C
:10AFE00069E877E0CE0101960E948D74BE016F5F23
:10AFF0007F4FCE018E960E94D87211E0811101C060
:10B0000010E0CE0101960E94EE73CE014C960E9494
:10B01000EE73112309F463C064E875E0CE01019674
:10B020000E948D74BE016F5F7F4FCE018E960E948D
:10B03000D872182FCE0101960E94EE73112399F059
:10B0400042E050E060E27FE0CE0101960E94971955
:10B05000BE016F5F7F4F8CEF9EE00E94B573CE0103
:10B0600001960E94EE7369E877E0CE0101960E9496
:10B070008D74BE016F5F7F4FCE018E960E94D87295
:10B08000182FCE0101960E94EE73112399F043E030
:10B0900050E060E27FE0CE0101960E949719BE0168
:10B0A0006F5F7F4F8CEF9EE00E94B573CE010196DB
:10B0B0000E94EE738CEF9EE00E943F72653B71052B
:10B0C00010F40C9409466BE078E0CE0101960E94E2
:10B0D0007B74CE0101960E94F8150C948D4B6DE89F
:10B0E00077E0CE0101960E948D74BE016F5F7F4FA5
:10B0F000CE018E960E94D872182FCE0101960E9422
:10B10000EE73112309F470C026E030E044E050E013
:10B1100060E27FE0CE0101960E94A274BE016F5FE3
:10B120007F4F8CEF9EE00E94B573CE0101960E9486
:10B13000EE7362EF75E0CE0101960E948D7440912E
:10B14000240F5091250F8D819E81481B590BBE0104
:10B150006F5F7F4F80E29FE00E94AC9CAC014F5F2D
:10B160005F4F60E27FE0CE014C960E949719BE01CE
:10B17000645E7F4F8CEF9EE00E94B573CE014C96CB
:10B180000E94EE73CE0101960E94EE738CEF9EE05A
:10B190000E94347288E2EAEBFBE0AAE7B0E101909A
:10B1A0000D928A95E1F784EF91E090936702809386
:10B1B000660263EA7FE00E949C086AEE77E082E024
:10B1C0009FE00E94797344E050E060E27FE0CE01AE
:10B1D00001960E949719BE016F5F7F4F82E09FE04A
:10B1E0000E9472730C94244361E977E0CE010196CA
:10B1F0000E948D74BE016F5F7F4FCE018E960E94BC
:10B20000D872182FCE0101960E94EE7311110C9482
:10B21000E34869E977E0CE0101960E948D74BE0192
:10B220006F5F7F4FCE018E960E94D872182FCE018D
:10B2300001960E94EE73112371F141E068E972E01A
:10B24000CE0101960E94438BBE016F5F7F4F87E066
:10B2500091E10E94081987E091E10E94F08A811132
:10B2600004C06EE977E00C94A24187E091E10E946E
:10B27000FC6E892B51F087E091E10E945086682F87
:10B280008CE39DE00E94256DF0CF87E091E10E9464
:10B29000FC8A0C94C83860EA77E0CE0101960E94DF
:10B2A0008D74BE016F5F7F4FCE018E960E94D87263
:10B2B000182FCE0101960E94EE731123E9F08DB78D
:10B2C0009EB7825391400FB6F8949EBF0FBE8DBFBC
:10B2D000ADB7BEB7119682E391E0E3EAFFE00190DB
:10B2E0000D920197E1F70E94022B0FB6F894DEBF92
:10B2F0000FBECDBF0C94C83869EA77E0CE01019645
:10B300000E948D74BE016F5F7F4FCE018E960E94AA
:10B31000D872182FCE0101960E94EE73112309F402
:10B3200057C0EDB7FEB7E253F1400FB6F894FEBF39
:10B330000FBEEDBFADB7BEB7119682E391E0E3EA71
:10B34000FFE001900D920197E1F70E9481240FB672
:10B35000F894DEBF0FBECDBF69ED77E0CE01019658
:10B360000E947B74ADB7BEB7A253B1400FB6F8943C
:10B37000BEBF0FBEADBF119682E391E0E3EAFFE0EE
:10B3800001900D920197E1F70E94B11D0FB6F8945C
:10B39000DEBF0FBECDBF8DB79EB7825391400FB6B3
:10B3A000F8949EBF0FBE8DBFADB7BEB7119682E3B6
:10B3B00091E0E3EAFFE001900D920197E1F70E942E
:10B3C000022B0FB6F894DEBF0FBECDBF0C94CD3D5F
:10B3D0006BEA77E0CE0101960E948D74BE016F5F2B
:10B3E0007F4FCE018E960E94D872182FCE01019603
:10B3F0000E94EE731123F9F067EC77E0CE0101961D
:10B400000E947B74BE016F5F7F4FCE014C960E94FD
:10B410008474CE014C960E94E115CE014C960E9498
:10B42000EE73EDB7FEB7E253F1400FB6F894FEBFEE
:10B430000FBEEDBFB9CF6FEA77E0CE0101960E9453
:10B440008D74BE016F5F7F4FCE018E960E94D872C1
:10B45000182FCE0101960E94EE73112309F4F5C056
:10B460006BEA77E0CE0182960E947B74BE016E5D2E
:10B470007F4FCE0101960E948474AE014F5F5F4FF3
:10B4800062E070E081E892E00E943426182FCE013D
:10B4900001960E94EE73111122C0BE016E5D7F4FB6
:10B4A000CE014C960E94847463EB77E0CE014C96FB
:10B4B0000E94F37263E57FE00E940973BC01CE0134
:10B4C00001960E948474CE0101960E94E115CE017E
:10B4D00001960E94EE73CE014C960E94EE7368EEC8
:10B4E00073E080E090E00E949177BE016E5D7F4F37
:10B4F000CE0101960E948474AE014F5F5F4F63E0FE
:10B5000070E084E792E00E943426182FCE01019665
:10B510000E94EE73111122C0BE016E5D7F4FCE01FD
:10B520004C960E94847463EC77E0CE014C960E94A6
:10B53000F37263E57FE00E940973BC01CE010196BE
:10B540000E948474CE0101960E94E115CE010196FD
:10B550000E94EE73CE014C960E94EE7368EE73E08B
:10B5600080E090E00E94917767E47FE0CE01019651
:10B570000E948474AE014F5F5F4F61E070E082EB28
:10B5800092E00E943426182FCE0101960E94EE739D
:10B59000111121C067E47FE0CE014C960E948474B3
:10B5A00063EC77E0CE014C960E94F37263E57FE096
:10B5B0000E940973BC01CE0101960E948474CE01E1
:10B5C00001960E94E115CE0101960E94EE73CE0114
:10B5D0004C960E94EE7368EE73E080E090E00E946B
:10B5E00091778091570C882311F40C94FC4443E12B
:10B5F00062EB72E0CE0101960E94438BBE016F5F49
:10B600007F4F8DE391E10E9408198DE391E10E9443
:10B61000F08A882311F40C94FC4467E47FE08DE306
:10B6200091E10E94D47566E970E080E090E00E94AC
:10B6300091778DE391E10E94FC8A62E370E080E003
:10B6400090E00E9491770C94FC446FEC77E0CE017F
:10B6500001960E948D74BE016F5F7F4FCE018E9662
:10B660000E94D872182FCE0101960E94EE7311230A
:10B67000A9F008EF1BE0D8018C910E5F1F4F60E02E
:10B680000E94D8766CE271E080E090E00E949177B1
:10B69000BBE00E3F1B0779F70C94C83863ED77E0E9
:10B6A000CE0101960E948D74BE016F5F7F4FCE0167
:10B6B0008E960E94D872182FCE0101960E94EE73CA
:10B6C0001123C1F008EF1BE08EEFE82E8BE0F82E7F
:10B6D000F80180810E5F1F4F61E00E94D8766CE216
:10B6E00071E080E090E00E949177E016F10681F72A
:10B6F0000C94C83868ED77E0CE0101960E948D74F5
:10B70000BE016F5F7F4FCE018E960E94D872182FB8
:10B71000CE0101960E94EE73112311F40C94C838E7
:10B7200027E030E046E050E060E27FE0CE010196A5
:10B730000E94A274BE016F5F7F4F8CEF9EE00E945B
:10B74000B573CE0101960E94EE738CEF9EE00E94CD
:10B750003F72672B71F41092B90B60E27FE0CE016B
:10B7600001960E948474CE0101960E94CD1A0C9419
:10B77000954781E08093B90BF0CF2F923F924F9283
:10B780005F926F927F928F929F92AF92BF92CF9271
:10B79000DF92EF92FF920F931F93CF93DF9300D02E
:10B7A00000D01F921F92CDB7DEB7609190027091CA
:10B7B000910280918E0290918F020E940F1684E177
:10B7C000482E512C612C712C312C212C8FEF281AF2
:10B7D000380AC301B2010E94917760919002709182
:10B7E000910280918E0290918F020E940F168C011F
:10B7F00083E02816310434F08EE12816310444F435
:10B80000012B51F084E1480E511C611C711CDECFEC
:10B810000115110509F0A6C080918E0290918F024A
:10B820008B30910509F086C08090D9109090DA1085
:10B83000A090DB10B090DC10C090D510D090D61046
:10B84000E090D710F090D81064E670E080E090E0CF
:10B850000E9491776DE075E0CE0101960E947B74A5
:10B86000CE0101960E94FF20CE0101960E94EE7348
:10B8700061E082E00E94347D21E0B501A401CE01A7
:10B8800001960E94F673BE016F5F7F4F89E591E1DB
:10B890000E94C675CE0101960E94EE736FED89E598
:10B8A00091E10E940C7D68E075E089E591E10E94DC
:10B8B000E87520E0B701A601CE0101960E94F6735B
:10B8C000BE016F5F7F4F89E591E10E94C675CE0191
:10B8D00001960E94EE736FED77E089E591E10E9499
:10B8E000BE7589829A82AB82BC82CD82DE82EF8273
:10B8F000F88629813A814B815C816D817E818F81BF
:10B90000988528960FB6F894DEBF0FBECDBFDF91A5
:10B91000CF911F910F91FF90EF90DF90CF90BF904C
:10B92000AF909F908F907F906F905F904F903F90DF
:10B930002F9008958631910509F476CF0C9709F080
:10B9400083CF8090DE0A9090DF0AA090E00AB0904A
:10B95000E10AC090DA0AD090DB0AE090DC0AF090AD
:10B96000DD0A72CF0F3F8FEF1807CCF06AEF74E05B
:10B97000CE0101960E947B744AE050E070E060E0E6
:10B98000CE0101960E942A20CE0101960E94EE73FC
:10B9900067ED74E082E09FE00E94797332C00E3F51
:10B9A0008FEF1807B9F169EC74E0CE0101960E949F
:10B9B0007B744AE050E070E060E0CE0101960E94A6
:10B9C0002A20CE0101960E94EE736AEB74E082E0B9
:10B9D0009FE00E947973B801CE0101960E94DB714D
:10B9E000BE016F5F7F4F82E09FE00E947273CE01C5
:10B9F00001960E94EE7364EA74E082E09FE00E9488
:10BA00001C7319821A821B821C821D821E821F8255
:10BA100018866FCF69E974E0CE0101960E947B74AD
:10BA20004AE050E070E060E0CE0101960E942A20DA
:10BA3000CE0101960E94EE7369E774E0ABCF2F92BE
:10BA40003F924F925F926F927F928F929F92AF92AE
:10BA5000BF92CF92DF92EF92FF920F931F93CF93FB
:10BA6000DF93CDB7DEB7AC970FB6F894DEBF0FBE4D
:10BA7000CDBF8C017B018091320C9091330C0196EB
:10BA80009093330C8093320C20914F0C222341F081
:10BA90006AE070E00E94E6AA181619060CF4C0C20B
:10BAA00081E080934F0C1092330C1092320C50E0D6
:10BAB00040E060E274E0C8010E94521982E0E8169A
:10BAC000F10409F4C6C263EC78E081E49FE00E94CF
:10BAD000D171609190027091910280918E0290914B
:10BAE0008F020E940F161C0160EF7AE0C8010E94CD
:10BAF000391961EE77E0C8010E94BE7563EE70E10E
:10BB0000CE0101960E948474BE016F5F7F4FC80111
:10BB10000E94C675CE0101960E94EE736AEE77E030
:10BB2000C8010E94BE756DEF75E0C8010E94E875FE
:10BB300069EE70E1CE0101960E948474BE016F5FD0
:10BB40007F4FC8010E94C67563EF75E0C8010E946F
:10BB5000E8756BEF7FE0CE0109960E948D74BE01FF
:10BB6000675F7F4FC8010E94C67566EE75E0C80129
:10BB70000E94E87563E670E1CE010F960E948D7415
:10BB8000BE01615F7F4FC8010E94C6756FED75E011
:10BB9000C8010E94E875CE010F960E94EE73CE0197
:10BBA00009960E94EE73CE0101960E94EE730E94E8
:10BBB0004F7828EE33E040E050E00E9464A929016C
:10BBC0003A0165ED75E0C8010E94E875CE01019665
:10BBD0000E947A1BBE016F5F7F4FC8010E94C6752D
:10BBE000CE0101960E94EE73C301B20120E13EE056
:10BBF00040E050E00E9486A94B015C01B901CE01F2
:10BC000087960E94A3194CE3C42ED12CE12CF12C71
:10BC1000C501B401A70196010E9486A9B901CE0110
:10BC200001960E94A3196FEA76E0CE0109960E9460
:10BC30008D74BE016F5F7F4FCE0109960E9409731C
:10BC4000BC01CE0187960E947273CE0109960E94B4
:10BC5000EE73CE0101960E94EE73C301B201A701FB
:10BC600096010E9486A9CE0101960E94A3196FEA4F
:10BC700076E0CE0109960E948D74BE016F5F7F4F02
:10BC8000CE0109960E940973BC01CE0187960E94DD
:10BC90007273CE0109960E94EE73CE0101960E9446
:10BCA000EE7360EF77E0CE0109960E948D74BE01BD
:10BCB000695D7F4FCE0109960E94097363EF77E0BB
:10BCC0000E94F372BC01CE0101960E948474BE01F1
:10BCD0006F5F7F4FC8010E94C675CE0101960E941A
:10BCE000EE73CE0109960E94EE7361E078E0C80120
:10BCF0000E94BE75CE0101960E940771B801CE0167
:10BD000001960E9460756CEF77E0C8010E94AA75E9
:10BD10000E94BD5B29833A834B835C836D837E8362
:10BD20008F83988749815A816B817C8121E0CE0184
:10BD30000F960E94F673BE01615F7F4FCE01099698
:10BD40000E94847469E078E0CE0109960E94F37243
:10BD5000BC0181E49FE00E949E73CE0109960E947F
:10BD6000EE73CE010F960E94EE7360E178E0CE0193
:10BD70000F960E948D7461E47FE0CE010F960E94C1
:10BD80000973BC01CE0109960E948474BE01675FED
:10BD90007F4FC8010E94C675CE0109960E94EE73BE
:10BDA000CE010F960E94EE734D815E816F81788582
:10BDB00021E0CE0109960E94F673BE01675F7F4FB6
:10BDC00081E49FE00E94B573CE0109960E94EE7354
:10BDD00062E278E0CE010F960E948D7461E47FE00C
:10BDE000CE010F960E94097363E378E00E94F3721C
:10BDF000BC01CE0109960E948474BE01675F7F4F2B
:10BE0000C8010E94C675CE0109960E94EE73CE014C
:10BE10000F960E94EE734091380C5091390C60914E
:10BE20003A0C70913B0C22E0CE010F960E94F67303
:10BE30006AE378E0CE0145960E948D74BE01615F91
:10BE40007F4FCE0145960E9409736CE478E00E9412
:10BE5000F372BC01CE0109960E948474BE01675F33
:10BE60007F4FC8010E94C675CE0109960E94EE73ED
:10BE7000CE0145960E94EE73CE010F960E94EE739E
:10BE80004091340C5091350C6091360C7091370C08
:10BE900022E0CE010F960E94F67365E578E0CE01B0
:10BEA00045960E948D74BE01615F7F4FCE0145961D
:10BEB0000E9409736CE478E00E94F372BC01CE0129
:10BEC00009960E948474BE01675F7F4FC8010E947B
:10BED000C675CE0109960E94EE73CE0145960E946A
:10BEE000EE73CE010F960E94EE73E6EF2E16EFEF83
:10BEF0003E062CF46BEE7BE0C8010E94391968EC19
:10BF00007AE0C8010E94391993EAE92E9FE0F92EE0
:10BF100027EDA22E22E0B22ECC24C394D12C4701CF
:10BF2000F8E08F0E911C82E0A80EB11C8091A30F47
:10BF30009091A40F8C159D050CF464C0B601CE0140
:10BF40000F960E94DB716BE777E0CE0145960E9469
:10BF50008D74BE01615F7F4FCE0145960E940973CB
:10BF60006FEE75E00E94F372BC01CE0109960E944B
:10BF70008474BE01675F7F4FC8010E94C675B70118
:10BF8000645E7F4FCE014B960E948D74BE01655E4C
:10BF90007F4FC8010E94C67563E678E0C8010E9421
:10BFA000BE75F50160817181660F771F660F771F7F
:10BFB0006155704FCE0181960E948D74BE016F5DF8
:10BFC0007F4FC8010E94C67568E678E0C8010E94EC
:10BFD000BE75CE0181960E94EE73CE014B960E94F3
:10BFE000EE73CE0109960E94EE73CE0145960E9433
:10BFF000EE73CE010F960E94EE73FFEFCF1ADF0AA9
:10C0000074018DCFCE0187960E94EE7381E08093FC
:10C010005A0C69EA7BE0C8010E94391910924F0C52
:10C02000AC960FB6F894DEBF0FBECDBFDF91CF91B7
:10C030001F910F91FF90EF90DF90CF90BF90AF9046
:10C040009F908F907F906F905F904F903F902F9038
:10C0500008956BEE7BE0C8010E943919DACF8F9208
:10C060009F92AF92BF92CF92DF92EF92FF920F9387
:10C070001F93CF93DF93CDB7DEB7A0970FB6F89499
:10C08000DEBF0FBECDBF63EC78E08BE69FE00E9481
:10C09000D17163EC78E08FE59FE00E94D17148E4B4
:10C0A000842E42E0942E53EAA52E5FE0B52E6FEC6D
:10C0B000E62E62E0F62E77EDC72E72E0D72E01E075
:10C0C00010E0F40181919191A191B1914F01892BDF
:10C0D0008A2B8B2B19F5F60182819381F70122813E
:10C0E000338182179307D1F0880F991FFC01EB541D
:10C0F000F44FD801AA0FBB1FAA50B44F60818C9196
:10C100000E94D876F60182819381F701938382831E
:10C1100064E670E080E090E00E949177F701628130
:10C1200073818091A30F9091A40F801791070CF455
:10C13000E5C2CE0145960E94DB71B801CE010F9693
:10C140000E94DB71B501645E7F4FCE0109960E94AB
:10C150008D746FEE75E0CE0101960E948D74BE0164
:10C16000675F7F4FCE0101960E9409736EE678E00B
:10C170000E94F372BE01615F7F4F0E94097362EFFC
:10C1800075E00E94F372BE016B5E7F4F0E940973DF
:10C19000BC018BE69FE00E947273CE0101960E9463
:10C1A000EE73CE0109960E94EE73CE010F960E94A7
:10C1B000EE73CE0145960E94EE730F5F1F4FF8E0BD
:10C1C000AF0EB11C22E0E20EF11C82E0C80ED11CC1
:10C1D0000430110509F075CFE091BD10F091BE104B
:10C1E000EE0FFF1FE153FD4F60817181CE0101967B
:10C1F0000E94DB7146E050E0BE016F5F7F4FCE01D1
:10C2000009960E941F1CBE01675F7F4F8FE59FE06C
:10C210000E947273CE0109960E94EE73CE010196C0
:10C220000E94EE73E091BF10F091C010EE0FFF1F5F
:10C23000E153FD4F60817181CE0101960E94DB7157
:10C2400046E050E0BE016F5F7F4FCE0109960E942D
:10C250001F1CBE01675F7F4F8FE59FE00E947273D6
:10C26000CE0109960E94EE73CE0101960E94EE73F4
:10C270006FEE75E0CE0145960E948D740E944F7856
:10C2800028EE33E040E050E00E9464A969017A01A1
:10C2900063EC78E0CE014B960E948D7463EC78E0FD
:10C2A00081E79FE00E94D171CE0101960E947A1B26
:10C2B00044E150E0BE016F5F7F4FCE0109960E94BE
:10C2C0001F1CBE01675F7F4F81E79FE00E94B5732F
:10C2D000CE0109960E94EE73CE0101960E94EE7384
:10C2E0002AE0B701A601CE0109960E942C7448E00D
:10C2F00050E0BE01675F7F4FCE010F960E941F1C6A
:10C3000061E77FE0CE0101960E948474BE01615F07
:10C310007F4FCE0101960E940973BC0185E69FE024
:10C320000E949E73CE0101960E94EE73CE010F967D
:10C330000E94EE73CE0109960E94EE732AE0B701C7
:10C34000A601CE0109960E942C7461E778E0CE0127
:10C3500001960E948D74BE01675F7F4FCE010196EA
:10C360000E940973BE016B5E7F4F0E940973BC017E
:10C3700081E79FE00E947273CE0101960E94EE73E6
:10C38000CE0109960E94EE734091380C5091390C01
:10C3900060913A0C70913B0C21E0CE0101960E9415
:10C3A000F673BE016F5F7F4FCE014B960E94B5734F
:10C3B000CE0101960E94EE7368E778E0CE01019607
:10C3C0000E948D74BE01655E7F4FCE0101960E9472
:10C3D0000973BE016B5E7F4F0E940973BC0181E748
:10C3E0009FE00E947273CE0101960E94EE73BE011F
:10C3F000655E7F4FCE0101960E94847446E050E056
:10C40000BE016F5F7F4FCE0109960E941F1CBE01C7
:10C41000675F7F4F85E69FE00E947273CE010996A9
:10C420000E94EE73CE0101960E94EE734091340C8F
:10C430005091350C6091360C7091370C21E0CE0193
:10C4400001960E94F673BE016F5F7F4FCE014B963F
:10C450000E94B573CE0101960E94EE7366E878E003
:10C46000CE0101960E948D74BE01655E7F4FCE01A4
:10C4700001960E940973BE016B5E7F4F0E94097393
:10C48000BC0181E79FE00E947273CE0101960E9479
:10C49000EE73BE01655E7F4FCE0101960E948474EB
:10C4A00046E050E0BE016F5F7F4FCE0109960E94CB
:10C4B0001F1CBE01675F7F4F85E69FE00E9472737D
:10C4C000CE0109960E94EE73CE0101960E94EE7392
:10C4D000609190027091910280918E0290918F02F2
:10C4E0000E940F169093450C8093440C892B71F099
:10C4F000609190027091910280918E0290918F02D2
:10C500000E940F169093450C8093440C8091440C2C
:10C510009091450C8C3F9F4F0CF410C10E94BD5B65
:10C5200029833A834B835C836D837E838F839887D3
:10C5300049815A816B817C8121E0CE0109960E945C
:10C54000F673BE01675F7F4FCE014B960E94B573B5
:10C55000CE0109960E94EE7360E978E0CE0109965B
:10C560000E948D74BE01655E7F4FCE0109960E94C8
:10C570000973BE016B5E7F4F0E940973BC0181E7A6
:10C580009FE00E947273CE0109960E94EE73BE0175
:10C59000655E7F4FCE0109960E94847446E050E0AC
:10C5A000BE01675F7F4FCE010F960E941F1CBE0128
:10C5B000615F7F4F85E69FE00E947273CE010F9608
:10C5C0000E94EE73CE0109960E94EE734D815E814A
:10C5D0006F81788521E0CE0109960E94F673BE0135
:10C5E000675F7F4FCE014B960E94B573CE010996CF
:10C5F0000E94EE736BE978E0CE0109960E948D747B
:10C60000BE01655E7F4FCE0109960E940973BE018F
:10C610006B5E7F4F0E940973BC0181E79FE00E941F
:10C620007273CE0109960E94EE73BE01655E7F4F64
:10C63000CE0109960E94847446E050E0BE01675F17
:10C640007F4FCE010F960E941F1CBE01615F7F4F7E
:10C6500085E69FE00E947273CE010F960E94EE73F2
:10C66000CE0109960E94EE736BE67FE081E79FE0C2
:10C670000E9472736FEE75E0CE0101960E948D7478
:10C680006FE57FE0CE0101960E940973BC0185E64B
:10C690009FE00E947273CE0101960E94EE7365E6E0
:10C6A0007FE0CE0101960E948474CE0101960E9423
:10C6B000E115CE0101960E94EE736AE070E080E021
:10C6C00090E00E949177CE014B960E94EE73CE01CE
:10C6D00045960E94EE73A0960FB6F894DEBF0FBE8B
:10C6E000CDBFDF91CF911F910F91FF90EF90DF9021
:10C6F000CF90BF90AF909F908F900895CE014596B8
:10C700000E94DB71B801CE010F960E94DB71B5016A
:10C710006C5E7F4FCE0109960E948D746FEE75E0BE
:10C72000CE0101960E948D74BE01675F7F4FCE01DE
:10C7300001960E9409736DE678E01ACD61EA78E00F
:10C7400081E79FE00E94687360EB78E085E69FE0F8
:10C750000E94687367EB78E081E79FE00E9468734E
:10C7600060EB78E085E69FE00E9468737DCFBF9222
:10C77000CF92DF92EF92FF920F931F93CF93DF93AD
:10C78000CDB7DEB7C455D1090FB6F894DEBF0FBEE2
:10C79000CDBF6C018B0165965FAF4EAF6597809101
:10C7A000320C9091330C01969093330C8093320CA1
:10C7B00080914F0C81113CC0BB24B394B0924F0CBC
:10C7C0001092330C1092320C63EC78E0CE01895B4E
:10C7D0009F4F0E948D7463EC78E0CE01835B9F4F86
:10C7E0000E948D7450E040E060E274E0C6010E9457
:10C7F00052190130110509F0A6C063EC78E081E719
:10C800009FE00E94D1716596EEADFFAD6597808186
:10C81000811124C00E942F60B0925A0CCE01835B1C
:10C820009F4F0E94EE73CE01895B9F4F0E94EE7373
:10C830000FB6F894DEBF0FBECDBFCC5ADF4F0FB698
:10C84000F894DEBF0FBECDBFDF91CF911F910F9146
:10C85000FF90EF90DF90CF90BF9008956596EEAD7A
:10C86000FFAD65978081882309F467C000E210E07E
:10C870009E012F5F3F4F40E250E0BE016F5D7F4F52
:10C88000CE018D5A9F4F0E942F70049739F3BE013D
:10C890006F5D7F4FCE018F5B9F4F0E948D74BE01F5
:10C8A0006F5B7F4FCE01895B9F4F0E94B573CE01B6
:10C8B0008F5B9F4F0E94EE73BE016F5F7F4FCE0173
:10C8C0008F5B9F4F0E948D74BE016F5B7F4FCE01C7
:10C8D000835B9F4F0E94B573CE018F5B9F4F0E9479
:10C8E000EE73BE01695B7F4F81E79FE00E94727328
:10C8F00063968EAD9FAD6397892B09F4AFCF62EF3E
:10C9000075E0CE018F5B9F4F0E948D74BE01635B0B
:10C910007F4FCE018F5B9F4F0E9409736FEE75E0D2
:10C920000E94F372BC0181E79FE00E947273CE0106
:10C930008F5B9F4F0E94EE7391CF61E77FE08DE4A4
:10C940009FE00E949E7310924F0C68CF2F923F92EF
:10C950004F925F926F927F928F929F92AF92BF920F
:10C96000CF92DF92EF92FF920F931F93CF93DF93BB
:10C97000CDB7DEB7C258D1090FB6F894DEBF0FBEEF
:10C98000CDBF6C015B0188EE482E83E0582E612CF0
:10C99000712C09EF13E09BE5892E912C8C0E9D1EC6
:10C9A0008CE0880E911C1B019FEF291A390AD601D1
:10C9B0005996ED90FC90F7018581823008F493C080
:10C9C00082859385A485B5858F719927AA27BB2772
:10C9D000892B8A2B8B2B09F086C040E250E0BE01E8
:10C9E0006F5F7F4FC7010E943285803209F07BC0A4
:10C9F0008981882309F477C0853E79F38E3269F303
:10CA00008C8583FDEACF22961FAE1EAE229785E865
:10CA100093E09FAF8EAF24961FAE2497BE016F5F49
:10CA20007F4FE0E080E04EE2DB019D91BD0190325E
:10CA3000A1F0883049F426E730E02C0F3D1F2E0F7F
:10CA4000311DD9014C93EF5F26E730E02C0F3D1FDD
:10CA50002E0F311DD9019C93EF5F8F5F8B3021F733
:10CA600086E790E08C0F9D1F8E0F911DFC011082B8
:10CA7000D60159966D917C9121E0AE014A585F4FE5
:10CA8000CE01CE960E943987882369F1BE01625C8F
:10CA90007F4FCE0181960E94A08AAE014A585F4F17
:10CAA000BE016F5D7F4FCE01855A9F4F0E940E8B56
:10CAB000CE01855A9F4F0E94F08A882309F4ACC0AA
:10CAC000F12CFA141B042CF569E0CE0101960E94AA
:10CAD0005974CE0101960E94F815CE0101960E946C
:10CAE000EE73F394EECF6F961FAE1EAE6F97A396C4
:10CAF0004CAE5DAE6EAE7FAEA3976D961FAF0EAF20
:10CB00006D97E6961FAE1EAEE697A8961FAEA89745
:10CB1000CFCFB401CE0101960E948D74CE01019653
:10CB20000E94F815CE0101960E94EE73E696EEADD6
:10CB3000FFADE697309709F447C08581823008F44D
:10CB400043C06AE674E0CE0101960E948D74CE0166
:10CB500001960E94E115CE0101960E94EE736F9638
:10CB60008EAD9FAD6F979C838B83A3968CAD9DAD4F
:10CB7000AEADBFADA3978D839E83AF83B887A796D5
:10CB80008CAD9DADAEADBFADA79789879A87AB87BA
:10CB9000BC871A8309838DE0F401DE011D960190A4
:10CBA0000D928A95E1F7E6968EAD9FADE6979B8F45
:10CBB0008A8FB101CE0101960E94A664CE01855AEA
:10CBC0009F4F0E94FC8AF3CE61EC78E0CE01019683
:10CBD0000E948D74CE0101960E94F815CE01019637
:10CBE0000E94EE73E696EEADFFADE69740E050E0B2
:10CBF000BA01309721F04389548965897689CE013D
:10CC000001960E940772CE0101960E94E115CE01A5
:10CC100001960E94EE73D2CFCE57DF4F0FB6F89435
:10CC2000DEBF0FBECDBFDF91CF911F910F91FF905F
:10CC3000EF90DF90CF90BF90AF909F908F907F90BC
:10CC40006F905F904F903F902F9008956F927F92DA
:10CC50008F929F92AF92BF92CF92DF92EF92FF920C
:10CC60000F931F93CF93DF93CDB7DEB7C456D1098F
:10CC70000FB6F894DEBF0FBECDBF40E052EC61E0CE
:10CC800070E08CE39DE00E94EB6F40E855E260E0CD
:10CC900070E08FE99CE00E94EB6F61E088E00E9409
:10CCA0003B7761E089E00E943B7760E08AE30E9485
:10CCB0003B7761E088E00E94D87660E089E00E94DE
:10CCC000D87661E08AE00E943B7761E08BE00E94C9
:10CCD0003B7760E08BE30E943B7761E08AE00E9453
:10CCE000D87660E08BE00E94D8760E94247784EFAB
:10CCF00091E0909367028093660265EB7AE08CE3A3
:10CD00009DE00E94E87563EC79E08CE39DE00E9471
:10CD1000EE7460ED77E080E090E00E9491778CE324
:10CD20009DE00E94C16C982E0EE110E091100BC0A6
:10CD30008CE39DE00E94C16C982E6EE170E080E073
:10CD400090E00E9491770150110981F7809166026D
:10CD50009091670203EA1FE09C01235A3F4079014A
:10CD6000C701800F911F0E943EA9F80181938F0196
:10CD7000F0E1053D1F07A1F76091BD107091BE1055
:10CD8000072E000C880B990B0E9421A89B01AC0177
:10CD90000E94E1AA882331F081E090E09093BE10D8
:10CDA0008093BD106091BF107091C010072E000CD1
:10CDB000880B990B0E9421A89B01AC010E94E1AA5B
:10CDC000882331F082E090E09093C0108093BF10F0
:10CDD00025E79216B1F06091B9107091BA10809168
:10CDE000BB109091BC100E9421A89B01AC010E9435
:10CDF000E1AA811106C08091A30F9091A40F8197A1
:10CE0000E8F08DB79EB7825391400FB6F8949EBF5D
:10CE10000FBE8DBFADB7BEB7119682E391E0E3EAD6
:10CE2000FFE001900D920197E1F70E9481240FB677
:10CE3000F894DEBF0FBECDBF15E7912E2DB73EB7DC
:10CE4000225331400FB6F8943EBF0FBE2DBFADB791
:10CE5000BEB7119682E391E0E3EAFFE001900D9204
:10CE60000197E1F70E94B11D0FB6F894DEBF0FBE27
:10CE7000CDBF95E7991619F0E3E79E121BC02DB7B9
:10CE80003EB7225331400FB6F8943EBF0FBE2DBFC0
:10CE9000ADB7BEB7119682E391E0E3EAFFE00190FF
:10CEA0000D920197E1F70E94022B0FB6F894DEBFB6
:10CEB0000FBECDBF63EA7AE089E59FE00E947973F7
:10CEC0006DE87AE083E59FE00E9479730E94247701
:10CED00064EC78E08CE39DE00E94AA75F12CE12CD3
:10CEE00017E201E000939B0C10939D0C10929C0C98
:10CEF00010929E0C81E00E94EF7B81114FC160ED8A
:10CF000078E08CE39DE00E94BE75812F0E944975F8
:10CF100010935D116CEE78E08CE39DE00E94BE758D
:10CF2000812F0E9449759FEFE91AF90A1F5F10349B
:10CF3000C9F661E279E0EF2811F067E379E08CE36C
:10CF40009DE00E94AA750E94247710925E11809144
:10CF50006211823018F098E090935E119091631105
:10CF6000992339F0813029F480915E118460809397
:10CF70005E1162E370E080E090E00E949177609142
:10CF8000641189E591E10E94DF7C68EE73E080E046
:10CF900090E00E94917760E389E591E10E94F37C43
:10CFA0000BE416E4C8010197F1F760E389E591E12C
:10CFB0000E94F37CC8010197F1F760E389E591E1F4
:10CFC0000E94F37C83E592E00197F1F760E289E546
:10CFD00091E10E94F37C80915E1180620E94237D2A
:10CFE00084E080935F118CE00E94237D81E00E94A9
:10CFF000237D0BE31FE1C8010197F1F782E08093E5
:10D00000601186E00E94237D82E00E94237DC8019A
:10D010000197F1F780E40E94237D0EE512E0F8010C
:10D0200061918F0189E591E10E940C7DF2E0063665
:10D030001F07A9F70E94DD080E94CD0864E670E092
:10D0400080E090E00E94917765E77AE0CE0101965A
:10D050000E947B74CE0101960E94E115CE010196DB
:10D060000E94EE7361E085E30E943B7761E085E317
:10D070000E94D87661E08AE00E943B7761E08AE016
:10D080000E94D87668EC70E080E090E00E94917792
:10D0900068EE73E080E090E00E94917764E67AE0C9
:10D0A000CE0101960E947B744AE050E06FEF7FEF63
:10D0B000CE0101960E942A20CE0101960E94EE73B5
:10D0C0001092F20D1092F00D1092ED0D1092EC0DE9
:10D0D00084E08093EB0D0E944F788B0161E080919A
:10D0E000EB0D0E943B7761E08091EB0D0E94D876BA
:10D0F0000E94BF1482E58093E50D1092E60D8091A9
:10D10000E50D9091E60D0E94DD09BAE0FB2E8FEF50
:10D110000E946F09FA94F110FACF87EE9DE00E9409
:10D12000BD7E20E030E0A90160E087EE9DE00E9436
:10D13000FF7EF82E8093F10D21E08217E1F10E942D
:10D140004F78601B710B613D774058F381E080930D
:10D15000EC0D87EE9DE00E94D37E66E57AE0CE017D
:10D1600001960E947B74CE0101960E94E115CE01CA
:10D1700001960E94EE7365E47AE0CE0101960E946A
:10D180007B744AE050E06FEF7FEFCE0101960E9482
:10D190000109CE0101960E94EE731FC1843009F08F
:10D1A000C5CE66E079E08CE39DE00E94BE75812FDC
:10D1B0000E944975BBCE2AEA31E040E050E068E0C9
:10D1C00087EE9DE00E94FF7E82FF2AC0F092F20D62
:10D1D0008091F20DC12CD12CE12CF0E4FF2E823095
:10D1E00019F0C12CD12C760120E030E0A90167E3D1
:10D1F00087EE9DE00E94FF7EA701960169E287EE1F
:10D200009DE00E94FF7E8093F10D8823D1F00E9463
:10D210004F78601B710B613D774030F388E097CF0A
:10D22000A4E0FA2E0E94E17E8093F10DFA94F110B1
:10D23000F9CF8A3A11F082E08ACF82E08093F20D32
:10D24000C7CF8091F20D8230D1F420E030E0A90107
:10D250006AE387EE9DE00E94FF7E882311F086E05E
:10D2600076CF0E94E17E807C803C19F483E080933D
:10D27000F20D0E94E17E0E94E17E0E94E17E87EE37
:10D280009DE00E94D37E80E58093E50D1092E60D2F
:10D2900081E00E94ED80882309F4AAC28091160ED5
:10D2A00081115BCF80910A0E803109F0A8C282E023
:10D2B0008093160E1092280E1092290E10922A0EAC
:10D2C00010922B0E80910B0E90910C0EB0E0A0E00E
:10D2D000E5E0880F991FAA1FBB1FEA95D1F780933D
:10D2E000240E9093250EA093260EB093270E83EF65
:10D2F0009DE090932D0E80932C0E81E08093150E6F
:10D300001092170E1092180E1092190E10921A0EFB
:10D3100010921B0E10921C0E10921D0E10921E0EDB
:10D3200010921F0E1092200E1092210E1092220EBB
:10D330001092230E69E37AE0CE0101960E947B747D
:10D34000CE0101960E94E115CE0101960E94EE7376
:10D3500041E06AE674E0CE0101960E94438BBE0173
:10D360006F5F7F4F82E291E10E9408198091241142
:10D37000909125119C838B83809126119091271188
:10D38000A0912811B09129118D839E83AF83B88716
:10D3900080912A1190912B11A0912C11B0912D11F7
:10D3A00089879A87AB87BC8789EF93E09A838983C3
:10D3B0008DE0EEE2F1E1DE011D9601900D928A957D
:10D3C000E1F780913B1190913C119B8F8A8F70E027
:10D3D00060E0CE0101960E94A66468EE73E080E0F2
:10D3E00090E00E94917743E162EB72E0CE010196FA
:10D3F0000E94438BBE016F5F7F4F8DE391E10E94DE
:10D40000081960E07AE087E49FE00E94797365EF95
:10D4100079E087E49FE00E941C738DE391E10E9414
:10D42000F08A882309F41CC21EAE1DAE85E893E085
:10D430009CAF8BAF21961FAE219719A218A29F8F88
:10D440008E8F1BA2812C712C7E019BE3E90EF11CB7
:10D4500001E11EE075E8A72E73E0B72E882D972D09
:10D46000FC01EE54FD4F20812F3209F40196DC01BE
:10D47000AE54BD4FFE01E85AFF4F30E020E06F018F
:10D480004D914F3249F0442339F001962F5F3F4FC1
:10D4900041932C303105A1F72C0D3D1DF90110826F
:10D4A000FC01EE54FD4F20812F3209F40196882EA5
:10D4B000792E8E549D4FFC0160801C821B82BA82A3
:10D4C000A9821E8221E0A601B801CE0101960E9428
:10D4D0003987882309F4E1C1CE0101960E9425878E
:10D4E0006110ACC12EE00131120719F0C8010E9491
:10D4F00025878DE391E10E94FC8A66E970E080E077
:10D5000090E00E9491771092560C04E610E0911082
:10D510000BC08CE39DE00E94C16C982E64E170E02A
:10D5200080E090E00E9491770150110981F760ED51
:10D5300079E0CE0101960E947B7448EC50E070E0E7
:10D5400060E0CE0101960E940109CE0101960E9481
:10D55000EE7332E781E0931280E00E942B0882E0B4
:10D5600090E00E94B6796CE271E080E090E00E9469
:10D57000917783E090E00E94B6796CE271E080E000
:10D5800090E00E94917768EB79E0CE0101960E94CD
:10D590007B74CE0101960E94E115CE0101960E9496
:10D5A000EE7364E670E080E090E00E94917768EAB4
:10D5B00079E0CE0101960E947B7448EC50E070E067
:10D5C00060E0CE0101960E942A20CE0101960E94C1
:10D5D000EE7301E010E010936F0200936E0210935F
:10D5E0005D0200935C0265E277E08CEF9EE00E94B2
:10D5F000D1716CEF7EE0CE0101960E94847462E0EE
:10D6000070E0CE0101960E94342FCE0101960E9457
:10D61000EE7361E876E08CEF9EE00E94D17162E3E8
:10D6200070E080E090E00E9491776CEF7EE0CE01A8
:10D6300001960E94847463E070E0CE0101960E941E
:10D64000342FCE0101960E94EE7310936F02009367
:10D650006E0262E979E0CE0101960E947B74CE01F0
:10D6600001960E94E115CE0101960E94EE7367E8D3
:10D6700079E0CE0101960E947B744AE050E06FEFA2
:10D680007FEFCE0101960E942A20CE0101960E94D2
:10D69000EE7368EE73E080E090E00E9491770E9464
:10D6A000D9270E94E12810924E0C8FE19DE59093BE
:10D6B000B10E8093B00E2091D20E2830D8F4822F74
:10D6C00090E0FC01EE0FFF1FEE0FFF1FEE54F14F35
:10D6D00040E559E0518340832F5F2093D20E880F9D
:10D6E000991F880F991FFC01EC54F14F89ED99E1C6
:10D6F000918380832091D20E2830D8F4822F90E03D
:10D70000FC01EE0FFF1FEE0FFF1FEE54F14F46E539
:10D7100059E0518340832F5F2093D20E880F991FC9
:10D72000880F991FFC01EC54F14F87EB93E691832E
:10D73000808382E49EE00E94E51165E779E0CE01F6
:10D7400001960E947B74CE0101960E94E115CE01E4
:10D7500001960E94EE738DB79EB7825391400FB62B
:10D76000F8949EBF0FBE8DBFADB7BEB7119682E3D2
:10D7700091E0E3EAFFE001900D920197E1F70E944A
:10D78000022B10924F0C0FB6F894DEBF0FBECDBF28
:10D790000E9470796093500C7093510C8093520CDE
:10D7A0009093530C8091A2108093580C882351F0D1
:10D7B0000E9470796093460C7093470C8093480CDC
:10D7C0009093490CCC59DF4F0FB6F894DEBF0FBED3
:10D7D000CDBFDF91CF911F910F91FF90EF90DF9020
:10D7E000CF90BF90AF909F908F907F906F90089553
:10D7F00080E00E94ED80882309F4AFCC4FCD8032C9
:10D8000009F0ABCC83E08093160E40910D0E509141
:10D810000E0E60910F0E7091100E4093280E5093D3
:10D82000290E60932A0E70932B0E24E23EE083EFC4
:10D830009DE00E94398381115ACD8FCC21E0A60151
:10D84000B801C7010E943987D82EFEE001311F07B9
:10D8500009F44DC0C8010E942587D1104DC024C0D5
:10D8600060EE79E0CE0101960E947B74CE010196B4
:10D870000E94F815CE0101960E94EE7362EB72E0F1
:10D88000CE0101960E948D74CE0101960E94E11591
:10D89000CE0101960E94EE7336CEFEE001311F07E5
:10D8A00019F0C8010E9425876EE379E0CE01019648
:10D8B0000E948D74CE0101960E94F815CE0101964A
:10D8C0000E94EE7362EB72E0CE0101960E948D74AD
:10D8D000CE0101960E94E115CE0101960E94EE73E1
:10D8E00067E47FE08DE391E10E94D47502CE882346
:10D8F000D9F28E01025E1F4F902F812F8701E92EF2
:10D90000F82EACCD089508950895AF92BF92CF92AE
:10D91000DF92EF92FF920F931F93CF93DF936C01EF
:10D920007B018B01040F151FEB015E01AE18BF08D0
:10D93000C017D10759F06991D601ED91FC91019082
:10D94000F081E02DC6011995892B79F7C501DF918A
:10D95000CF911F910F91FF90EF90DF90CF90BF90EC
:10D96000AF900895FC01538D448D252F30E0842F16
:10D9700090E0821B930B541710F0CF9608950197F7
:10D980000895FC01918D828D981761F0A28DAE0FE4
:10D99000BF2FB11D5D968C91928D9F5F9F73928F6B
:10D9A00090E008958FEF9FEF0895FC01918D828D97
:10D9B000981731F0828DE80FF11D858D90E0089564
:10D9C0008FEF9FEF0895FC01918D228D892F90E0BC
:10D9D000805C9F4F821B91098F73992708958FE96F
:10D9E0009CE00E94E36C21E0892B09F420E0822F67
:10D9F00008958CE39DE00E94E36C21E0892B09F4FB
:10DA000020E0822F0895FC01A48DA80FB92FB11D2D
:10DA1000A35ABF4F2C91848D90E001968F73992764
:10DA2000848FA689B7892C93A089B1898C91837042
:10DA300080648C93938D848D981306C00288F3893B
:10DA4000E02D80818F7D80830895EF92FF920F9368
:10DA50001F93CF93DF93EC0181E0888F9B8D8C8D9A
:10DA600098131AC0E889F989808185FF15C09FB78E
:10DA7000F894EE89FF896083E889F9898081837051
:10DA8000806480839FBF81E090E0DF91CF911F9100
:10DA90000F91FF90EF900895F62E0B8D10E00F5F21
:10DAA0001F4F0F731127E02E8C8D8E110CC00FB6F7
:10DAB00007FCFACFE889F989808185FFF5CFCE018F
:10DAC0000E94036DF1CFEB8DEC0FFD2FF11DE35A9A
:10DAD000FF4FF0829FB7F8940B8FEA89FB89808112
:10DAE0008062CFCFCF93DF93EC01888D8823B9F08C
:10DAF000AA89BB89E889F9898C9185FD03C0808159
:10DB000086FD0DC00FB607FCF7CF8C9185FFF2CFD5
:10DB1000808185FFEDCFCE010E94036DE9CFDF91BB
:10DB2000CF91089580E090E0892B29F00E94F96C54
:10DB300081110E94000080E090E0892B49F080E094
:10DB400090E0892B29F00E94000081110E940000C2
:10DB500080E090E0892B49F080E090E0892B29F06B
:10DB60000E94000081110E94000080E090E0892B5B
:10DB700029F00E94EF6C81110C94000008958150EF
:10DB8000823108F05AC0E82FF0E08827E553F249C7
:10DB90008F4F0C94FAAAEB6DEF6DDD6DE36DE76DC1
:10DBA0001D6EF26DF86DFC6D026E066E0A6E106EE3
:10DBB000146E1D6E186E1E6E226E809180008F771F
:10DBC000809380000895809180008F7DF9CF8091AF
:10DBD0008000877FF5CF84B58F7784BD089584B5A5
:10DBE0008F7DFBCF8091B0008F778093B000089538
:10DBF0008091B0008F7DF9CF809190008F778093D6
:10DC000090000895809190008F7DF9CF80919000D1
:10DC1000877FF5CF8091A0008F778093A000089533
:10DC20008091A0008F7DF9CF8091A000877FF5CFF4
:10DC3000809120018F7780932001089580912001A9
:10DC40008F7DF9CF80912001877FF5CFCF93DF9330
:10DC5000282F30E0F901E650F34F8491F901EC549C
:10DC6000F34FD491F901E259F34FC491CC23A1F0C1
:10DC700081110E94BF6DEC2FF0E0EE0FFF1FEC5AF8
:10DC8000F34FA591B491EC91ED2381E090E009F47C
:10DC900080E0DF91CF91089580E090E0FACF20916D
:10DCA0009211260F3327331F21323105ECF42091D6
:10DCB000950CFC0190E080E0243069F082E008954A
:10DCC000A09192112191AC014E585E4EA40FB52F38
:10DCD000B11D2C930196861798F380919211680FCD
:10DCE0006093921180E0089581E008950895E09195
:10DCF000550C8091540CE81730F4F0E0EF5FF34FCF
:10DD0000808190E008958FEF9FEF08959091550CDA
:10DD10008091540C2FEF3FEF981748F4E92FF0E073
:10DD2000EF5FF34F208130E09F5F9093550CC90166
:10DD300008958091540C9091550C891B990B08956E
:10DD4000CF92DF92EF92FF920F931F93CF93DF93C7
:10DD50007C01CB018A0120919B0C222389F0EB01ED
:10DD60006B01C40ED51ECC15DD0569F06991D70194
:10DD7000ED91FC910190F081E02DC7011995F3CF51
:10DD8000642F0E944F6EC801DF91CF911F910F91B8
:10DD9000FF90EF90DF90CF900895CF93DF931F9285
:10DDA000CDB7DEB7698320919B0C2223F9F0209137
:10DDB0009E0C203258F021E030E0FC0133832283B6
:10DDC00090E080E00F90DF91CF91089580919C0CBE
:10DDD000E82FF0E0EB5EFA4E998190838F5F80939D
:10DDE0009C0C80939E0C81E090E0ECCF61E0CE0132
:10DDF00001960E944F6EF7CFDC015996ED91FC9190
:10DE00003097B9F083899489A589B689428553856D
:10DE100064857585841B950BA60BB70B811520E8CF
:10DE20009207A105B10538F08FEF9FE7A0E0B0E0C1
:10DE3000089590E080E00895CF93DF931F92CDB7CF
:10DE4000DEB76983DC01ED91FC910280F381E02D66
:10DE500041E050E0BE016F5F7F4F19950F90DF9159
:10DE6000CF9108950E9423AD0F931F93CF93DF931B
:10DE7000EC0188819981009759F02A813B8126170E
:10DE8000370730F081E0DF91CF911F910F91089516
:10DE90008B016F5F7F4F0E9442AC009759F09983CE
:10DEA00088831B830A832C813D81232B59F7FC0136
:10DEB0001082E8CF80E0E7CFEF92FF920F931F939D
:10DEC000CF93DF936115710541F480E0DF91CF912D
:10DED0001F910F91FF90EF90089541155105B1F0FA
:10DEE0007B01EC010C811D81040F151FB8010E94FC
:10DEF000346F882351F3288139818C819D81B7014A
:10DF0000820F931F0E9473AD1D830C8381E0DECFCF
:10DF1000CF93DF93EC0188819981009711F00E94E3
:10DF2000B9AB198218821D821C821B821A82DF9172
:10DF3000CF910895EF92FF920F931F93CF93DF93AA
:10DF4000EC017B018A01BA010E94346F81110BC080
:10DF5000CE010E94886FCE01DF91CF911F910F916A
:10DF6000FF90EF9008951D830C83B70188819981FC
:10DF70000E9473ADF0CFCF92DF92EF92FF920F939A
:10DF80001F93CF93DF93EC017A018B016C01C40ED8
:10DF9000D51ECC15DD05A9F00E946D098FE00E9409
:10DFA0006F098D2F0E946F098C2F0E946F09219697
:10DFB00080E00E946F09F80181938F010E946B0934
:10DFC000E8CFC701DF91CF911F910F91FF90EF90A4
:10DFD000DF90CF900895CF93DF93EC019A01AB01CE
:10DFE000E889F98982E08083211581EE38074105AF
:10DFF000510581F160E079E08DE390E00E9464A931
:10E000002150310941095109569547953795279572
:10E01000EC85FD851082EE85FF852083188EEC89C6
:10E02000FD8986E08083EA89FB8980818061808325
:10E03000EA89FB89808188608083EA89FB89808105
:10E0400080688083EA89FB8980818F7D8083DF916E
:10E05000CF910895E889F989108220E1D9CF2F92D4
:10E060003F924F925F926F927F928F929F92AF9268
:10E07000BF92CF92DF92EF92FF920F931F93CF93B5
:10E08000DF9300D0CDB7DEB71C013B014A01290167
:10E090005801FC01C080D18070E060E0C3010E94A3
:10E0A00058ADA80170E060E0C2010E9458ADF601D1
:10E0B000808110E000E0811162C004E010E004C043
:10E0C0007601F101F182E082C8010F900F900F906C
:10E0D000DF91CF911F910F91FF90EF90DF90CF9044
:10E0E000BF90AF909F908F907F906F905F904F9078
:10E0F0003F902F9008956B3209F482C06D3309F080
:10E100004EC081818823E9F2F7018FEFE81AF80AFF
:10E110006081653209F452C00CF048C0662309F4EE
:10E1200056C082E0A816B1040CF061C0012B09F4BE
:10E130006BC003E010E0E8CF81818983882309F276
:10E1400082818A837601811104C0F2E0EF0EF11C16
:10E15000B8CF83E0E80EF11C1B8240E150E070E094
:10E1600060E0CE0101960E94DD9F19C0F30160833B
:10E17000F1E08F1A9108C30101963C016701760115
:10E18000FFEFEF1AFF0AF6016081663209F499CFBA
:10E190000CF0B1CF662309F493CF653269F2F2E057
:10E1A0008F1691041CF701E010E0E8CF663209F405
:10E1B00088CF6B3209F0B5CF60E2B3CF818189831C
:10E1C000882301F182818A83811103C032967F0105
:10E1D00078CF7F0193E0E90EF11C1B8240E150E013
:10E1E00070E060E0CE0101960E94DD9F9ACFF201BF
:10E1F0006083F1E0AF1AB108C20101962C0184CF0F
:10E2000060E2CDCFF701E3CF02E010E07DCFCF9306
:10E21000DF93EC0187E194E0998388831A821B8263
:10E220001C821D8280E590E00E94DD09BE016E5FC8
:10E230007F4F44E050E08FE090E00E94BB6F0E946F
:10E24000DC09CE01DF91CF9108950F931F93CF93F7
:10E25000DF934115510541F0FC0104811581011541
:10E26000110539F4FB011082DF91CF911F910F91BD
:10E270000895415051094017510708F48A01EB01F4
:10E28000FC0160817181A801CE010E9488ADC00FA0
:10E29000D11F1882E9CFCF93C82F462F61E070E0DD
:10E2A0000E94760961E070E08C2F0E949109811133
:10E2B000F9CFCF910895FF920F931F93CF93DF93E0
:10E2C000F82E10E000E08F2D0E94C209EC01892B8E
:10E2D00021F08F2D0E94C2098C01C017D10799F738
:10E2E000CE01DF91CF911F910F91FF900895AF92D2
:10E2F000BF92CF92DF92EF92FF920F931F93CF9333
:10E30000DF931F921F92CDB7DEB77A836983BA017C
:10E31000A901E981FA81F770082F10E0000F111FA1
:10E320000D59134FD8018D919C918E0F9F1F9F0106
:10E33000240F351F21303840A0F05A016B0160E0F6
:10E3400078E07B01EE1AFF0AA701B6010E94BB6FBD
:10E35000A5014E195F09B6016E0D7F1DF801808180
:10E3600091810F900F90DF91CF911F910F91FF90AE
:10E37000EF90DF90CF90BF90AF900C94BB6F20E3F5
:10E38000FC0120833296862F82958F706F706A30E1
:10E3900030F4605D6293682F8111F5CF0895695C58
:10E3A000F9CFFB0101900020E9F73197AF01461B3F
:10E3B000570B0C949A6F0F931F93CF93DF93CDB7A6
:10E3C000DEB762970FB6F894DEBF0FBECDBF8C01EB
:10E3D000CB01F801118210821382128215821482FD
:10E3E0004AE0BE016F5F7F4F0E9424A1BE016F5FB4
:10E3F0007F4FC8010E94D17162960FB6F894DEBFBC
:10E400000FBECDBFDF91CF911F910F9108950F9354
:10E410001F93CF93DF93CDB7DEB7A1970FB6F894D4
:10E42000DEBF0FBECDBF8C01CB01BA01F801118256
:10E43000108213821282158214822AE0AE014F5F8D
:10E440005F4F0E945EA1BE016F5F7F4FC8010E94B7
:10E45000D171A1960FB6F894DEBF0FBECDBFDF918C
:10E46000CF911F910F910895FC01808191810097B8
:10E4700011F00C94E0A060E070E0CB010895FC0185
:10E4800080819181009711F00C94E4A060E070E02D
:10E49000CB010895AF92BF92CF92DF92EF92FF929D
:10E4A0000F931F93CF93DF93DC01CD90DC901197F6
:10E4B000C114D10439F01496CD91DC918C01760110
:10E4C000209761F4DF91CF911F910F91FF90EF9012
:10E4D000DF90CF90BF90AF90089575015701BFEFC7
:10E4E000AB1ABB0AF7018081082E000C990B0E9421
:10E4F0000BA1892B91F72197CC0DDD1D8881082E6A
:10E50000000C990B0E940BA1892B29F0CE15DF0579
:10E5100010F02197F3CFAE014F5F5F4F4E195F09A7
:10E52000D80115965C934E931497CE14DF0420F413
:10E53000B701C6010E943DADD801ED91FC91119744
:10E5400014968D919C91E80FF91F1082BBCFFC01AE
:10E55000248135816217730748F480819181009787
:10E5600029F0860F971FFC018081089580E00895AF
:10E57000FC0124813581FB01448155812417350735
:10E58000A0F0FC0180819181009779F0FB0160810E
:10E5900071816115710549F0241B350B820F931FA2
:10E5A0000E946AAD21E0892B09F020E0822F0895B6
:10E5B000FB0144815581FC012481358124173507F5
:10E5C00078F080819181009759F0FB016081718121
:10E5D0006115710529F00E947AAD21E0892B09F0BF
:10E5E00020E0822F0895CF93DF93EC01FB0101908F
:10E5F0000020E9F73197AF01461B570B0E945C6F73
:10E60000811103C0CE010E94886FCE01DF91CF91AE
:10E610000895CF93DF93EC01FB0144815581608124
:10E6200071810E945C6F811103C0CE010E94886FCE
:10E63000CE01DF91CF910895EF92FF920F931F9338
:10E64000CF93DF93EC017B01CB010E941BA10097CC
:10E65000A9F00C811D81080F191FB801CE010E947D
:10E66000346F882361F0288139818C819D81B701C5
:10E67000820F931F0E9414A11D830C8381E0DF9100
:10E68000CF911F910F91FF90EF900895CF93DF935B
:10E690001F921F92CDB7DEB769831A8241E050E026
:10E6A000BE016F5F7F4F0E945C6F0F900F90DF91F4
:10E6B000CF910895CF93DF93EC010E9446738111AF
:10E6C00003C0CE010E94886FCE01DF91CF910895E3
:10E6D000FB0101900020E9F73197AF01461B570B72
:10E6E0000C945C6FFB0144815581608171810C94B5
:10E6F0005C6FEF92FF920F931F93CF93DF93EC0128
:10E700008B01CB010E941BA17C01BC01CE010E94A8
:10E71000346F81110BC0CE010E94886FCE01DF9152
:10E72000CF911F910F91FF90EF900895FD82EC82A1
:10E73000B801888199810E9414A1F0CFCF93DF9313
:10E74000EC01FB018617970749F060817181611523
:10E75000710541F0448155810E949A6FCE01DF918D
:10E76000CF9108950E94886FF9CF0F931F93CF9395
:10E77000DF938C01EB01FC01808191810097E1F036
:10E780006881798161157105A9F0428153812C81DD
:10E790003D814217530770F00E9473AD8C819D81BB
:10E7A000F801958384831D821C82DF91CF911F9194
:10E7B0000F9108950E94B9AB88819981F8019183E6
:10E7C00080838A819B81938382838C819D819583C1
:10E7D0008483198218821B821A82E5CFFC01808112
:10E7E0009181009711F00C94B9AB0895EF92FF92CC
:10E7F0000F931F93CF93DF93CDB7DEB7A1970FB6DB
:10E80000F894DEBF0FBECDBF7C01CB01BA01F7018A
:10E8100011821082138212821582148242E0420F0A
:10E820008E010F5F1F4F0E941B9F009789F0BC0154
:10E83000C7010E94D171A1960FB6F894DEBF0FBE3A
:10E84000CDBFDF91CF911F910F91FF90EF90089571
:10E85000C7010E94886FEFCF0F931F93CF93DF9371
:10E86000CDB7DEB7A2970FB6F894DEBF0FBECDBF0F
:10E870008C01CB01BA01F80111821082138212823D
:10E880001582148230E0AE014F5F5F4F0E942FA1CE
:10E89000BE016F5F7F4FC8010E94D171A2960FB673
:10E8A000F894DEBF0FBECDBFDF91CF911F910F91C6
:10E8B0000895CF93DF931F921F92CDB7DEB7FC016F
:10E8C00011821082138212821582148269831A8245
:10E8D000BE016F5F7F4F0E94D1710F900F90DF914B
:10E8E000CF910895FC011182108213821282158249
:10E8F00014820C94B573FC0111821082138212826F
:10E90000158214820C947973FC0111821082138297
:10E910001282158214820C949E73FC011182108263
:10E9200013821282158214826115710551F0FB0168
:10E9300001900020E9F73197AF01461B570B0C946B
:10E940009A6F0895AF92BF92CF92DF92EF92FF92AB
:10E950000F931F93CF93DF936C015B017A018901C1
:10E960002417350720F48F2D7901042F182F63EC1D
:10E9700078E0C6010E948D74D5011496CD91DC918A
:10E98000EC16FD06E0F40C171D0708F4E801D501AC
:10E99000ED91FC911197EC0FFD1F108110826D918C
:10E9A0007C916E0D7F1DC60161157105A1F00E945D
:10E9B000D171F50180819181C80FD91F1883C601DB
:10E9C000DF91CF911F910F91FF90EF90DF90CF904B
:10E9D000BF90AF9008950E94886FEBCFFB0101902C
:10E9E0000020E9F73197AF01461B570BDC01ED9191
:10E9F000FC910280F381E02D19948F929F92AF9247
:10EA0000BF92EF92FF920F931F93CF93DF93CDB7F7
:10EA1000DEB7A1970FB6F894DEBF0FBECDBF7C0165
:10EA2000FA01CB0119A2223008F42AE08E010F5D11
:10EA30001F4F822E912CB12CA12CBF01A501940156
:10EA40000E9464A9F901CA016A300CF5605DD80121
:10EA50006E938D01232B242B252B79F790E080E0FA
:10EA6000109721F0BD01C7010E94EE74A1960FB668
:10EA7000F894DEBF0FBECDBFDF91CF911F910F91F4
:10EA8000FF90EF90BF90AF909F908F900895695C3A
:10EA9000DECFCF93DF93482F50E070E060E020E1BD
:10EAA0008CE39DE00E94FD74EC0163EC79E08CE363
:10EAB0009DE00E94EE748C0F9D1FDF91CF91089511
:10EAC0008F929F92AF92BF92CF92DF92EF92FF927E
:10EAD0000F931F93CF93DF937C01EB016C0182E0D6
:10EAE000C80ED11C4701E5E08E0E911C10E000E03D
:10EAF000F60141916F0150E070E060E02AE0CE0144
:10EB00000E94FD745C01E881F9810190F081E02DA3
:10EB10006EE2CE0119958A0D9B1D080F191FC814AE
:10EB2000D90431F7F701458150E070E060E02AE058
:10EB3000CE010E94FD74800F911FDF91CF911F9134
:10EB40000F91FF90EF90DF90CF90BF90AF909F908C
:10EB50008F9008950F931F93CF93DF93EC010E9442
:10EB6000EE748C0163EC79E0CE010E94EE74800FAC
:10EB7000911FDF91CF911F910F910895611571053C
:10EB800011F00C94EE7490E080E00895DB0114968F
:10EB90004D915C9115976D917C91DC01ED91FC910B
:10EBA0000280F381E02D19940F931F93CF93DF938D
:10EBB000EC010E94C6758C0163EC79E0CE010E94E5
:10EBC000EE74800F911FDF91CF911F910F910895E7
:10EBD000EF92FF920F931F93CF93DF938C017B01F2
:10EBE000D0E0C0E0F701EC0FFD1F6491662361F0F7
:10EBF000D801ED91FC910190F081E02DC8011995AB
:10EC0000892B11F02196EECFCE01DF91CF911F918C
:10EC10000F91FF90EF900895DC0187E194E08D93D0
:10EC20009D9384E0FB0101900D928A95E1F7089590
:10EC30001F920F920FB60F9211240BB60F922F93C3
:10EC40003F934F935F936F937F938F939F93AF9374
:10EC5000BF93EF93FF938FE99CE00E94036DFF91B8
:10EC6000EF91BF91AF919F918F917F916F915F9144
:10EC70004F913F912F910F900BBE0F900FBE0F90B1
:10EC80001F9018951F920F920FB60F9211240BB67A
:10EC90000F922F938F939F93EF93FF93E091AF0C7D
:10ECA000F091B00C8081E091B50CF091B60C82FD32
:10ECB0001DC090818091B80C8F5F8F732091B90C2B
:10ECC000821741F0E091B80CF0E0E156F34F958FD8
:10ECD0008093B80CFF91EF919F918F912F910F909E
:10ECE0000BBE0F900FBE0F901F9018958081F2CF32
:10ECF0001F920F920FB60F9211240BB60F922F9303
:10ED00003F934F935F936F937F938F939F93AF93B3
:10ED1000BF93EF93FF938CE39DE00E94036DFF91FF
:10ED2000EF91BF91AF919F918F917F916F915F9183
:10ED30004F913F912F910F900BBE0F900FBE0F90F0
:10ED40001F9018951F920F920FB60F9211240BB6B9
:10ED50000F922F938F939F93EF93FF93E0914C0D1E
:10ED6000F0914D0D8081E091520DF091530D82FD97
:10ED70001DC090818091550D8F5F8F732091560D2E
:10ED8000821741F0E091550DF0E0E45CF24F958F71
:10ED90008093550DFF91EF919F918F912F910F903F
:10EDA0000BBE0F900FBE0F901F9018958081F2CF71
:10EDB0001F93CF93DF93282F30E0F901E650F34FF4
:10EDC0008491F901EC54F34FD491F901E259F34FD6
:10EDD000C491CC23A9F0162F81110E94BF6DEC2F96
:10EDE000F0E0EE0FFF1FE65CF34FA591B4918FB7F3
:10EDF000F894EC91111108C0D095DE23DC938FBFFD
:10EE0000DF91CF911F910895DE2BF8CF1092950CD2
:10EE100081E08093940C10926F0C61E084E10E9479
:10EE2000D87661E085E10E94D876E9EBF0E0808158
:10EE30008E7F808380818D7F808388E48093B8007B
:10EE400085E48093BC0008951092550C1092540CE8
:10EE500010929C0C10929E0C0E94067782E89CE611
:10EE60009093AA128093A91283E89CE69093A8122B
:10EE70008093A7120895CF93DF9390E0FC01EC54A8
:10EE8000F34F24918259934FFC0184918823D1F050
:10EE900090E0880F991FFC01E05EF34FA591B491BB
:10EEA000FC01E65CF34FC591D49161110EC09FB790
:10EEB000F8948C91E22FE0958E238C932881E223A5
:10EEC000E8839FBFDF91CF9108958FB7F894EC91BD
:10EED000E22BEC938FBFF6CF3FB7F89480919D1251
:10EEE00090919E12A0919F12B091A01226B5A89B5E
:10EEF00005C02F3F19F00196A11DB11D3FBFBA2FCC
:10EF0000A92F982F8827BC01CD01620F711D811D8B
:10EF1000911D42E0660F771F881F991F4A95D1F710
:10EF200008958F929F92AF92BF92CF92DF92EF920D
:10EF3000FF926B017C010E946C774B015C01C11454
:10EF4000D104E104F104B9F00E946C7768197909E1
:10EF50008A099B09683E73408105910580F321E091
:10EF6000C21AD108E108F10888EE880E83E0981EE5
:10EF7000A11CB11CE4CFFF90EF90DF90CF90BF9029
:10EF8000AF909F908F900895AF92BF92CF92DF92F3
:10EF9000EF92FF920F931F93CF93DF93C82FD62F3B
:10EFA0001092DD101092DE101092DF101092E0101F
:10EFB0001092E11061E00E943B7760E08C2F0E948C
:10EFC000D8766D2F70E090E080E00E94917760E04D
:10EFD0008C2F0E943B778BE990E00197F1F700E9D5
:10EFE00011E08C2F0E94266E892B81F401501109AB
:10EFF000C1F78EEF9FEFDF91CF911F910F91FF909F
:10F00000EF90DF90CF90BF90AF90089500E911E0AE
:10F010008C2F0E94266E019721F401501109C1F72F
:10F02000E8CF18E2D0E800E090E9E92EFF24F3945D
:10F030008C2F0E94266E892B29F481E0E81AF108B2
:10F04000B9F7D7CF0E946C776B017C0180E9A82EBD
:10F05000BB24B3948C2F0E94266E019729F481E083
:10F06000A81AB108B9F7C5CF0E946C776C197D0951
:10F070008E099F09693271058105910538F0E02FED
:10F08000F0E0EB52FF4E80858D2B8087D69511F4F2
:10F090000F5FD0E8115041F690E080E0ACCF2FB781
:10F0A000F8946091991270919A1280919B129091AC
:10F0B0009C122FBF0895CF92DF92EF92FF92CF93D1
:10F0C000DF938091540E843051F4CFEFDFEFCE0107
:10F0D000DF91CF91FF90EF90DF90CF900895E09176
:10F0E000770EE1113EC00E944F786B017C0128EE43
:10F0F000C20E23E0D21EE11CF11C88E49EE00E94B7
:10F10000A60C882311F38091AD0E882331F08091F5
:10F11000780E9091790E892BC1F288E49EE00E94CE
:10F12000770BEC01CF3FDC0771F08091AD0E8823A7
:10F1300071F28091780E9091790E01979093790EEB
:10F140008093780EC4CF0E944F78C616D706E80683
:10F15000F90698F61092770E88E49EE00E9451120C
:10F16000B6CFE150E093770EF0E0E25CF14FC18D55
:10F17000D0E0ADCF0F931F93CF93DF93EC018C01C1
:10F18000F80181918F018823A1F10E945B78F80139
:10F190002291022E000C330B8217930789F38F3FC5
:10F1A000980781F0A091770E91E09A0F9093770ED7
:10F1B000B0E0A25CB14F59968C93903219F48FE174
:10F1C0008093770E2FE1EC17FD07C9F092919F3FD6
:10F1D000D1F3A091770E81E08A0F8093770EB0E093
:10F1E000A25CB14F59969C93803269F72093770EB9
:10F1F000EACF81E0DF91CF911F910F91089580E0D8
:10F20000F9CF1F920F920FB60F9211242F933F93B5
:10F210008F939F93AF93BF938091991290919A127D
:10F22000A0919B12B0919C123091981223E0230F71
:10F230002D3758F50196A11DB11D2093981280938A
:10F24000991290939A12A0939B12B0939C12809162
:10F250009D1290919E12A0919F12B091A0120196C2
:10F26000A11DB11D80939D1290939E12A0939F1299
:10F27000B093A012BF91AF919F918F913F912F9129
:10F280000F900FBE0F901F90189526E8230F02963F
:10F29000A11DB11DD2CF60939412709395128093EB
:10F2A000961290939712645D7E4F8F4F9F4F60939D
:10F2B000901270939112809392129093931282E025
:10F2C00090E090938F1280938E120E944F786093FB
:10F2D0008A1270938B1280938C1290938D120895E2
:10F2E000CF92DF92EF92FF920F931F930E944F787D
:10F2F0008B019C01C0908A12D0908B12E0908C12EE
:10F30000F0908D12609194127091951280919612E6
:10F31000909197120C191D092E093F09083E1340C0
:10F3200021053105E0F0DC01CB010196A11DB11DE5
:10F330008093941290939512A0939612B093971283
:10F34000B701A60148515C4F6F4F7F4F40938A121F
:10F3500050938B1260938C1270938D12C7CF1F91B4
:10F360000F91FF90EF90DF90CF900895CF93DF93B0
:10F37000EC010E9470799E01220F331F220F331F70
:10F38000F901E152FD4F6083718382839383CE0143
:10F39000880F991FFC01E952FD4F408151811416DD
:10F3A000150644F4FC01E153FD4F408151811416D0
:10F3B000150614F1FC01E952FD4F41E050E0518384
:10F3C000408381539D4FFC015183408321543D4F25
:10F3D00088E097E0A0E0B0E0F90180839183A28308
:10F3E000B383CE010E94F51464EF71E080E090E0F9
:10F3F000DF91CF910C949177DF91CF9108954F9247
:10F400005F926F927F928F929F92AF92BF92CF92B4
:10F41000DF92EF92FF920F931F93CF93DF934B01F5
:10F420005C018091861290918712A0918812B09110
:10F43000891288159905AA05BB0509F4C6C08CE395
:10F44000C82ED12CE12CF12CC501A70196010E94F8
:10F4500064A96093210CCA01B901A70196010E9419
:10F4600064A96093220CC501B40120E13EE040E0B4
:10F4700050E00E9464A9CA01B90128E130E040E0EF
:10F4800050E00E9464A96093230CC501B40120E8F8
:10F4900031E541E050E00E9464A969017A01CA01A6
:10F4A000B9016C5F7F4F8F4F9F4F27E030E040E006
:10F4B00050E00E9464A96F5F6093240C412C512C92
:10F4C000320140E004E610E0C0E9D1E0242F30E052
:10F4D0002E54384FF901E370FF273097F9F4C90132
:10F4E000B8010E94E6AA892B31F4C901BE010E942D
:10F4F000E6AA892B99F48EE691E0A0E0B0E0480EF0
:10F50000591E6A1E7B1ED301C201AA27BB27C8163B
:10F51000D906EA06FB0638F04F5FD8CF8DE691E0BA
:10F52000A0E0B0E0ECCF4093270CC90164E670E0A6
:10F530000E94E6AAEC01C90160E971E00E94E6AA16
:10F54000309721F42097D9F40097C9F04DE651E0A7
:10F5500060E070E0441A550A660A770AC418D508B4
:10F56000E608F708A5E3B3E020E0213069F430971E
:10F57000E9F5209711F40097C9F54DE106C04EE674
:10F5800051E060E070E0E6CF4C9150E070E060E068
:10F5900031E0320FC416D506E606F70640F0C41A6D
:10F5A000D50AE60AF70A1196232F3C30F1F62F5FB1
:10F5B0002093260CC394C092250C809286129092C0
:10F5C0008712A0928812B0928912DF91CF911F9179
:10F5D0000F91FF90EF90DF90CF90BF90AF909F90F2
:10F5E0008F907F906F905F904F9008954CE1CDCFBA
:10F5F0000E9470790E94FF798091270C90E08E54D0
:10F60000984F08950E9470790E94FF798091260C8E
:10F6100090E008950E9470790E94FF798091250CF6
:10F6200090E008950E9470790E94FF798091220CE9
:10F6300090E008950E9470790E94FF798091230CD8
:10F6400090E008951F920F920FB60F9211240BB6FF
:10F650000F922F933F934F935F936F937F938F936B
:10F660009F93AF93BF93EF93FF938091B6110E9446
:10F67000266E2091B9113091BA112F5F3F4F309310
:10F68000BA112093B9119091B811953618F096E0FF
:10F690009093B5119091B511943009F46EC0F8F4BF
:10F6A000923031F1933009F44CC09091B711992305
:10F6B00019F0811171C02F9AFF91EF91BF91AF9115
:10F6C0009F918F917F916F915F914F913F912F917A
:10F6D0000F900BBE0F900FBE0F901F901895953096
:10F6E00009F457C0963009F791E0909385124FC006
:10F6F0008111DBCF2091B9113091BA112436310537
:10F7000028F41092BA111092B911CFCF109285122D
:10F710001092B811E091B81191E09E0F9093B8113A
:10F72000F0E02091B9113091BA11EE0FFF1FE554AE
:10F73000FE4E318320831092BA111092B91193E0DA
:10F7400019C0813009F0B1CFE091B81191E09E0F5E
:10F750009093B811F0E02091B9113091BA11EE0FE9
:10F76000FF1FE554FE4E318320831092BA11109290
:10F77000B91194E09093B51198CF882359F2209154
:10F78000B9113091BA112536310508F48ECF95E0C4
:10F79000F1CF81118ACFB5CF2F988ECFCF93DF9342
:10F7A00091E0909371118823B9F0C091B800D09185
:10F7B000BA008091BC008A7B8093BC0060E084E149
:10F7C0000E94D87660E085E10E94D8760E94067794
:10F7D000D093BA00C093B800DF91CF9108958F9273
:10F7E0009F92AF92BF92CF92DF92EF92FF920F93D0
:10F7F0001F93CF93DF93D0919E0CD13208F0D7C0E6
:10F80000182FC0919D0C0E946C776B017C01809138
:10F81000950C81116BC082E08093950C1093940C31
:10F820008FEF8093930C1092920CD093910CA5E1E2
:10F83000B5E1E1E7FCE080E0D81391C01092700CD4
:10F840008091700CCC0FC82BC093700C80916F0C02
:10F85000813009F088C010926F0C0E946C776B01A8
:10F860007C018091700C8093BB008091970C9091EB
:10F87000980CA091990CB0919A0C892B8A2B8B2B08
:10F88000A1F00E946C770091970C1091980C209138
:10F89000990C30919A0C6C197D098E099F090617F5
:10F8A00017072807390708F442C08091BC0083FD80
:10F8B000D8CF85EC8093BC000E946C776B017C01F3
:10F8C0008091950C823009F450C08091930C8F3F49
:10F8D00009F46FC08091930C803209F46CC0809160
:10F8E000930C803309F469C084E026C08091970CA2
:10F8F0009091980CA091990CB0919A0C892B8A2B1D
:10F900008B2B09F484CF0E946C778090970C909099
:10F91000980CA090990CB0909A0C6C197D098E09E6
:10F920009F0986169706A806B90608F070CF809141
:10F93000960C0E94CE7B85E010929C0C10929E0C3F
:10F9400010929B0CDF91CF911F910F91FF90EF9040
:10F95000DF90CF90BF90AF909F908F9008959D9132
:10F9600091938F5F69CF85EEA5CF8091970C909191
:10F97000980CA091990CB0919A0C892B8A2B8B2B07
:10F9800009F49ECF0E946C770091970C1091980C0F
:10F990002091990C30919A0C6C197D098E099F0960
:10F9A000061717072807390708F08ACFC0CF81E06C
:10F9B000C3CF80E0C1CF82E0BFCF83E0BDCFFC01E9
:10F9C000248131E030939B0C20939D0C10929C0C71
:10F9D00010929E0C8385682B89ED9DE00E94CD6E70
:10F9E00081E00C94EF7B0F931F93CF938C01C62F74
:10F9F0000E94DF7C6C2F6460C8010E94DF7C6C2F4A
:10FA00006B7FC8010E94DF7C83EC90E00197F1F7E7
:10FA1000CF911F910F9108950F931F93CF938C0156
:10FA2000C62F607F61600E94F37C80E1C89FB001B7
:10FA300011246160C8010E94F37C81E090E0CF91C5
:10FA40001F910F910895CF93C82F682F607F89E58C
:10FA500091E10E94F37C80E1C89FB001112489E507
:10FA600091E1CF910C94F37CCF93DF9300D000D041
:10FA70001F921F92CDB7DEB798E0EBE2F3E0DE0114
:10FA8000119601900D929A95E1F790916211961757
:10FA900008F46FEF70E0660F771F21E030E02C0F65
:10FAA0003D1F620F731FFB019081890F80682896AC
:10FAB0000FB6F894DEBF0FBECDBFDF91CF910C948F
:10FAC000237D85ED8093BC008091970C9091980CDC
:10FAD000A091990CB0919A0C0796A11DB11D23E03D
:10FAE000B695A795979587952A95D1F72091BC0053
:10FAF00024FD03C01092950C08954091970C5091ED
:10FB0000980C6091990C70919A0C452B462B472BC1
:10FB100069F30097A105B10541F025E32A95F1F7B6
:10FB200000000197A109B109E1CF8091960C0C94D6
:10FB3000CE7B1F920F920FB60F9211240BB60F922D
:10FB40002F933F934F935F936F937F938F939F93E5
:10FB5000AF93BF93EF93FF938091B900887F803676
:10FB600009F44DC008F040C0883209F4A9C028F556
:10FB7000803109F49DC0C8F4882309F4FBC08830A3
:10FB800009F496C0FF91EF91BF91AF919F918F9132
:10FB90007F916F915F914F913F912F910F900BBE8D
:10FBA0000F900FBE0F901F901895883109F488C0F0
:10FBB000803241F78093930C14C0803409F49DC0C7
:10FBC00040F48033B9F38833E9F68093930C85ECE5
:10FBD000B0C0803509F485C0883509F496C08834F2
:10FBE00089F60E94617DCECF883909F48CC038F542
:10FBF000883729F050F4883611F0803719F683E001
:10FC00008093950C1092B41157C0883809F47BC0CA
:10FC1000803919F0803809F0B5CF8091B411803265
:10FC200008F071C0E091B41181E08E0F8093B4119F
:10FC30008091BB00F0E0EC56FE4E80833DC0803BDF
:10FC400039F0E0F4803A09F479C0883A09F09ACFA3
:10FC500084E08093950C1092931110929211E09190
:10FC6000A912F091AA1219958091921181110FC0D9
:10FC700081E0809392111092721109C0803C09F4C6
:10FC8000A6CF883C09F4A3CF883B09F07BCFE09155
:10FC9000931181E08E0F80939311F0E0EE58FE4EA9
:10FCA00080818093BB00909193118091921129C023
:10FCB0008091700C8093BB0085EC8093BC0062CF78
:10FCC0009091920C8091910C981758F5E091920CBC
:10FCD00081E08E0F8093920CF0E0EF58F34F80811B
:10FCE000E9CFE091920C81E08E0F8093920C80918D
:10FCF000BB00F0E0EF58F34F80839091920C80911D
:10FD0000910C9817C8F285E8D8CFE091920C81E069
:10FD10008E0F8093920C8091BB00F0E0EF58F34F70
:10FD200080838091940C81115CCF81E080936F0C73
:10FD300084EA8093BC001092950C24CF85EC8093CC
:10FD4000BC001092950C8091B411803230F4E09197
:10FD5000B411F0E0EC56FE4E10826091B41170E0E8
:10FD6000E091A712F091A81284E991E119951092FF
:10FD7000B41108CF1092930C34CFCF93DF93EC01E2
:10FD800080916B11811109C081E080936B1180918A
:10FD9000E50D9091E60D0E94DD0960E08C81DF9118
:10FDA000CF910C94D87661E0FC0184810E94D876D2
:10FDB00080916B11882321F010926B110C94DC0957
:10FDC00008958FEF0C946F090F931F93CF93DF93D8
:10FDD000EC010E944F788B010E94E17E8F3F69F019
:10FDE0000E944F78601B710B6C177D07A8F380E0B1
:10FDF000DF91CF911F910F91089581E0F9CF8F92FC
:10FE00009F92AF92BF92FF920F931F93CF93DF9376
:10FE1000EC01F62E49015A018E81882389F08F81E9
:10FE200098859C012F5F3F4F38872F838230924007
:10FE300018F40E94E17EF3CFCE010E94D37E1E8291
:10FE4000CE010E94BD7E8CE291E00E94E47E8F2D67
:10FE500080640E946F0908E110E0D501C401002E02
:10FE600004C0B695A795979587950A94D2F70E94F6
:10FE70006F0908501109083F8FEF180771F785E9DE
:10FE8000FF2021F028E087E8F2128FEF0E946F092F
:10FE900010E00E94E17E8A8787FF04C01F3F11F0B7
:10FEA0001F5FF7CFDF91CF911F910F91FF90BF9010
:10FEB000AF909F908F900895AF92BF92CF92DF92B4
:10FEC000EF92FF920F931F93CF93DF93EC016901A1
:10FED000C801820F931F8130924050F58E81882394
:10FEE00079F088819981AA81BB8184179507A6073B
:10FEF000B70731F48F819885C816D90608F042C03B
:10FF0000488359836A837B838B85833039F089E00A
:10FF1000440F551F661F771F8A95D1F79A01AB01D1
:10FF200061E1CE010E94FF7E882389F083E08D830A
:10FF3000CE010E94D37E80E0DF91CF911F910F917F
:10FF4000FF90EF90DF90CF90BF90AF9008950E9408
:10FF50004F785B010E94E17E8A878F3F69F40E949F
:10FF60004F786A197B096D327140A0F38FE08D8361
:10FF7000CE010E94D37EDCCF8E3F89F418861F828B
:10FF800081E08E838F8198858C159D0550F40E94A9
:10FF9000E17E8F819885019698878F83F3CF8DE0DE
:10FFA000E6CF6701E00EF11E0E94E17EF60181932B
:10FFB0006F01EE15FF05C1F78F819885080F191F96
:10FFC00018870F838985882319F001151240A0F046
:10FFD0008E81882389F08F8198859C012F5F3F4F08
:10FFE00038872F838230924018F40E94E17EF3CF4D
:10FFF000CE010E94D37E1E8281E09ECFEF92FF92BF
:020000021000EC
:100000000F931F93CF93DF93EC01790182E14115A8
:1000100051056105710599F08B85833039F089E0D0
:10002000440F551F661F771F8A95D1F79A01AB01C0
:1000300068E1CE010E94FF7E882319F084E08D8361
:1000400030C08EEF0E946F0987018EEFF81AF80119
:1000500081918F010E946F090E151F05C1F78FEF67
:100060000E946F098FEF0E946F090E94E17E8A87CC
:100070008F71853089F488E592E00E94E47E8823C0
:10008000A9F020E030E0A9016DE0CE010E94FF7EE2
:10009000882371F084E1D3CF81E18D83CE010E946A
:1000A000D37ECE010E94D37E80E00AC085E1C7CF17
:1000B0000E94E17E8111EECFCE010E94D37E81E0CD
:1000C000DF91CF911F910F91FF90EF900895CF9303
:1000D000DF9380916C118823A9F1C091AB14D0916A
:1000E000AC1440916A0250916B0260916C02709165
:1000F0006D022BEA32E1CE010E94FE7F811104C025
:1001000080E0DF91CF91089540916D1150916E1173
:1001100060916F1170917011411551056105710564
:1001200079F02BEA32E1CE010E94FE7F882341F371
:1001300010926D1110926E1110926F111092701139
:1001400010926C1181E0DDCF8F929F92AF92BF929F
:10015000EF92FF920F931F93CF934B015C01C42F3B
:1001600080916A0290916B02A0916C02B0916D0235
:1001700088159905AA05BB0549F10E946780811180
:100180000BC080E0CF911F910F91FF90EF90BF9037
:10019000AF909F908F9008958BEAE82E82E1F82E21
:1001A00000E012E030E020E0B501A4018091AB1442
:1001B0009091AC140E945C7F882319F380926A02AC
:1001C00090926B02A0926C02B0926D0240916C1101
:1001D0004C2B40936C1181E0D5CF8F929F92AF92C0
:1001E000BF92CF92DF92EF92FF92CF9327EE3DE046
:1001F0003093AC142093AB14882309F46DC040E015
:1002000060E070E0CB010E94A48081110BC080E00F
:10021000CF91FF90EF90DF90CF90BF90AF909F90E5
:100220008F900895809169148F7789F78091751464
:1002300090917614A0917714B0917814843691053A
:10024000A105B10520F3C0907114D0907214E09014
:100250007314F0907414C114D104E104F104B9F2E0
:1002600040E0C701B6010E94A480882381F28091FA
:10027000B6129091B7128115924049F6A091BB1227
:10028000AA2329F26091B9127091BA126115710511
:1002900009F4BDCF2091B812222309F4B8CFA0935E
:1002A000050E2093F70D90E080E030E0E1E0F0E013
:1002B000C82FAF01082E02C0440F551F0A94E2F761
:1002C0002417350769F041E0480F01968930910500
:1002D00079F74093000E9BCFC12CD12C7601C0CF73
:1002E0008093000E2091C1123091C21250E040E084
:1002F0002115310541F42091CF123091D012409157
:10030000D1125091D2122093F80D3093F90D4093F1
:10031000FA0D5093FB0D46015701860E971EA11C46
:10032000B11C8092060E9092070EA092080EB09219
:10033000090EE091BC12F091BD12F0930C0EE09307
:100340000B0EB0E00E94A5A9DC01CB01880D991D20
:10035000AA1DBB1D80930D0E90930E0EA0930F0E41
:10036000B093100E25E0EE0FFF1F2A95E1F7E15044
:10037000FE4FEF2FFF27E6958E0F9F1FA11DB11D8A
:100380008093010E9093020EA093030EB093040E7F
:100390008090BE129090BF12B12CA12C81149104B8
:1003A00041F48090CB129090CC12A090CD12B090DE
:1003B000CE12C81AD90AEA0AFB0AC80CD91CEA1CD0
:1003C000FB1C04C0F694E794D794C794CA95D2F75F
:1003D000C092FC0DD092FD0DE092FE0DF092FF0D4B
:1003E00085EFC8168FE0D806E104F10428F48CE00C
:1003F00080930A0E81E00CCF80E125EFC2162FEF2B
:10040000D206E104F104A0F38091D7129091D812A2
:10041000A091D912B091DA1280930D0E90930E0E26
:10042000A0930F0EB093100E80E2E2CF4F925F9236
:100430006F927F928F929F92AF92BF92CF92DF92F4
:10044000EF92FF920F931F93CF93DF93EC01423013
:1004500051056105710590F480E0DF91CF911F9106
:100460000F91FF90EF90DF90CF90BF90AF909F9053
:100470008F907F906F905F904F90089589859A85B7
:10048000AB85BC850196A11DB11D84179507A607F4
:10049000B70710F3CB88DC88ED88FE888F89803120
:1004A00009F042C0BB27A72F962F852F480159017D
:1004B0002A013B01C80ED91EEA1EFB1E80916A026A
:1004C00090916B02A0916C02B0916D02C816D90692
:1004D000EA06FB0699F58F898031C1F5B301A201C7
:1004E000552766277727440F551F45555D4EFA015E
:1004F0009182808280916C11816080936C118A89D5
:10050000823080F08D819E81AF81B8858C0D9D1DDC
:10051000AE1DBF1D80936D1190936E11A0936F114E
:10052000B093701181E099CFDB01CA01E7E0B69585
:10053000A79597958795EA95D1F7B8CF40E0C70181
:10054000B6010E94A4808111C6CF86CFB301A2015B
:100550004F77552766277727440F551F440F551FA0
:1005600045555D4EFA0180829182A282B382C2CF4C
:100570008F929F92AF92BF92CF92DF92EF92FF92B3
:100580000F931F93CF93DF93FC0181859285A38501
:10059000B4850196A11DB11D84179507A607B7075D
:1005A00070F480E0DF91CF911F910F91FF90EF9059
:1005B000DF90CF90BF90AF909F908F9008958388E9
:1005C0009488A588B6888789803189F5BB27A72FAD
:1005D000962F852FE9016A017B018F01BC01CD01B6
:1005E000680D791D8A1D9B1D80906A0290906B0298
:1005F000A0906C02B0906D0286169706A806B90608
:1006000001F5F8018789803111F5DD24EE24FF24FE
:10061000F601EE0FFF1FE555FD4E80819181B0E0A0
:10062000A0E088839983AA83BB8381E0BBCFDB01F1
:10063000CA01C7E0B695A79597958795CA95D1F752
:10064000C9CF40E00E94A4808111DBCFAACFE894FB
:10065000C7F8DD24EE24FF24F601EE0FFF1FEE0F96
:10066000FF1FE555FD4E80819181A281B381BF704E
:10067000D8CF4F925F926F927F92AF92BF92CF92FC
:10068000DF92EF92FF920F931F93CF93DF9300D0EF
:100690001F92CDB7DEB78C0149835A836B837C836D
:1006A0005901C12CD12C7601412C82E0582E612CAD
:1006B000712C49815A816B817C819E012F5F3F4F54
:1006C000C8010E94B882882339F1F8018585A30109
:1006D000920104C0220F331F441F551F8A95D2F781
:1006E000DA01C901C80ED91EEA1EFB1E49815A81D2
:1006F0006B817C818789803111F188EF9FEFAFEFAB
:10070000BFE0481759076A077B0798F2F501C082D6
:10071000D182E282F38281E00F900F900F900F90D0
:10072000DF91CF911F910F91FF90EF90DF90CF90CD
:10073000BF90AF907F906F905F904F90089588EF3B
:100740009FEFA0E0B0E0DDCF8F929F92AF92BF927B
:10075000CF92DF92EF92FF920F931F93CF93DF938D
:10076000EC018D8181110EC080E0DF91CF911F914E
:100770000F91FF90EF90DF90CF90BF90AF909F9040
:100780008F9008950B891C892D893E8904171507C0
:100790002607370748F34A015B01823031F48A8625
:1007A0009B86AC86BD8681E0E0CF81149104A104D4
:1007B000B10449F41E821F82188619861A861B8688
:1007C0001C861D86F0CF0A851B852C853D85EB8D0B
:1007D000FC8D858590E00996B901A8014150510929
:1007E00061097109082E04C076956795579547955C
:1007F0000A94D2F775016401E1E0CE1AD108E1084C
:10080000F10804C0F694E794D794C7948A95D2F778
:10081000C416D506E606F70620F0012B022B032BA3
:1008200011F58F89988DA98DBA8D8E839F83A887A6
:10083000B9878E010A5F1F4FC114D104E104F1048E
:1008400009F4ADCF4E815F816885798598018B8DE4
:100850009C8D0E94B88291E0C91AD108E108F10884
:100860008111EACF81CFC41AD50AE60AF70AE1CF8F
:100870003F924F925F926F927F928F929F92AF9230
:10088000BF92CF92DF92EF92FF920F931F93CF937D
:10089000DF93CDB7DEB72C970FB6F894DEBF0FBE4F
:1008A000CDBF5C01DC015B968D909C905C971696A9
:1008B0004D905D906D907C901997411451046104A6
:1008C000710409F468C0BFEF4B1A5B0A6B0A7B0A1C
:1008D000312CF40181859285A385B4859C01AD01FD
:1008E0002F5F3F4F4F4F5F4F29873A874B875C877A
:1008F000730162011D821E821F821886F4018185A8
:100900009285A385B4852D813E814F815885281716
:1009100039074A075B0708F056C089859A85AB8579
:10092000BC858C159D05AE05BF0550F482E0C82E30
:10093000D12CE12CF12C92E0492E512C612C712C00
:100940009E012F5F3F4FB701A601C4010E94B882EC
:100950008823C9F189819A81AB81BC81892B8A2B3B
:100960008B2B09F1260137019FEF491A590A690AB1
:10097000790A2D813E814F8158852F5F3F4F4F4F20
:100980005F4F2D833E834F8358873FEFC31AD30AAF
:10099000E30AF30AB3CFF401408051806280738090
:1009A0003324339496CFC414D504E604F70409F72E
:1009B0000FEF1FEF2FEF3FE0B701A601C4010E9428
:1009C0001682811119C080E02C960FB6F894DEBF14
:1009D0000FBECDBFDF91CF911F910F91FF90EF9090
:1009E000DF90CF90BF90AF909F908F907F906F904F
:1009F0005F904F903F900895F50146815781608543
:100A00007185411551056105710539F09701860120
:100A1000C4010E9416828823B1F2D5011696CD92A8
:100A2000DD92ED92FC921997332051F0D701C60167
:100A30000196A11DB11DF40180839183A283B3832C
:100A4000F5018789908DA18DB28D892B8A2B8B2BF7
:100A500039F4C78AD08EE18EF28E848180688483D7
:100A600081E0B2CF2F923F924F925F926F927F922E
:100A70008F929F92AF92BF92CF92DF92EF92FF92AE
:100A80000F931F93CF93DF93EC015B012A018D81BC
:100A9000811115C08FEF9FEFDF91CF911F910F91C3
:100AA000FF90EF90DF90CF90BF90AF909F908F908E
:100AB0007F906F905F904F903F902F9008958C8122
:100AC00080FFE8CF0B891C892D893E894A855B858B
:100AD0006C857D85C201B0E0A0E068017901C41A8F
:100AE000D50AE60AF70AC816D906EA06FB0618F47C
:100AF0002801441A550A42011E0126E0220E311C2B
:100B00008114910409F4B3C04A855B856C857D85A9
:100B10006A0181E0D8228B8D9C8D8A019B01E9E0DE
:100B20003695279517950795EA95D1F7ED81E2302F
:100B3000E1F5FC01628D738D848D958D600F711FC1
:100B4000821F931F612C22E0722E6C187D08861480
:100B5000970408F434012C8126FD04C06114F2E0EE
:100B60007F0671F400916A0210916B0220916C0271
:100B700030916D02061717072807390709F053C08F
:100B800040E00E94A480882309F484CFC6018555E3
:100B90009D4ED5019C01260D371DFC012E173F07E8
:100BA00009F460C041914D93F9CFFC0174807A94AF
:100BB0007022C114D10471F471100CC0452B462B66
:100BC000472B39F58F89988DA98DBA8D8E839F8398
:100BD000A887B987EB8DFC8D6E817F81888599858B
:100BE0006250710981099109258504C0660F771F3C
:100BF000881F991F2A95D2F7068517852089318984
:100C0000600F711F821F931F670D711D811D911D44
:100C100099CF4E815F816885798591010E94B88264
:100C20008111D8CF37CF750183019601AB01BC018B
:100C30008091AB149091AC140E945C7F882309F4DE
:100C400029CFA60CB71C8A859B85AC85BD85860DF2
:100C5000971DA11DB11D8A879B87AC87BD8786180C
:100C600097084ECF281B390BA20EB31EECCFC20142
:100C700013CFCF93DF931F92CDB7DEB741E050E0A3
:100C8000BE016F5F7F4F0E943285019731F48981E9
:100C900090E00F90DF91CF9108958FEF9FEFF9CF04
:100CA000FC01818D928D009711F00C9439868FEFA5
:100CB0009FEF08950F931F93CF93DF93EC01898DDE
:100CC0009A8D10E000E0009799F00E9439868C011F
:100CD0000F3F100769F0898D9A8DFC01428553857D
:100CE0006485758541505109610971090E94A48389
:100CF000C801DF91CF911F910F910895CF93DF939A
:100D0000EC018D81882389F18C8187FF2AC06E8553
:100D10007F858889998941E00E94A480882329F1F0
:100D2000EA8980E2E89FF0011124E555FD4E3097F5
:100D3000E1F08D81823040F48B899C89AD89BE8938
:100D4000848F958FA68FB78F8F89988D938F828F81
:100D50008F89988DA98DBA8DB58BA48B8C818F7757
:100D60008C83DF91CF910C94678080E0DF91CF91ED
:100D70000895CF92DF92EF92FF921F93CF93DF936C
:100D8000EC0180E2689FF0011124E555FD4E93854A
:100D9000917161F0842F827449F080E0DF91CF91EE
:100DA0001F91FF90EF90DF90CF900895142F6A8BE2
:100DB00080916A0290916B02A0916C02B0916D02D9
:100DC0008E879F87A88BB98BC488D588F12CE12C9E
:100DD0007601DD24CC24CF8AD88EE98EFA8E828DDE
:100DE000938DB0E0A0E0AC01BD014C295D296E29D6
:100DF0007F294F8B588F698F7A8F83858871B1F4E3
:100E0000848D958DA68DB78D8B8B9C8BAD8BBE8B7A
:100E100081E08D831F701C831E821F8218861986B5
:100E20001A861B861C861D8681E0B8CF803109F0AA
:100E3000B4CF9E012D5E3F4F8B8D9C8D0E943983D8
:100E4000882309F4AACF84E0E4CFCF93DF93EC01A9
:100E50000E947E86882311F01D8281E0DF91CF9170
:100E60000895FC01818D928D009711F00C947E867F
:100E700008953F924F925F926F927F928F929F92CE
:100E8000AF92BF92CF92DF92EF92FF920F931F9398
:100E9000CF93DF9300D000D000D01F921F92CDB728
:100EA000DEB77C01DC0115968C91811115C0FE0125
:100EB0003196CE010C966F0130E23193E817F907B5
:100EC000E1F7DA0130E087E09D91B92E992329F10D
:100ED0009E3239F48A3011F480E0E3C038E08AE0D1
:100EE000F3CFE0E1FCE04491442321F031969413E8
:100EF000FACFF2CF831780F34FED490F4E3560F7ED
:100F00004FE9490F4A3118F440EEB42EB90EF601FC
:100F1000E30FF11DB0823F5FD7CF89818032E1F2CC
:100F2000322E8B01FB01838D948DD7015C969C93AF
:100F30008E935B971682178210861186128613860F
:100F400014861586F80182859385A485B585438925
:100F500054896589768984179507A607B70708F02D
:100F60004DC025E0B695A795979587952A95D1F719
:100F7000F82FFF70AF2ED80115968C91823008F4AF
:100F8000ABCFC8010E94398697FDA6CFF8018285B4
:100F90009385A485B5854F96A11DB11D8287938742
:100FA000A487B587F0E2AF9EB001112465557D4E50
:100FB0006115710509F490CFDB018C91882341F014
:100FC000853E09F061C0BB2029F0BB24B394BACFA1
:100FD000B1100EC0F701A28A80916A0290916B0253
:100FE000A0916C02B0916D0286879787A08BB18B20
:100FF000DB018C918111E9CFBB24B394832D8271E5
:10100000823109F069CFBB2009F463C0F70166851E
:1010100077858089918941E00E94A480882309F422
:101020005BCFD70152968C91B0E28B9FC001112407
:1010300085559D4E009709F44FCFFC013A9626E165
:10104000DF011D922A95E9F72BE0F601DC01019002
:101050000D922A95E1F721E238E2FC01318B208BD9
:1010600040E058E057874687338B228B318F208FA3
:10107000578B468B0E946780882309F42DCF432D20
:10108000D70152966C910AC04BE050E0C6010E9415
:1010900030AD892B09F056CF432D6A2DC7010E9430
:1010A000B9862B960FB6F894DEBF0FBECDBFDF9189
:1010B000CF911F910F91FF90EF90DF90CF90BF9055
:1010C000AF909F908F907F906F905F904F903F90E8
:1010D0000895F8018581823009F4FECEC8010E948E
:1010E0003884882309F4F8CED8015B96ED91FC9101
:1010F0005C9716968D909D90AD90BC901997B2E03C
:101100008B1A9108A108B108858504C0880C991C28
:10111000AA1CBB1C8A95D2F786859785A089B189C0
:10112000880E991EAA1EBB1E848124013501480E1B
:10113000511C611C711C84149504A604B70401F1B0
:10114000E1E04E1A5108610871080E946780882307
:1011500009F4C2CEEBEAF2E111928BEA94E18E1728
:101160009F07D1F740926A0250926B0260926C0224
:1011700070926D0280916C11816080936C11DBCF55
:10118000D8015B96ED91FC91258580E092E0A0E08E
:10119000B0E004C0880F991FAA1FBB1F2A95D2F781
:1011A000F8014389548965897689840F951FA61FA4
:1011B000B71F838B948BA58BB68BD70152961C924D
:1011C0008BEA92E13ACF2F923F924F925F926F92C9
:1011D0007F928F929F92AF92BF92CF92DF92EF92C7
:1011E000FF920F931F93CF93DF9300D01F92CDB741
:1011F000DEB78C015B011A01DC0115968C91159705
:10120000813009F0C8C014968C9181FFC4C082FD62
:10121000AEC06101D8011A964D915D916D917C919E
:101220001D97C114D10409F429C15B968D919C913D
:101230005C97FC0174802FEF270D2A013B0139E0F8
:1012400076946794579447943A95D1F7722E742008
:101250007A01F1E0FF22711020C0E114F104E9F4F9
:1012600016964D915D916D917C911997411551059F
:101270006105710509F098C057968D919D910D906B
:10128000BC91A02D0097A105B10509F0AFC0C80120
:101290000E943884882309F47EC080E092E08E1991
:1012A0009F0946018C159D0508F44C01D8015B96F9
:1012B0004D915C915C9716968D919D910D90BC918E
:1012C000A02D0297A109B109FA01258504C0880F54
:1012D000991FAA1FBB1F2A95D2F74685578560899B
:1012E0007189840F951FA61FB71F9C01AD01270DA3
:1012F000311D411D511D29013A01811432E093062F
:1013000009F07AC080916A0290916B02A0916C0200
:10131000B0916D0284159505A605B70559F48FEFB8
:101320009FEFDC0180936A0290936B02A0936C02A2
:10133000B0936D029501B301A2018091AB1490911D
:10134000AC140E94FE7F882331F19EEFB91AC818B1
:10135000D908F80182859385A485B585880D991DE6
:10136000A11DB11D82879387A487B58753CFF8014C
:10137000438954896589768982859385A485B58555
:10138000481759076A077B0709F443CFC8010E9431
:10139000A48381113ECF81E090E0D80113969C9305
:1013A0008E93129780E007C09E012F5F3F4F0E94EF
:1013B000B882811102C090E077C089819A81AB81A7
:1013C000BC81F801238D348DF901278948EF5FEF47
:1013D00060E070E0203121F048EF5FEF6FEF7FE0D9
:1013E00084179507A607B70708F051CFF801868341
:1013F0009783A087B18751CFE114F10491F5D8010B
:101400001A964D915D916D917C911D9753968D919A
:101410009D910D90BC91A02D481759076A077B0735
:1014200000F10E946780882309F4B5CF40926A02D8
:1014300050926B0260926C0270926D0280916C11FE
:10144000816080936C11970125553D4ED501C901EE
:10145000880D991DF9018E179F0759F04D91419301
:10146000FACF41E0C301B2010E94A4808111EBCF09
:1014700092CF821B930BA80EB91E69CFF801838906
:101480009489A589B68984179507A607B70738F404
:101490008481438B548B658B768B80688483F801C1
:1014A000848183FD18C0C1010F900F900F900F90A1
:1014B000DF91CF911F910F91FF90EF90DF90CF9030
:1014C000BF90AF909F908F907F906F905F904F9064
:1014D0003F902F900895C8010E947E86882309F4CA
:1014E0005ACFE1CFCF93DF931F92CDB7DEB7698399
:1014F00041E050E0BE016F5F7F4F0E94E3880F9094
:10150000DF91CF910895CF93DF93EC01E98DFA8DB0
:10151000309749F481E090E09B838A8390E080E0FB
:10152000DF91CF91089513821282898D9A8D0E9446
:10153000E388E98DFA8D22813381232B59F7F0CF8F
:10154000FC01DB0112968D919C911397938382830A
:1015500085E893E09183808314968C91149784831B
:1015600015968C911597858316964D915D916D9189
:101570007C91199746835783608771871A964D919E
:101580005D916D917C911D97428753876487758724
:101590001E964D915D916D917C915197468757872D
:1015A000608B718B52968C915297828B53964D9192
:1015B0005D916D917C915697438B548B658B768BA7
:1015C00057964D915D916D917C915A97478B508FB5
:1015D000618F728F5B968D919C91948F838F08950C
:1015E000DC015996ED91FC91309721F081E09581D5
:1015F000911101C080E00895CF93DF93EC01898DB4
:101600009A8D009741F00E942587898D9A8D0E94BE
:10161000B9AB1A8E198EDF91CF910895EF92FF9298
:101620000F931F93CF93DF93EC017B018A011B8201
:101630001A8288EE93E0A0E0B0E08C839D83AE83B5
:10164000BF8389EF93E0998388838DE190E00E94C6
:101650001DAB9A8F898F009779F02DE1F701DC019E
:1016600001900D922A95E1F74CE050E0B801CE01CF
:101670000C960E9488AD188EDF91CF911F910F912B
:10168000FF90EF9008952F923F924F925F926F924A
:101690007F928F929F92AF92BF92CF92DF92EF9202
:1016A000FF920F931F93CF93DF93CDB7DEB7C7564B
:1016B000D1090FB6F894DEBF0FBECDBF5C013B0170
:1016C000A6964FAFA6974E018EE1880E911C61E160
:1016D0007EE0C4010E94A08A1C821B8285E893E000
:1016E0009A8389831E8263018E010F5F1F4F24013D
:1016F00018016FE270E0C6010E945FAD009709F427
:1017000059C0F60120812F3271F4FFEFCF1ADF0AA2
:10171000902F812F8201492E582E942D852D28013E
:10172000092F182FE6CF8C198D3008F08CE0E82EA9
:10173000F12CA701B601CE01885A9F4F0E9488ADB7
:10174000E8E5F0E0EC0FFD1FEE0DFF1D1082C80173
:101750000E94258721E0AE01485A5F4FB201C801BF
:101760000E943987811120C01EAE1DAE85E893E02E
:101770009CAF8BAF21961FAE2197A896EEADFFAD23
:10178000A8976E0E7F1EF3018081811120C0BE01DB
:10179000655C7F4FC1010E94A08A4AE654E0B10116
:1017A000C5010E940E8B31C0CE0CDF1CC2010E940D
:1017B0002587B3CFC60186199709A8969FAF8EAF2C
:1017C000A897B201CE01CB960E94A08AD6CF19A2CB
:1017D00018A285E893E09F8F8E8F1BA221968FAD74
:1017E000219781112DC0F5011382128288EE93E0BA
:1017F000A0E0B0E084839583A683B78389EF93E06C
:1018000091838083128E118E1486C501C959DF4FD2
:101810000FB6F894DEBF0FBECDBFDF91CF911F9101
:101820000F91FF90EF90DF90CF90BF90AF909F907F
:101830008F907F906F905F904F903F902F90089582
:101840008250A6962FADA697A3018230C8F461E11D
:101850007EE0C4010E943987882329F2A6968FADC5
:10186000A697867039F049A95AA96BA97CA9C40129
:101870000E94A483B401C1010E94A08AA3018FCF5A
:10188000BE01655C7F4FC4010E943987882309F43B
:10189000AACFCE01CB960E942587E0CF0F931F934E
:1018A000CF93DF93CDB7DEB7AD970FB6F894DEBF19
:1018B0000FBECDBF80915A0C882331F08091750FF7
:1018C0009091760F892B11F40E942F6063EC78E0E1
:1018D000CE0188960E948D748091590C8823E1F086
:1018E00063EA7DE0CE0101960E947B74CE010196F1
:1018F0000E94F815CE0101960E94EE7368E972E02D
:10190000CE0101960E948D74CE0101960E94E115D0
:10191000CE0101960E94EE7380915A0C81111BC07A
:101920008091580C81117BC08091570C882309F459
:1019300049C10FE110E08091560C882309F4BAC028
:101940000150110909F45CC064E170E080E090E0AE
:101950000E949177F0CF8091750F9091760F892B2F
:10196000F9F264E170E080E090E00E94917765E92F
:101970007DE0CE0188960E94797361E77FE0CE0119
:1019800001960E948474AE014F5F5F4F63E070E088
:1019900088E992E00E943426182FCE0101960E9419
:1019A000EE73111127C0BE01685D7F4FCE014C96CA
:1019B0000E94847463E57FE0CE014C960E94097317
:1019C000BC01CE0101960E948474CE0101960E9452
:1019D000E115CE0101960E94EE73CE014C960E9455
:1019E000EE73809113159091141501969093141530
:1019F0008093131510925A0C8091580C811190CF3E
:101A0000CE0188960E94EE73AD960FB6F894DEBFB5
:101A10000FBECDBFDF91CF911F910F91089580919F
:101A2000690F90916A0F892B09F47ECF67E87DE0FA
:101A3000CE0188960E94797365E67FE0CE0101961B
:101A40000E948474AE014F5F5F4F62E070E082EBF2
:101A500092E00E943426182FCE0101960E94EE7368
:101A6000111162CFBE01685D7F4FCE014C960E947E
:101A7000847463E57FE0CE014C960E940973BC013B
:101A8000CE0101960E948474CE0101960E94E11558
:101A9000CE0101960E94EE73CE014C960E94EE7329
:101AA00080911315909114150196909314158093BD
:101AB00013153ACF43E165EA72E0CE0101960E9428
:101AC000438BBE016F5F7F4F8DE391E10E94081948
:101AD00081E08093560C8DE391E10E94F08A882387
:101AE000E1F161E77FE08DE391E10E94D4758DE340
:101AF00091E10E94FC8A62E370E080E090E00E9445
:101B000091771092560C8091590C882331F1CE01B7
:101B10004C960E947A1B6EE679E0CE0182960E9476
:101B20008D74BE01645E7F4FCE0182960E94097360
:101B3000BC01CE0101960E948474CE0101960E94E0
:101B4000E115CE0101960E94EE73CE0182960E94AD
:101B5000EE73CE014C960E94EE738DE391E10E94EC
:101B6000FC8A62E370E080E090E00E94917710923E
:101B7000560C43E162EB72E0CE0101960E94438B6A
:101B8000BE016F5F7F4F8DE391E10E94081981E0F4
:101B90008093560C8DE391E10E94F08A882331F006
:101BA00065E67FE08DE391E10E94D4758DE391E1DC
:101BB0000E94FC8A62E370E080E090E00E949177EE
:101BC0001092560C63EC78E085E69FE00E94D1719C
:101BD00063EC78E081E79FE00E94D17111CFCF9252
:101BE000DF92EF92FF920F931F93CF93DF93EC015D
:101BF0007A018B016C01C40ED51ECC15DD05A1F058
:101C00000E946D0980EF0E946F098D2F0E946F095D
